:020000040000FA
:04000000ACEF00F071
:100008005582D9CF05F0DACF06F00F0112A91BD01F
:100018008EBC02D0839483928EA802D083A20ED085
:10002800899424EE04F0010EDBBE07D0000EDE5CDE
:10003800020EDE5802E3899201D089828EB883B21B
:1000480001D08984129912A17BD08EB883B289928B
:10005800901C086E8E1C076E04C409F005C40AF0D3
:100068000ABE03D0020E0A5C2FE28EA802D083A239
:100078002BD0094A0A2A09C004F40AC005F402C4AC
:1000880009F003C40AF0060E0924D96E040E0A20EA
:10009800DA6E08C0DFFF060E0924D96E060E0A20A4
:1000A800DA6E07C0DFFF094A0A2A0168010E026EEC
:1000B80009C003F00AC004F00150031602500416E8
:1000C80003C002F404C003F48EB883B2898489841F
:1000D8008EA0FED78EA802D083A202D0899401D028
:1000E800898424EE04F0010EDBBE07D0000EDE5C2E
:1000F800020EDE5802E3899201D0898207A81ED039
:100108000BD0838202D0838405D0839417D083A236
:1001180015D08394839212D00850016E026A02505F
:100128000DE10150040AF3E0100AF1E0340AE9E0B5
:100138001F0AF0E07F0AE7E01F0AE7E00F011291CB
:100148000E01CA9906C0DAFF05C0D9FF5592110001
:10015800EDEF4EF07CC0D9FF7DC0DAFFDE6ADD6AC4
:100168007EC00BF068EC4BF00BC0B6F00CC0B7F0DB
:100178000001B7BF0B0CD890B635D96EB735DA6E1B
:100188008C0ED926010EDA22DECFD0F0DDCFD1F0E9
:10019800D051D11101E10C0C7CC0D9FF7DC0DAFF30
:1001A800D0C0DEFFD1C0DDFFD0C0D9FFD1C0DAFF9B
:1001B800DF5012E020EE01F0D051D926D151DA22D9
:1001C800DF50B3EC5DF00001C26FC2B105D07F51C2
:1001D800D8A4C2A5000C0A0CD0C0D9FFD1C0DAFF40
:1001E800DF6A20EE01F0D051D926D151DA22B6C00B
:1001F800DFFF20EE01F0D051D926D151DA22DF50AD
:100208008AEC47F00001C26FC2B1030C7F5102E0D3
:10021800C2B50A0CC96BCA6BCB6BCC6BD0C044F0AF
:10022800D1C045F0C9C046F0CAC047F0CBC048F0BD
:10023800CCC049F0D1EC41F00001CF6FCF0501E00F
:10024800D4D0CD6BCE6BCE5105E1040ECD5D01E36C
:1002580090D001D08ED0CDC080F0CEC081F0803B50
:10026800813BF00E811780510F0B8113F00E801720
:10027800D0C082F0D1C083F080518227815183237E
:10028800EC0E8225C36F010E8321C46F20EE04F0AB
:10029800C351D926C451DA22DF5005E1A86BA96BF6
:1002A800AA6BAB6B55D020EE09F0C351D926C451C7
:1002B800DA22DF50816F806B20EE0AF0C351D92615
:1002C800C451DA22DF50826F82C083F0846B856B61
:1002D800866B84C086F083C085F0846B836B20EEC8
:1002E8000BF0C351D926C451DA22DF50876F87C07B
:1002F80088F0896B8A6B8B6B88C08BF08A6B896BF3
:10030800886B835188118C6F845189118D6F855149
:100318008A118E6F86518B118F6F80518C11906F5F
:1003280081518D11916F000E8E11926F000E8F11F9
:10033800936F20EE08F0C351D926C451DA22DF505A
:100348009011A86F9151A96F9251AA6F9351AB6FF9
:10035800CD51040DF350980FD96EDA6AA8C0DEFFAC
:10036800A9C0DEFFAAC0DEFFABC0DEFFCD4BCE2B9F
:100378006AD7CD6BCE6BCD51CE1103E0CD07D8A097
:10038800CE07CD51040DF350980FD96EDA6ADECF3F
:10039800C9F0DECFCAF0DECFCBF0DECFCCF0C9514A
:1003A800CA11CB11CC1105E1000EAD6F020EAC6F76
:1003B80011D0D0C044F0D1C045F0C9C046F0CAC081
:1003C80047F0CBC048F0CCC049F0D1EC41F0000177
:1003D800AC6FAD6BACC0CFF0CF5107E0CD4BCE2B9F
:1003E800CE5103E1040ECD5DCCE3030ECF1901E13C
:1003F800010CCF5101E00D0C20EE3AF0D051D92676
:10040800D151DA22DF50816F806B20EE39F0D05164
:10041800D926D151DA22DF508013020E81198011BA
:1004280001E00D0C20EE45F0D051D926D151DA2249
:10043800DF50816F806B20EE44F0D051D926D15126
:10044800DA22DF50801380C0C5F081C0C6F0C76BC8
:10045800C86BC551C611C711C81155E120EE53F03C
:10046800D051D926D151DA22DF50816F806B20EE2E
:1004780054F0D051D926D151DA22DF50826F82C090
:1004880083F0846B856B866B84C086F083C085F0AF
:10049800846B836B20EE55F0D051D926D151DA22E6
:1004A800DF50876F87C088F0896B8A6B8B6B88C039
:1004B8008BF08A6B896B886B835188118C6F8451A0
:1004C80089118D6F85518A118E6F86518B118F6FAF
:1004D80080518C11906F81518D11916F000E8E118A
:1004E800926F000E8F11936F20EE52F0D051D926E3
:1004F800D151DA22DF509011C56F9151C66F9251D8
:10050800C76F9351C86F20EE16F0D051D926D1513C
:10051800DA22C5C0DEFFC6C0DEFFC7C0DEFFC8C026
:10052800DEFF20EE3EF0D051D926D151DA2210EE6E
:1005380003F0D051E126D151E222DFCFE7FF20EED0
:1005480003F0D051D926D151DA22DE040AE020EE98
:1005580003F0D051D926D151DA22020EDE1801E07B
:100568000D0CC5C00BF0C6C00CF0C7C00DF0C8C05C
:100578000EF020EE03F0D051D926D151DA22DF5007
:100588000F6E106A116A126A9FEC54F00BC0C5F026
:100598000CC0C6F00DC0C7F00EC0C8F020EE3BF08E
:1005A800D051D926D151DA2210EE02F0D051E126ED
:1005B800D151E222DFCFE7FF20EE02F0D051D92659
:1005C800D151DA22DF50D8B40D0C20EE02F0D05110
:1005D800D926D151DA22DF50806F20EE02F0D051B7
:1005E800D926D151DA22DF50816F8105801501E0CB
:1005F8000D0C20EE40F0D051D926D151DA22DF502F
:10060800816F806B20EE3FF0D051D926D151DA228C
:10061800DF50801320EE08F0D051D926D151DA22CC
:1006280080C0DEFF81C0DDFF20EE08F0D051D92662
:10063800D151DA22DF50806F0F0E801701E00D0CC8
:1006480020EE42F0D051D926D151DA22DF50816F05
:10065800806B20EE41F0D051D926D151DA22DF50FB
:10066800801380C0BAF081C0BBF0BC6BBD6BBA51BF
:10067800BB11BC11BD1155E120EE4FF0D051D92668
:10068800D151DA22DF50816F806B20EE50F0D051CB
:10069800D926D151DA22DF50826F82C083F0846B71
:1006A800856B866B84C086F083C085F0846B836B12
:1006B80020EE51F0D051D926D151DA22DF50876F80
:1006C80087C088F0896B8A6B8B6B88C08BF08A6BCC
:1006D800896B886B835188118C6F845189118D6F58
:1006E80085518A118E6F86518B118F6F80518C11B5
:1006F800906F81518D11916F000E8E11926F000EC7
:100708008F11936F20EE4EF0D051D926D151DA22B5
:10071800DF509011BA6F9151BB6F9251BC6F9351DA
:10072800BD6F20EE3CF0D051D926D151DA22DF50EE
:10073800806F20EE3DF0D051D926D151DA22DF501A
:10074800816F8051B86F81C0B9F0B851B91101E11A
:100758000D0C20EE08F0D051D926D151DA22DECF87
:1007680080F0DDCF81F0040E826FD8908133803322
:10077800822FFBD7B8518025836FB9518121846FAF
:10078800856BD8B0852B866BC5518325B26FC65152
:100798008421B36FC7518521B46FC8518621B56FC5
:1007A800B251BA5DB351BB59B451BC59B551BD59D9
:1007B80001E20D0CB251BA5D0B6EB351BB590C6E10
:1007C800B451BC590D6EB551BD590E6E20EE02F0F4
:1007D800D051D926D151DA22DF500F6E106A116A32
:1007E800126A5BEC55F00BC0BEF00CC0BFF00DC038
:1007F800C0F00EC0C1F00001BE51BF11C011C1113F
:1008080001E10D0C010ECF6FC151C01105E1F60ECB
:10081800BE5D0F0EBF5902E3020ECF6FC151C0116A
:1008280005E1F60EBE5DFF0EBF5902E3030ECF6F62
:10083800020EBE25806F000EBF21816F000EC02101
:10084800826F000EC121836F20EE12F0D051D9269D
:10085800D151DA2280C0DEFF81C0DEFF82C0DEFF18
:1008680083C0DEFF20EE1AF0D051D926D151DA220A
:10087800C9C0DEFFCAC0DEFFCBC0DEFFCCC0DEFFD2
:10088800B851C925806FB951CA21816F000ECB219B
:10089800826F000ECC21836F20EE1EF0D051D92636
:1008A800D151DA2280C0DEFF81C0DEFF82C0DEFFC8
:1008B80083C0DEFFB251C925806FB351CA21816F51
:1008C800B451CB21826FB551CC21836F20EE26F035
:1008D800D051D926D151DA2280C0DEFF81C0DEFF97
:1008E80082C0DEFF83C0DEFF030ECF1901E08CD08B
:1008F80020EE08F0D051D926D151DA22DE50DE1090
:1009080001E00D0C20EE5BF0D051D926D151DA224E
:10091800DF50816F806B20EE5CF0D051D926D15129
:10092800DA22DF50826F82C083F0846B856B866B1E
:1009380084C086F083C085F0846B836B20EE5DF005
:10094800D051D926D151DA22DF50876F87C088F07D
:10095800896B8A6B8B6B88C08BF08A6B896B886B11
:10096800835188118C6F845189118D6F85518A113B
:100978008E6F86518B118F6F80518C11906F8151C2
:100988008D11916F000E8E11926F000E8F11936F63
:1009980020EE5AF0D051D926D151DA22DF509011E9
:1009A800946F9151956F9251966F9351976F20EE76
:1009B80022F0D051D926D151DA2294C0DEFF95C059
:1009C800DEFF96C0DEFF97C0DEFF20EE12F0D051AA
:1009D800D926D151DA22DECF80F0DECF81F0DECF0A
:1009E80082F0DECF83F0020ED890803781378237CD
:1009F8008337E82EF9D780C0AEF081C0AFF082C04F
:100A0800B0F083C0B1F0B7D020EE08F0D051D926AD
:100A1800D151DA22DE50DE1001E10D0C20EE1EF07D
:100A2800D051D926D151DA22DECF80F0DECF81F045
:100A3800DECF82F0DECF83F0C5518025846FC651AA
:100A48008121856FC7518221866FC8518321876FA5
:100A580020EE22F0D051D926D151DA2284C0DEFF0F
:100A680085C0DEFF86C0DEFF87C0DEFF020ECF191D
:100A78006BE020EE12F0D051D926D151DA22DECF28
:100A880080F0DECF81F0DECF82F0DECF83F0010E82
:100A98008015846F856B866B876B20EE12F0D051C2
:100AA800D926D151DA22DECF88F0DECF89F0DECF29
:100AB8008AF0DECF8BF0030E8803F3CF8CF0F4CFEF
:100AC8008DF08E6B8F6B8903F3508D27F4508E2336
:100AD800000E8F238803F3508D27F4508E23000EC9
:100AE8008F23030E8A03F3508E27F4508F23000EB2
:100AF8008903F3508E27F4508F23000E8803F35098
:100B08008E27F4508F23030E8B03F3508F27000E8C
:100B18008A03F3508F27000E8903F3508F27000EA6
:100B28008803F3508F27D8908F338E338D338C33CF
:100B380084518C25AE6F85518D21AF6F86518E21E2
:100B4800B06F87518F2116D020EE12F0D051D926E0
:100B5800D151DA22DECF80F0DECF81F0DECF82F015
:100B6800DECF83F0D8908035AE6F8135AF6F823598
:100B7800B06F8335B16FFF0EAE25806F010EAF21C8
:100B8800816F000EB021826F000EB121836F0A0EB3
:100B980005D0D8908333823381338033E82EF9D758
:100BA80020EE16F0D051D926D151DA228051DE5CE0
:100BB8008151DE588251DE588351DE5801E20D0C16
:100BC80020EE0EF0D051D926D151DA22DE68DE6847
:100BD800DE68DD68DD52DD5210EE0AF0D051E12604
:100BE800D151E222DECFE6FFDECFE6FFDECFE6FF21
:100BF800DECFE6FF20EE05F0D051D926D151DA221A
:100C0800800EDF6E030ECF1901E0D3D120EE5FF026
:100C1800D051D926D151DA22DF50816F806B20EE76
:100C28005EF0D051D926D151DA22DF5080138005E9
:100C3800811101E0BED1D0C039F0D1C03AF0C92944
:100C48003B6E000ECA213C6E000ECB213D6E000E9D
:100C5800CC213E6EA5EC52F0000901E0AAD10001BA
:100C680020EE05F0D051D926D151DA22DF6A22EEE2
:100C78002DF0D051D926D151DA22DF50816F806B07
:100C880022EE2CF0D051D926D151DA22DF50801330
:100C9800550E801903E1AA0E8119D8A48AD120EE35
:100CA8002FF0D051D926D151DA22DF50816F806BD5
:100CB80020EE30F0D051D926D151DA22DF50826FA0
:100CC80082C083F0846B856B866B84C086F083C09A
:100CD80085F0846B836B20EE31F0D051D926D15149
:100CE800DA22DF50876F87C088F0896B8A6B8B6B3D
:100CF80088C08BF08A6B896B886B835188118C6FE5
:100D0800845189118D6F85518A118E6F86518B118F
:100D18008F6F80518C11906F81518D11916F000EE2
:100D28008E11926F000E8F11936F20EE2EF0D0511E
:100D3800D926D151DA22DF509011946F9151956FD5
:100D48009251966F9351976F520E941909E1520E72
:100D5800951906E1610E961903E1410E9719D8A479
:100D680028D122EE13F0D051D926D151DA22DF5002
:100D7800816F806B22EE14F0D051D926D151DA223E
:100D8800DF50826F82C083F0846B856B866B84C072
:100D980086F083C085F0846B836B22EE15F0D0510A
:100DA800D926D151DA22DF50876F87C088F0896B46
:100DB8008A6B8B6B88C08BF08A6B896B886B8351CD
:100DC80088118C6F845189118D6F85518A118E6FAE
:100DD80086518B118F6F80518C11906F81518D11BD
:100DE800916F000E8E11926F000E8F11936F22EE8D
:100DF80012F0D051D926D151DA22DF509011946FD8
:100E08009151956F9251966F9351976F720E9419F5
:100E180009E1720E951906E1410E961903E1610E7A
:100E28009719D8A4C6D022EE17F0D051D926D1519F
:100E3800DA22DF50816F806B22EE18F0D051D9266C
:100E4800D151DA22DF50826F82C083F0846B856BC8
:100E5800866B84C086F083C085F0846B836B22EE3A
:100E680019F0D051D926D151DA22DF50876F87C0C7
:100E780088F0896B8A6B8B6B88C08BF08A6B896B67
:100E8800886B835188118C6F845189118D6F8551BE
:100E98008A118E6F86518B118F6F80518C11906FD4
:100EA80081518D11916F000E8E11926F000E8F116E
:100EB800936F22EE16F0D051D926D151DA22DF50A5
:100EC8009011946F9151956F9251966F9351976FBE
:100ED80020EE0EF0D051D926D151DA2294C0DEFF8F
:100EE80095C0DEFF96C0DEFF97C0DEFF22EE1BF046
:100EF800D051D926D151DA22DF50816F806B22EE92
:100F08001CF0D051D926D151DA22DF50826F82C02D
:100F180083F0846B856B866B84C086F083C085F014
:100F2800846B836B22EE1DF0D051D926D151DA2281
:100F3800DF50876F87C088F0896B8A6B8B6B88C09E
:100F48008BF08A6B896B886B835188118C6F845105
:100F580089118D6F85518A118E6F86518B118F6F14
:100F680080518C11906F81518D11916F000E8E11EF
:100F7800926F000E8F11936F22EE1AF0D051D9267E
:100F8800D151DA22DF509011946F9151956F92519F
:100F9800966F9351976F20EE0AF0D051D926D15110
:100FA800DA2294C0DEFF95C0DEFF96C0DEFF97C050
:100FB800DEFFD0C0D9FFD1C0DAFFCFC0DFFF01010B
:100FC8008A4B8B2B000120EE06F0D051D926D15147
:100FD800DA228AC1DEFF8BC1DDFF000C0C6A0B6AC6
:100FE80053EC5DF00F0B0101FE6F9B6B070E8C6ECF
:100FF800010EFD6FA06B0F0E0F01596F116B196B6E
:10100800216B266B2E6B886889688A688A8E88901F
:1010180088928382020E0101FF6F00EC5CF08894D5
:101028008384889C839C889E838E8B688968EB0E5A
:101038000001606FF40E616FA30E626FFF0E636FA5
:10104800E70E646FFE0E656F310E666FFF0E676FF9
:101058008AEC5DF08A988588CFEC5BF017D08E0E0D
:101068000001606FFE0E616F8FCF62F0636B8AECD8
:101078005DF0290E0101D96F960ED86F7F0EE82E0C
:10108800FED7D82FFCD7D92FFAD704008FB2E7D7CD
:10109800FAEC4BF00101FE6F570E0001606FFB0E7A
:1010A800616FFEC162F0636B8AEC5DF00400520E62
:1010B8000101D96F2B0ED86F000EE82EFED7D82F5E
:1010C800FCD7D92FFAD700F0010E80EC5DF0D25092
:1010D800F00B0109D26ED09E0E01C691CF0ECF162D
:1010E800CF82CF80C2890F01138113891489F28EB0
:1010F8000E01BA8925EC57F08392839408EC4EF0E0
:1011080008EC4EF0000E0B6E340E45EC59F04C0E08
:101118000F6EFF0E106EE2EC54F0A30E0F6EFF0E72
:10112800106EE2EC54F0000E0B6E390E45EC59F0DF
:101138008380040052EC2DF0F1C193FFDDEC44F004
:1011480096EC55F0000E0B6E800E45EC59F09CECB9
:101158005CF0000E0B6E800E45EC59F00101FE515B
:101168000F0D340EF3240F6E0C0EF420106EE2EC0B
:1011780054F001019A5101E1DCD0900E0001606F3A
:10118800FD0E616F8AEC5DF05CEC57F00FC0E3F187
:1011980010C0E4F111C0E5F112C0E6F10101E3511C
:1011A800E411E511E61117E1E20E0001606FFB0E94
:1011B800616FE3C162F0E4C163F0E5C164F0E6C1C8
:1011C80065F08AEC5DF00A0E0E6E000E0F6A106A6A
:1011D800116ACAEC58F00101E76BE86BE8BF05D06B
:1011E800E85119E1040EE75D16E2DC0E0001606FBC
:1011F800FF0E616FE30E0101E725D96E010EE821AC
:10120800DA6EDF500001626F636B8AEC5DF00101FA
:10121800E74BE82BE3D75E0E0001606FFC0E616FB1
:101228008AEC5DF0600E0001606FFA0E616F8AEC67
:101238005DF022EE00F000EECDF01F0EDBCFEBFFED
:10124800E806FCE2D00E0001ED6FFF0EEE6FEEEC4B
:1012580038F0CDC074F1CEC075F1CFC076F1D0C0F2
:1012680077F10101745175117611771162E0460E1C
:101278000001606FFA0E616F74C162F075C163F0AE
:1012880076C164F077C165F08AEC5DF0000E00016C
:10129800A66F020EA76F74C1D9F175C1DAF176C1D4
:1012A800DBF10101D86B000ED8250001A86F010EF3
:1012B8000101D9210001A96F000E0101DA21000105
:1012C800AA6F000E0101DB210001AB6FDFEC12F009
:1012D800000E846F020E856F340E866F0A0E876FBC
:1012E800896B080E886FE00E8A6F010E8B6FC9EC50
:1012F80015F00101E96BEA6BEABF05D0EA5119E183
:10130800080EE95D16E2D80E0001606FFF0E616FEE
:10131800340E0101E925D96E0A0EEA21DA6EDF5092
:101328000001626F636B8AEC5DF00101E94BEA2B07
:10133800E3D7A0AF12D08A6883928382290E010175
:10134800D96F960ED86F7F0EE82EFED7D82FFCD710
:10135800D92FFAD7D6EC45F0EFD7FD5104E0020EAD
:101368009F6F2D0E0BD0A00E0001606FFD0E616FF8
:101378008AEC5DF0010E01019F6F040E9E6FDC6B1D
:10138800DD6BEE6B000EEC6F010EEB6FECBF05D062
:10139800EC5168E1040EEB5D65E20F0EEB03F3CF51
:1013A800D8F1F4CFD9F1EC03F350D927240ED8257E
:1013B8000B6E0D0ED9210C6E3AEC5AF00C5003E16D
:1013C800030E0B5C4BE3FD0E0001606FFD0E616FB9
:1013D8000F0E0101EB03F3CFD8F1F4CFD9F1EC03F1
:1013E800F350D927240ED8250001626F0D0E010194
:1013F800D9210001636F8AEC5DF0EBC1D8F1ECC133
:10140800D9F1050ED8900101D837D937E82EFAD787
:10141800000ED8250001D26F020E0101D92100016A
:10142800D36F0F0E0101EB03F3CFDAF1F4CFDBF149
:10143800EC03F350DB27240EDA250001D46F0D0EE0
:101448000101DB210001D56F030ED66FE2EC1AF023
:101458000101DE6FDF6BDE51F3EC58F00101EB4B5D
:10146800EC2B94D79C0502E1070E8C6E020E9C199A
:1014780004E10F01108B070E2D6F839E000E0B6E7B
:10148800C00E45EC59F09CEC5CF0000E0B6EC00EE3
:1014980045EC59F00101A1510CE0A10E0F6E010EAF
:1014A800106EE2EC54F04B0E0F6EFC0E106EE2EC78
:1014B80054F0910E0F6EFF0E106EE2EC54F029D12D
:1014C8008EA889940DEC5DF00B500C1001E1F8D05A
:1014D800EEC1E2F1ED0E0B6E010E0C6E17EC54F03E
:1014E8000101EE6FEDB9EE9F350EEE1907E15E0EC4
:1014F8000001606FFC0E616F8AEC5DF03A0E00012E
:10150800606FFF0E616FEEC162F0636B0101010E47
:10151800EDA9000E0001646F656B8AEC5DF00101B6
:10152800EDA936D0600EEE1933E15F0EE21930E115
:10153800750E0001606FFC0E616FEEC162F0636BA7
:10154800E2C164F0656B010E8EA2000E666F676BD8
:10155800010E8EA4000E686F696B8AEC5DF00101C4
:10156800FF832AEE34F09FC1DFFF2AEE35F09EC1DB
:10157800DFFF8384496A020E486EA4EC37F0839437
:101588000101FF93536A2CEC5DF00101EE6BC1D0B1
:10159800FD514BE0ED51100B0001A96F000EAA6F31
:1015A8000101EE516EEC3CF0A9C0EFF1AAC0F0F1D8
:1015B800080E0101EF19F01101E100F0070E010119
:1015C800EF19F01102E11FEC55F00101EF05F011E0
:1015D80002E159EC4FF0020EEF19F01102E1DBECD9
:1015E80042F0030EEF19F01106E17FEC18F0E4C0A9
:1015F800DCF1E5C0DDF1050E0101EF19F01106E19E
:101608002CEC32F0EDC0DCF1EEC0DDF1090E010189
:10161800EF19F01102E1C5EC5CF00A0E0101EF19B7
:10162800F01177E1EBEC5CF074D0ED51100B0B6E20
:10163800000E0C6EEE517AEC2BF00BC0EFF10CC0E3
:10164800F0F1070E0101EF19F01102E1D0EC55F0AD
:10165800020EEF19F01102E1F0EC57F0EF05F0116E
:1016680002E147EC3BF0030EEF19F01102E1C4EC84
:1016780046F0040EEF19F01102E19AEC5AF0050E4B
:10168800EF19F01102E11FEC3AF0060E0101EF1913
:10169800F01102E15FEC5DF0080EEF19F01102E1C4
:1016A800F3EC2EF0090EEF19F01102E1B6EC3FF061
:1016B8000A0E0101EF19F0112CE18DEC4DF029D043
:1016C800FAEC4BF001019B6F9C5123E0FE519B19F2
:1016D80020E0838E000E0B6EC00E45EC59F09CEC9A
:1016E8005CF0000E0B6EC00E45EC59F0FE0E0F6E4E
:1016F800FE0E106EE2EC54F09BC1FEF14D0E00019F
:10170800606FFC0E616FFEC162F0636B8AEC5DF086
:1017180031D08FB22FD0050E0101DC19DD112AE07E
:10172800CFD68E0E0001606FFE0E616F8FCF62F014
:10173800636B8AEC5DF0290E0101D96F960ED86FA4
:101748007F0EE82EFED7D82FFCD7D92FFAD7040062
:10175800000E0B6EC00E45EC59F09CEC5CF0000ED0
:101768000B6EC00E45EC59F0540E0F6EFF0E106E46
:10177800E2EC54F08FB2D5D7090E0101D96F1E0ED5
:10178800D86FE40EE82EFED7D82FFCD7D92FFAD77A
:1017980000F0839483920001D26BD36B600ED46FF8
:1017A800FC0ED56FD66BF3EC52F0C3D4496E486A81
:1017B80020D3495015E14E5013E0F90E606FFB0E2F
:1017C800616FCECF62F0636BCDCF64F0656B8AEC4E
:1017D8005DF0486A0101896B0A0EBFD083907BD304
:1017E800020E491813E14E5011E0B40E606FFB0E63
:1017F800616FCECF62F0636BCDCF64F0656B8AEC1E
:101808005DF0486A0101896B140EA7D01F0E496468
:101818003ED0300E49603BD04E5039E04950E00F81
:101828004F6E000E606FF90E616FCECF62F0636B82
:10183800CDCF64F0656B4FC066F0676B8AEC5DF0E6
:10184800486A4F50200D0A0EF324D96E020EF42078
:10185800DA6EDE50DE10DE10DE1003E0030E4F6499
:1018680042D0010E4D6E4F50140D130EF324D96E55
:10187800010EF420DA6E4F50140D130EF324E16EAE
:10188800010EF420E26EE7500409DF6E2CD03F0E03
:1018980049642DD0500E49602AD04E5028E04F5050
:1018A800140D000EF324D96E010EF420DA6E49509F
:1018B800C00FDF6E4B0E606FF80E616FCECF62F017
:1018C800636BCDCF64F0656B4F50140D000EF3249D
:1018D800D96E010EF420DA6EDF50666F676B8AEC02
:1018E8005DF0486A4D6A0101886B896B77D7310EC4
:1018F800491807E14E5005E00C0E0101896F1D0ED5
:1019080064D2340E491813E14E5011E0240E606F72
:10191800FC0E616FCECF62F0636BCDCF64F0656B68
:101928008AEC5DF00101886B896B486A57D7350EE0
:10193800491815E14E5013E0120E606FFA0E616FF0
:10194800CECF62F0636BCDCF64F0656B8AEC5DF04F
:10195800486A0D0E0101896FAC0E886F3FD7370EAC
:10196800491807E14E5005E00E0E0101896F750E0A
:101978002CD20D0E491817E14E5015E0486A020E98
:101988000101896FBC0E886F8390C30E0001606FE0
:10199800F90E616FCECF62F0636BCDCF64F0656BEB
:1019A8008AEC5DF098D2100E491807E14E5005E018
:1019B800030E0101896FE90E08D2180E491807E1D4
:1019C8004E5005E0070E0101896F090EFED13B0E4E
:1019D800491807E14E5005E00E0E0101896F7E0E91
:1019E800F4D13E0E491807E14E5005E00F0E0101F3
:1019F800896F3D0EEAD1560E606FF90E616FCECF3A
:101A080062F0636BCDCF64F0656B49C066F0676BBD
:101A18008AEC5DF060D24F50140D010EF324D96E9C
:101A2800010EF420DA6E49C0DFFF030E0101896F51
:101A3800EA0ECBD14F50140D020EF324D96E010ECD
:101A4800F420DA6E49C0DFFF030E0101896FEB0E47
:101A5800BCD14F50140D030EF324D96E010EF4209F
:101A6800DA6E49C0DFFF030E0101896FEC0EADD1BC
:101A78004F50140D040EF324D96E010EF420DA6EC3
:101A880049C0DFFF030E0101896FED0E9ED14F5053
:101A9800140D050EF324D96E010EF420DA6E49C038
:101AA800DFFF030E0101896FEE0E8FD14F50140D29
:101AB800060EF324D96E010EF420DA6E49C0DFFF5A
:101AC8004F50140D060EF324D96E010EF420DA6E71
:101AD800DF50866F86C087F0886B896B8A6B89C0F8
:101AE8008AF088C089F087C088F0876B4F50140D42
:101AF800050EF324D96E010EF420DA6EDF508B6FD9
:101B08008BC08CF08D6B8E6B8F6B8DC08FF08CC003
:101B18008EF08D6B8C6B4F50140D040EF324D96E20
:101B2800010EF420DA6EDF50906F90C091F0926B46
:101B3800936B946B91C094F0936B926B916B4F5035
:101B4800140D030EF324D96E010EF420DA6EDF5063
:101B58009125956F000E9221966F000E9321976F35
:101B6800000E9421986F8C519525996F8D5196216F
:101B78009A6F8E5197219B6F8F5198219C6F875137
:101B880099259D6F88519A219E6F89519B219F6F3E
:101B98008A519C21A06F4F50140D070EF324D96E63
:101BA800010EF420DA6E9DC0DEFF9EC0DEFF9FC0EE
:101BB800DEFFA0C0DEFF690E606FF70E616FCECF4B
:101BC80062F0636BCDCF64F0656B4F50140D070E58
:101BD800F324D96E010EF420DA6EDECF66F0DECF84
:101BE80067F0DECF68F0DECF69F08AEC5DF00101C6
:101BF800886B896B70D14F50140D120EF324D96E77
:101C0800010EF420DA6E49C0DFFF070E0101896F6B
:101C18000A0EDBD04F50140D110EF324D96E010EAD
:101C2800F420DA6E49C0DFFF070E0101896F0B0E41
:101C3800CCD04F50140D100EF324D96E010EF420A1
:101C4800DA6E49C0DFFF070E0101896F0C0EBDD0A7
:101C58004F50140D0F0EF324D96E010EF420DA6ED6
:101C680049C0DFFF0B0E606FF80E616FCECF62F0D8
:101C7800636BCDCF64F0656B4F50140D0F0EF324DA
:101C8800D96E010EF420DA6EDECF66F0DECF67F093
:101C9800DECF68F0DECF69F08AEC5DF0A8D70101ED
:101CA800886B896BEB0E0001606FF70E616FCECF0A
:101CB80062F0636BCDCF64F0656B49C066F0676B0B
:101CC8008AEC5DF04D6A8AD549C06CF10F0E0101AE
:101CD800896F3E0E7AD049C06DF10F0E0101896FF0
:101CE8003F0E73D049C06EF10F0E0101896F400E8F
:101CF8006CD049C06FF10F0E0101896F410E65D09C
:101D080049C070F10F0E0101896F420E5ED049C0C3
:101D180071F10F0E0101896F430E57D049C072F15E
:101D28000F0E0101896F440E50D049C073F1800E27
:101D3800606FF40E616FCECF62F0636BCDCF64F04D
:101D4800656B6CC166F0676B6DC168F0696B6EC1DD
:101D58006AF06B6B6FC16CF06D6B70C16EF06F6B7E
:101D680071C170F0716B72C172F0736B73C174F0F2
:101D7800756B8AEC5DF03BD7240E606FFC0E616FCB
:101D8800CECF62F0636BCDCF64F0656B8AEC5DF00B
:101D98002ED70C0E0101896F1E0E17D06A0E606FC8
:101DA800F80E616FCECF62F0636BCDCF64F0656BD8
:101DB8008AEC5DF00C0E0101896F1C0E886F0A0E0B
:101DC80016D00E0E0101896F760E886F84D0A80E8A
:101DD800606FF90E616FCECF62F0636BCDCF64F0A8
:101DE800656B8AEC5DF00101886B896B090E486EA2
:101DF800F5D488C186F089C187F00001875111E0C8
:101E0800030A13E0040A25E00B0A31E0010A35E071
:101E1800030A39E0010A40E0130A58E03B0A59E096
:101E28005AD0865101E1C5D456D08651E90A01E15C
:101E3800F2D5030A01E1FED5010A01E10AD6070A33
:101E480001E116D6010A01E122D6030A01E12ED6E4
:101E580042D08651090A01E1CED6030A01E1DAD659
:101E6800010A01E1E6D6070A01E1F2D634D086512B
:101E78001D0A8FE0030A92E02ED08651480A01E13C
:101E88007BD7E40A28D08651750A9BE0030A9FE0B5
:101E9800080A01E104D71FD086513D0A01E114D791
:101EA800030A01E118D7010A01E11CD77F0A01E101
:101EB80020D7010A01E124D7030A01E128D7010A42
:101EC80001E12CD7070A01E130D705D086512A0A4B
:101ED80002D086510F0A48501200A8C0BAF0A9C013
:101EE800BBF0AC51D96EDA6ADE6ADD6AA6C00CF0C6
:101EF800A7C00DF0D0EC53F00001B96FB95102E062
:101F0800B951120020EE05F0A651D926A751DA22C0
:101F1800DF5008E020EE05F0A651D926A751DA22B5
:101F2800DF50120020EE04F0A651D926A751DA227C
:101F3800DFA2070C20EE06F0A651D926A751DA2217
:101F480010EE06F0A651E126A751E222E6CFB1F045
:101F5800E6CFB2F0E6CFB3F0E6CFB4F0AA51B125A0
:101F6800B56FAB51B221B66F000EB321B76F000E3B
:101F7800B421B86FDE50B55DDE50B659DE50B759A2
:101F8800DE50B85901E3E1D2AA6BAB6BDED220EE8A
:101F980006F0A651D926A751DA22FF0EDE14AD6F3E
:101FA800010EDE14AE6F000EDE14AF6F000EDE14ED
:101FB800B06FAD51AE11AF11B01101E032D220EEC9
:101FC80006F0A651D926A751DA22DECFADF0DECF32
:101FD800AEF0DECFAFF0DECFB0F00A0E05D0D8906D
:101FE800B033AF33AE33AD33E82EF9D7A6C0D9FF3F
:101FF800A7C0DAFF10EE02F0DE50E126DD50E22243
:10200800E750B16FB105AD15BC6FBC5101E099D077
:1020180020EE06F0A651D926A751DA22DE50DE10AE
:10202800DE10DE1022E120EE0EF0A651D926A751CF
:10203800DA22DECFC3F0DECFC4F0DECFC5F0DECFCC
:10204800C6F0C351C411C511C6112FE1A6C0D9FFEE
:10205800A7C0DAFFDECF8FF0DDCF90F0916B926BE7
:10206800936B946BFBEC34F018D0A6C0D9FFA7C0D3
:10207800DAFFDECF8FF0DDCF90F020EE12F0A65120
:10208800D926A751DA22DECF91F0DECF92F0DECF4B
:1020980093F0DECF94F0FBEC34F08FC0C3F090C027
:1020A800C4F091C0C5F092C0C6F0C351C411C511A7
:1020B800C61101E14ED2C305C411C511C61109E10B
:1020C80020EE05F0A651D926A751DA22020EDF6EBE
:1020D800020CC3290FE1C4290DE1C5290BE1C6296A
:1020E80009E120EE05F0A651D926A751DA22010E02
:1020F800DF6E010C20EE12F0A651D926A751DA2284
:10210800C3C0DEFFC4C0DEFFC5C0DEFFC6C0DEFF41
:1021180020EE0EF0A651D926A751DA22DE50DE10A5
:10212800DE10DE100EE120EE0EF0A651D926A751E2
:10213800DA22C3C0DEFFC4C0DEFFC5C0DEFFC6C0F2
:10214800DEFF20EE16F0A651D926A751DA22A6C046
:10215800E1FFA7C0E2FF00EE2AF0E650E926E550CD
:10216800EA22DE50EE1816E1DE50EE1813E1DE50DA
:10217800EE1810E1DE50EE180DE1A6C0D9FFA7C099
:10218800DAFFDECF24F0DDCF25F003EC49F00009BB
:1021980001E083D1A6C0D9FFA7C0DAFFDECF0BF0DC
:1021A800DDCF0CF0000120EE12F0A651D926A75180
:1021B800DA22DECF0DF0DECF0EF0DECF0FF0DECF6D
:1021C80010F085EC4CF00BC0BFF00CC0C0F00DC097
:1021D800C1F00EC0C2F00001BF51C011C111C2113F
:1021E80001E16ED7BC51BF27000EC023C123C22313
:1021F800AAC0ADF0ABC0AEF0090EAF6FD890AE3349
:10220800AD33AF2FFBD7ADC0BDF0AEC0BEF0BD51F2
:10221800BE1101E1C3D0BC51BD25AD6F000EBE217A
:10222800AE6FA6C0D9FFA7C0DAFF10EE02F0DE50ED
:10223800E126DD50E222E750AF6FB06BAD51AF5DE4
:10224800AE51B05912E2A6C0D9FFA7C0DAFF10EE0E
:1022580002F0DE50E126DD50E222E750AD6FBC51BE
:10226800AD5DBD6FBE6BD8A0BE07BAC01AF0BBC0CB
:102278001BF0BFC01CF0C0C01DF0C1C01EF0C2C022
:102288001FF0BDC020F0BEC021F0A6C0D9FFA7C076
:10229800DAFF10EE01F0DE50E126DD50E222E750D1
:1022A8007BEC4EF0000901E0F8D00001BD51AD6FA4
:1022B800BE51AE6FAF6BB06BA6C0D9FFA7C0DAFF37
:1022C80010EE2AF0DE50E126DD50E222E6CFB1F032
:1022D800E6CFB2F0E6CFB3F0E6CFB4F0BF51B15DD0
:1022E800B56FC051B259B66FC151B359B76FC2512A
:1022F800B459B86FAD51B55DAE51B659AF51B75974
:10230800B051B8593CE2A6C0D9FFA7C0DAFFDECF6A
:10231800ADF0DDCFAEF02E0EAD250B6E000EAE216A
:102328000C6EA6C0D9FFA7C0DAFF10EE2AF0DE5067
:10233800E126DD50E222E6CFAFF0E5CFB0F0BF51A5
:10234800AF5FC051B05B090ED890AF37B037E82EF9
:10235800FBD7AF51BA250D6EB051BB210E6E020EE0
:10236800106E0F6A7BEC5AF0A6C0D9FFA7C0DAFF3F
:1023780010EE04F0DE50E126DD50E222E76ABDC02F
:10238800ADF0BEC0AEF0090ED890AD37AE37E82E2E
:10239800FBD7ADC0C7F0AEC0C8F0BBD020EE0AF086
:1023A800A651D926A751DA2210EE06F0A651E12649
:1023B800A751E222DE50E65CDE50E658DE50E658D1
:1023C800DE50E6581FE3A6C0D9FFA7C0DAFFDECF6C
:1023D80024F0DDCF25F003EC49F0000901E05DD0E1
:1023E800A6C0D9FFA7C0DAFF10EE2AF0DE50E1261A
:1023F800DD50E222BFC0E6FFC0C0E6FFC1C0E6FF75
:10240800C2C0E6FF000120EE16F0A651D926A7515A
:10241800DA22BFC0DEFFC0C0DEFFC1C0DEFFC2C01F
:10242800DEFFAD69010EAE6F20EE06F0A651D9268B
:10243800A751DA22DECFAFF0DDCFB0F0AD51AF1744
:10244800AE51B017AF510008C76FB051D8A0E82AF5
:102458000208C86FC751AA5DC851AB5904E2AAC0A7
:10246800C7F0ABC0C8F0A6C0D9FFA7C0DAFFDECF5F
:1024780039F0DDCF3AF020EE16F0A651D926A75153
:10248800DA22DECF3BF0DECF3CF0DECF3DF0DECF10
:102498003EF0A5EC52F0000902E0000122D600014E
:1024A800AD69010EAE6F20EE06F0A651D926A751F0
:1024B800DA22DECFAFF0DDCFB0F0AD51AF17AE51BD
:1024C800B017A6C0D9FFA7C0DAFFDECFB1F0DDCFC5
:1024D800B2F0AF51B127B051B2232E0EB1250B6E19
:1024E800000EB2210C6EBAC00DF0BBC00EF0C7C012
:1024F8000FF0C8C010F07BEC5AF0A6C0D9FFA7C0F7
:10250800DAFF10EE04F0DE50E126DD50E222010E83
:10251800E76EC751BA27C851BB2320EE06F0A65173
:10252800D926A751DA22C751DE26C851DE22000E6D
:10253800DE22DE22AC51D96EDA6AC751DE26C851D6
:10254800DD22C751AA5FC851AB5BAA51AB1101E0AC
:102558001ED520EE06F0A651D926A751DA2210EE94
:102568000AF0A651E126A751E222DE50E65CDE50D1
:10257800E658DE50E658DE50E65814E220EE06F043
:10258800A651D926A751DA2210EE0AF0A651E12663
:10259800A751E222DECFE6FFDECFE6FFDECFE6FF81
:1025A800DECFE6FF20EE04F0A651D926A751DA22A5
:1025B800000EDB8A000CA6C00CF0A7C00DF0D0EC12
:1025C80053F00001C06FC05102E0C051120020EE6C
:1025D80005F0A651D926A751DA22DF5008E020EEEF
:1025E80005F0A651D926A751DA22DF50120020EEB5
:1025F8000AF0A651D926A751DA22A851DE5CA951C2
:10260800DE58AA51DE58AB51DE5816E220EE04F02F
:10261800A651D926A751DA22DFB20ED020EE0AF051
:10262800A651D926A751DA22DECFA8F0DECFA9F02D
:10263800DECFAAF0DECFABF020EE06F0A651D92609
:10264800A751DA22DECFBCF0DECFBDF0DECFBEF080
:10265800DECFBFF0C16BC26BC36BC46B20EE06F05C
:10266800A651D926A751DA22C1C0DEFFC2C0DEFFBB
:10267800C3C0DEFFC4C0DEFFA851A911AA11AB1167
:1026880001E119D2A6C0D9FFA7C0DAFF10EE02F007
:10269800DE50E126DD50E222E750AC6FACC0ADF071
:1026A800AE6BAF6BB06B090ED890AD37AE37AF37A6
:1026B800B037E82EF9D7ADC0C5F0AEC0C6F0AFC090
:1026C800C7F0B0C0C8F0BC51BD11BE11BF1101E1C7
:1026D80096D0FF0EA8250B6EFF0EA9210C6EFF0EDB
:1026E800AA210D6EFF0EAB210E6EC5C00FF0C6C03D
:1026F80010F0C7C011F0C8C012F05BEC55F00BC069
:10270800ACF00CC0ADF00DC0AEF00EC0AFF0FF0ED7
:102718000001BC250B6EFF0EBD210C6EFF0EBE2105
:102728000D6EFF0EBF210E6EC5C00FF0C6C010F0B3
:10273800C7C011F0C8C012F05BEC55F00B50000197
:10274800AC5D0C50AD590D50AE590E50AF5957E312
:10275800FF0EC525AC6FFF0EC621AD6FFF0EC7215A
:10276800AE6FFF0EC821AF6FAC1DB06FAD1DB16F5E
:10277800AE1DB26FAF1DB36FFF0EBC25B46FFF0E59
:10278800BD21B56FFF0EBE21B66FFF0EBF21B76F1B
:10279800B051B415B86FB151B515B96FB251B6157E
:1027A800BA6FB351B715BB6F20EE06F0A651D92604
:1027B800A751DA22B8C0DEFFB9C0DEFFBAC0DEFF1B
:1027C800BBC0DEFF20EE06F0A651D926A751DA22BB
:1027D800DE50A85FDE50A95BDE50AA5BDD50AB5B24
:1027E80020EE12F0A651D926A751DA22DECFC9F081
:1027F800DECFCAF0DECFCBF0DECFCCF064D020EE57
:102808000EF0A651D926A751DA22DECFC9F0DECFC5
:10281800CAF0DECFCBF0DECFCCF0C951CA11CB1154
:10282800CC1143E1A6C0D9FFA7C0DAFFDECF8FF0F5
:10283800DDCF90F0916B926B936B946BFBEC34F063
:102848008FC0C9F090C0CAF091C0CBF092C0CCF054
:10285800C905CA11CB11CC1109E120EE05F0A6512A
:10286800D926A751DA22020EDF6E020CC9290FE120
:10287800CA290DE1CB290BE1CC2909E120EE05F0AD
:10288800A651D926A751DA22010EDF6E010C20EEDF
:102898000EF0A651D926A751DA22C9C0DEFFCAC058
:1028A800DEFFCBC0DEFFCCC0DEFF20EE12F0A6516B
:1028B800D926A751DA22C9C0DEFFCAC0DEFFCBC0C5
:1028C800DEFFCCC0DEFFC951CA11CB11CC1101E02B
:1028D80095D0F1D020EE04F0A651D926A751DA22DE
:1028E800DFA228D0A6C0D9FFA7C0DAFFDECF8FF0BD
:1028F800DDCF90F0C9C091F0CAC092F0CBC093F080
:10290800CCC094F0FBEC34F08FC0C9F090C0CAF092
:1029180091C0CBF092C0CCF0C951CA11CB11CC11E7
:1029280023E1C5C0A8F0C6C0A9F0C7C0AAF0C8C0B6
:10293800ABF06ED0A6C0D9FFA7C0DAFFDECF44F057
:10294800DDCF45F0C9C046F0CAC047F0CBC048F05B
:10295800CCC049F0A2EC1FF044C0C9F045C0CAF091
:1029680046C0CBF047C0CCF00001C92907E1CA290D
:1029780005E1CB2903E1CC2901E180D7CC51CB116A
:10298800CA1104E1020EC95D01E267D7A6C0D9FFEA
:10299800A7C0DAFF10EE12F0DE50E126DD50E22289
:1029A800E650C95DE650CA59E650CB59E650CC59B5
:1029B80001E353D720EE12F0A651D926A751DA2207
:1029C800C9C0DEFFCAC0DEFFCBC0DEFFCCC0DEFF61
:1029D80020EE06F0A651D926A751DA22C551DE26E7
:1029E800C651DE22C751DE22C851DE22C551A85F7A
:1029F800C651A95BC751AA5BC851AB5BA851C55D5D
:102A0800A951C659AA51C759AB51C85901E262D751
:102A180020EE06F0A651D926A751DA22A851DE26C3
:102A2800A951DE22AA51DE22AB51DE22A851AC6F99
:102A3800010EA915AD6FAE6BAF6BAC11AE11AF1136
:102A48003AE0A6C0D9FFA7C0DAFFDECF0BF0DDCF92
:102A58000CF0C9C00DF0CAC00EF0CBC00FF0CCC04E
:102A680010F085EC4CF00BC0C1F00CC0C2F00DC0EA
:102A7800C3F00EC0C4F00001C151C211C311C4118A
:102A880001E1EBD6A8C0ACF0A9C0ADF0AAC0AEF089
:102A9800ABC0AFF00A0E05D0D890AF33AE33AD332C
:102AA800AC33E82EF9D7AC51C127AD51C223AE5192
:102AB800C323AF51C42320EE06F0A651D926A7514F
:102AC800DA22FF0EDE14AC6F010EDE14AD6F000EBD
:102AD800DE14AE6F000EDE14AF6FAC51AD11AE1147
:102AE800AF1120E020EE16F0A651D926A751DA2220
:102AF800C151DE1809E1C251DE1806E1C351DE18E2
:102B080003E1C451DE180EE020EE16F0A651D926D6
:102B1800A751DA22C1C0DEFFC2C0DEFFC3C0DEFF9C
:102B2800C4C0DEFF20EE06F0A651D926A751DA224E
:102B380010EE0AF0A651E126A751E222DE50E65C2B
:102B4800DE50E658DE50E658DE50E65801E33DD543
:102B580020EE06F0A651D926A751DA2210EE0AF087
:102B6800A651E126A751E222DECFE6FFDECFE6FF3F
:102B7800DECFE6FFDECFE6FF20EE04F0A651D92631
:102B8800A751DA22000EDB8A20D586C0A1F087C0C3
:102B9800A2F08AC0D9FF8BC0DAFFDE6ADD6A84C082
:102BA8000CF085C00DF0D0EC53F000019C6F9C51E7
:102BB80002E09C51120020EE05F08451D92685517F
:102BC800DA22DF5008E020EE05F08451D92685513D
:102BD800DA22DF50120020EE04F08451D926855104
:102BE800DA22DFA0070C20EE06F08451D9268551A1
:102BF800DA22DECF8CF0DECF8DF0DECF8EF0DECFA6
:102C08008FF020EE0AF08451D9268551DA22DECFE2
:102C180090F0DECF91F0DECF92F0DECF93F08C51C2
:102C2800905D986F8D519159996F8E5192599A6F05
:102C38008F5193599B6F88518C6F89518D6F8E6B13
:102C48008F6B8C51985D8D5199598E519A598F512E
:102C58009B5901E34BD298C088F099C089F046D2BD
:102C680020EE06F08451D9268551DA22FF0EDE14B3
:102C78008C6F010EDE148D6F000EDE148E6F000E49
:102C8800DE148F6F8C518D118E118F1101E0A5D13B
:102C980020EE06F08451D9268551DA22DECF8CF059
:102CA800DECF8DF0DECF8EF0DECF8FF00A0E05D0AE
:102CB800D8908F338E338D338C33E82EF9D784C078
:102CC800D9FF85C0DAFF10EE02F0DE50E126DD50B4
:102CD800E222E750906F90058C15A36FA3516AE12B
:102CE80020EE06F08451D9268551DA22DE50DE1016
:102CF800DE10DE100FE120EE0EF08451D92685514A
:102D0800DA22DECF9DF0DECF9EF0DECF9FF0DECF61
:102D1800A0F020D084C0D9FF85C0DAFFDECF44F010
:102D2800DDCF45F020EE12F08451D9268551DA2204
:102D3800DECF46F0DECF47F0DECF48F0DECF49F0F9
:102D4800A2EC1FF044C09DF045C09EF046C09FF025
:102D580047C0A0F00001A0519F119E110CE1020E86
:102D68009D5D09E220EE05F08451D9268551DA22CD
:102D7800020EDF6E020C9D290FE19E290DE19F29AD
:102D88000BE1A02909E120EE05F08451D9268551EF
:102D9800DA22010EDF6E010C20EE12F08451D926E2
:102DA8008551DA229DC0DEFF9EC0DEFF9FC0DEFF98
:102DB800A0C0DEFF84C0D9FF85C0DAFFDECF0BF0EC
:102DC800DDCF0CF020EE12F08451D9268551DA229D
:102DD800DECF0DF0DECF0EF0DECF0FF0DECF10F03D
:102DE80085EC4CF00BC0A4F00CC0A5F00DC0A6F00B
:102DF8000EC0A7F00001A451A511A611A71101E169
:102E0800B1D7A351A427000EA523A623A72388C0C2
:102E18008CF089C08DF0090E8E6FD8908D338C336D
:102E28008E2FFBD78CC0A8F08DC0A9F0A851A9118E
:102E380001E1C5D0A351A8258C6F000EA9218D6F83
:102E480084C0D9FF85C0DAFF10EE02F0DE50E1261B
:102E5800DD50E222E7508E6F8F6B8C518E5D8D5165
:102E68008F5912E284C0D9FF85C0DAFF10EE02F054
:102E7800DE50E126DD50E222E7508C6FA3518C5DD5
:102E8800A86FA96BD8A0A907A1C01AF0A2C01BF00F
:102E9800A4C01CF0A5C01DF0A6C01EF0A7C01FF05E
:102EA800A8C020F0A9C021F084C0D9FF85C0DAFFEE
:102EB80010EE01F0DE50E126DD50E222E750B7ECDB
:102EC80051F0000901E0C5D084C0D9FF85C0DAFF00
:102ED80010EE04F0DE50E126DD50E222E7505FE01C
:102EE8000001A8518C6FA9518D6F8E6B8F6B84C0B8
:102EF800D9FF85C0DAFF10EE2AF0DE50E126DD505A
:102F0800E222E6CF90F0E6CF91F0E6CF92F0E6CF5E
:102F180093F0A451905D946FA5519159956FA65166
:102F28009259966FA7519359976F8C51945D8D5113
:102F380095598E5196598F51975931E284C0D9FFCE
:102F480085C0DAFF10EE2AF0DE50E126DD50E222DD
:102F5800E6CF8CF0E5CF8DF0A4518C5FA5518D5B49
:102F6800090ED8908C378D37E82EFBD78C51A125C8
:102F78000B6E8D51A2210C6E84C0D9FF85C0DAFF7B
:102F8800DECF8EF0DDCF8FF02E0E8E250D6E000E6B
:102F98008F210E6E020E106E0F6A7BEC5AF0A8C0DD
:102FA8008CF0A9C08DF0090ED89000018C378D37B0
:102FB800E82EFAD78CC0AAF08DC0ABF07AD020EEFC
:102FC80016F08451D9268551DA22A4C0DEFFA5C0A7
:102FD800DEFFA6C0DEFFA7C0DEFF8C69010E8D6F85
:102FE80020EE06F08451D9268551DA22DECF8EF004
:102FF800DDCF8FF08C518E178D518F178E510008B1
:10300800AA6F8F51D8A0E82A0208AB6FAA51885D31
:10301800AB51895904E288C0AAF089C0ABF084C0DA
:10302800D9FF85C0DAFFDECF39F0DDCF3AF020EEE8
:1030380016F08451D9268551DA22DECF3BF0DECF57
:103048003CF0DECF3DF0DECF3EF0A5EC52F00009BB
:1030580002E0000198D6A1C00BF0A2C00CF000015C
:103068008C69010E8D6F20EE06F08451D9268551AA
:10307800DA22DECF8EF0DDCF8FF08C518E178D5196
:103088008F1784C0D9FF85C0DAFFDECF90F0DDCF7F
:1030980091F08E5190278F5191232E0E90250D6E11
:1030A800000E91210E6EAAC00FF0ABC010F07BECA1
:1030B8005AF0AA51A127AB51A22320EE06F0845161
:1030C800D9268551DA22AA51DE26AB51DE22000E1E
:1030D800DE22DE228AC0D9FF8BC0DAFFAA51DE26A3
:1030E800AB51DD22AA51885FAB51895B88518911A8
:1030F80001E0B6D5000C838E8380480E0001606F16
:10310800F70E616FCECF62F0636BCDCF64F0656B65
:103118004F50140D070EF324D96E010EF420DA6E09
:10312800DECF66F0DECF67F0DECF68F0DECF69F085
:103138004F50140D070EF324D96E010EF420DA6EE9
:10314800DECF6AF0DECF6BF0DECF6CF0DECF6DF055
:103158008AEC5DF0E0EC43F0CDC0B3F1CEC0B4F141
:103168000101B351B4111AE04F50140D130EF3249A
:10317800D96E010EF420DA6E4F50140D130EF3249D
:10318800E16E010EF420E26EE7500409DF6E17ECE1
:103198005CF0B3C1E4F0B4C1E5F012004F50140D77
:1031A800070EF324D96E010EF420DA6E74C1EBF029
:1031B80075C1ECF076C1EDF00001EA6B000EEA256E
:1031C800EE6F010EEB21EF6F000EEC21F06F000E99
:1031D800ED21F16FDE50EE195EE1DE50EF195BE193
:1031E800DE50F01958E1DE50F11955E15CEC57F06A
:1031F8000FC0B8F110C0B9F111C0BAF112C0BBF1DB
:10320800000EE8CF34FA2AEE35F0BBC1DFFFE8CF75
:1032180036FA2AEE37F0BAC1DFFFE8CF38FA2AEEDD
:1032280039F0B9C1DFFFE8CF3AFA2AEE3BF0B8C16E
:10323800DFFF0101FF93010E496E000E486AA4ECFE
:1032480037F00101FF937A0E0001606FF50E616F90
:10325800CECF62F0636BCDCF64F0656B2AEE35F0AC
:10326800DF50666F676B2AEE37F0DF50686F696B67
:103278002AEE39F0DF506A6F6B6B2AEE3BF0DF50B5
:103288006C6F6D6B8AEC5DF04D6A83904DC0E4F015
:103298000001E56B12004F50140D0F0EF324D96E88
:1032A800010EF420DA6EDECFE6F0DECFE7F0DECFF7
:1032B800E8F0DECFE9F0E7C0E6F0E8C0E7F0E9C003
:1032C800E8F0E96BE6C0AFF1E7C0B0F14F50140D7C
:1032D8000F0EF324D96E010EF420DA6EDECFE6F07D
:1032E800DDCFE7F0E6510101B56FB66BFF93AB6B2D
:1032F800AC6BAD6BAE6BB16BB26BABD0E669E7692B
:10330800AFC1E8F0B0C1E9F0E651E827E751E92399
:103318000101B1510001E8190AE10101B2510001AE
:10332800E91905E10101B551B61101E1FF834F50DB
:10333800200D000EF3240001846F020EF420856F27
:10334800340E866F0A0E876F010E896F886BBC0E6C
:103358008A6F010E8B6FC9EC15F00101B76FE10E92
:103368000001606FF60E616FCECF62F0636BCDCF58
:1033780064F0656BB7C166F0676BBCC168F0BDC12E
:1033880069F08AEC5DF00101B75101E0EDD6BCC1EE
:1033980048F0BDC149F0A4EC37F00101BC51AB279E
:1033A800BD51AC23000EAD23AE234F50140D070EB4
:1033B800F324D96E010EF420DA6E000EDE2400012B
:1033C800E66F010EDE20E76F000EDE20E86F000ECC
:1033D800DE20E96F4F50140D070EF324D96E010E4D
:1033E800F420DA6EE6C0DEFFE7C0DEFFE8C0DEFFED
:1033F800E9C0DEFF3A0E606FF90E616FCECF62F062
:10340800636BCDCF64F0656B4F50140D070EF3243A
:10341800D96E010EF420DA6EDECF66F0DECF67F0EB
:10342800DECF68F0DECF69F04F50140D070EF3249D
:10343800D96E010EF420DA6EDECF6AF0DECF6BF0C3
:10344800DECF6CF0DECF6DF08AEC5DF00101B14BA0
:10345800B22BAF51B15DB251800A0001E66F010194
:10346800B051800A0001E65901E248D70101B6BF10
:103478008AD0B65103E1B50501E285D04F50200D41
:10348800000EF3240001846F020EF420856F340EC1
:10349800866F0A0E876FB5C188F0B6C189F0BC0E79
:1034A8008A6F010E8B6FC9EC15F00101B76FEE0E34
:1034B8000001606FF60E616FB7C162F0636BBCC14B
:1034C80064F0BDC165F08AEC5DF00101B75101E01F
:1034D8004BD6FF83B5C148F0B6C149F0A4EC37F02C
:1034E8000101BC51AB27BD51AC23000EAD23AE2367
:1034F8004F50140D070EF324D96E010EF420DA6E26
:10350800000EDE240001E66F010EDE20E76F000EDC
:10351800DE20E86F000EDE20E96F4F50140D070E15
:10352800F324D96E010EF420DA6EE6C0DEFFE7C0A0
:10353800DEFFE8C0DEFFE9C0DEFF890E606FFC0E2B
:10354800616F4F50140D070EF324D96E010EF4204D
:10355800DA6EDECF62F0DECF63F0DECF64F0DECF6E
:1035680065F04F50140D070EF324D96E010EF420A8
:10357800DA6EDECF66F0DECF67F0DECF68F0DECF42
:1035880069F08AEC5DF00101FF93C60E0001606FDF
:10359800FA0E616FCECF62F0636BCDCF64F0656BCE
:1035A800ABC166F0ACC167F0ADC168F0AEC169F0FF
:1035B8008AEC5DF04D6A8390839E68D6D251D31110
:1035C80001E1090CD2C0D9FFD3C0DAFFDE6ADD6A97
:1035D8008CC1C2F18DC1C3F11F0ED617C20E7C6F0C
:1035E800010E7D6FD40E7E6FD651FE0B7F6FAEEC51
:1035F80000F00101BF6FBF5101E040D2AB0ED66FA2
:10360800010ED76FC20E0001BF6F010EC06FD4C08C
:10361800C1F0D5C0C2F048EC48F00101BF6FD4C179
:10362800C0F1D5C1C1F1BF5105E1C051C11102E1DD
:10363800060EBF6FD6C0D7F01C0E0001D71701E1E8
:1036480014D10101BF5113E0040EBF1909E1C20EE4
:103658000001C36F010EC46F01EC51F00101BF6F8F
:103668000001D687D4C1C0F1D5C1C1F113D020EE75
:103678000BF0C051D926C151DA22DF500001D76FB3
:10368800110ED71702E0070E03D0D6A503D0080EF7
:103698000101BF6F0101BF5101E002D10001D6A7AE
:1036A800FFD00101BB6BBC6B210EBD6F460EBE6F18
:1036B80020EE0EF0C051D926C151DA22DF6A20EE81
:1036C8000FF0C051D926C151DA22BCC1DFFF20EE6C
:1036D80010F0C051D926C151DA22BDC1DFFF20EE5A
:1036E80011F0C051D926C151DA22BEC1DFFF20EE48
:1036F80016F0C051D926C151DA22DF6A20EE17F040
:10370800C051D926C151DA22BCC1DFFF20EE18F022
:10371800C051D926C151DA22BDC1DFFF20EE19F010
:10372800C051D926C151DA22BEC1DFFF20EE0BF00D
:10373800C051D926C151DA22DF6A20EE1CF0C051EF
:10374800D926C151DA22DF6A20EE1DF0C051D926F0
:10375800C151DA22DF6A20EE1EF0C051D926C151CC
:10376800DA22DF6A20EE1FF0C051D926C151DA22D1
:10377800DF6AC2C10BF0C3C10CF0C0C10DF0C1C1FA
:103788000EF062EC51F00BC0B7F10CC0B8F10DC0EF
:10379800B9F10EC0BAF1C0C10BF0C1C10CF00D6A8D
:1037A8000E6A0F6A106A19EC5AF0010120EE04F053
:1037B800C251D926C351DA22010EDF6EB751B811B2
:1037C800B911BA116DE020EE2AF0C251D926C351C1
:1037D800DA22DECFBBF1DECFBCF1DECFBDF1DECF2A
:1037E800BEF1C2C18FF0C3C190F0B7C191F0B8C1AA
:1037F80092F0B9C193F0BAC194F0D2EC4AF0010149
:10380800BF6FBF514DE1FF0EB7250001D76FFF0E07
:103818000101B8210001D86FFF0E0101B921000193
:10382800D96FFF0E0101BA210001DA6F010120EE04
:103838000AF0C251D926C351DA22D7C0DEFFD8C058
:10384800DEFFD9C0DEFFDAC0DEFFC2C139F0C3C176
:103858003AF0BBC13BF0BCC13CF0BDC13DF0BEC1BC
:103868003EF0A5EC52F001011AD00101BF5118E158
:1038780020EE0BF0C051D926C151DA22DFA802D0C0
:10388800040E0DD00001D6A30BD0010120EE0BF0E1
:10389800C051D926C151DA22DFA002D0070EBF6F6E
:1038A8000101BF5123E10001D6B7D68B010120EEFB
:1038B8002AF0C251D926C351DA22000110EE1AF0BB
:1038C800D251E126D351E222DECFE6FFDECFE6FF7A
:1038D800DECFE6FFDECFE6FF20EE1EF0D251D9267E
:1038E800D351DA22C0C1DEFFC1C1DDFF0101BF51E2
:1038F80001E0C4D0000120EE04F0D251D926D35102
:10390800DA22D6C0DFFF20EE05F0D251D926D351F6
:10391800DA22DF6AC2C10BF0C3C10CF0C0C10DF0DE
:10392800C1C10EF062EC51F0000120EE0EF0D25150
:10393800D926D351DA220BC0DEFF0CC0DEFF0DC042
:10394800DEFF0EC0DEFF010120EE1DF0C051D926BA
:10395800C151DA22DF500001D86FD76B010120EE88
:103968001EF0C051D926C151DA22DF500001D96FAB
:10397800D9C0DAF0DB6BDC6BDD6BDBC0DDF0DAC005
:10398800DCF0DB6BDA6B010120EE1FF0C051D926A9
:10399800C151DA22DF500001DE6FDEC0DFF0E06BDC
:1039A800E16BE26BDFC0E2F0E16BE06BDF6BDA51F9
:1039B800DF11E36FDB51E011E46FDC51E111E56FDA
:1039C800DD51E211E66FD751E311E76FD851E411E9
:1039D800E86F000EE511E96F000EE611EA6F0101CC
:1039E80020EE1CF0C051D926C151DA22DF50000167
:1039F800E711EB6FE851EC6FE951ED6FEA51EE6FAB
:103A080020EE0AF0D251D926D351DA22EBC0DEFFDC
:103A1800ECC0DEFFEDC0DEFFEEC0DEFF20EE06F0FC
:103A2800D251D926D351DA22DE6ADE6ADE6ADD6A2D
:103A380020EE16F0D251D926D351DA22DE6ADE6A98
:103A4800DE6ADD6AD2C0D9FFD3C0DAFFC2C1DEFFA9
:103A5800C3C1DDFFD2C0D9FFD3C0DAFF10EE06F034
:103A6800DE50E126DD50E22220EE02F0D251D926C6
:103A7800D351DA22E6CFDEFFE5CFDDFF0101BF51EA
:103A8800120065516411631103E1020E625D10E3D7
:103A980020EE12F06051D9266151DA22DE50625DC3
:103AA800DE506359DE506459DE50655901E22FD269
:103AB800020E8C6F41D262C08AF063C08BF0D8903E
:103AC8008B316B6F8A316A6F6A518A276B518B23EE
:103AD80060C039F061C03AF020EE1EF06051D9267E
:103AE8006151DA22DECF6AF0DECF6BF0DECF6CF008
:103AF800DECF6DF08AC06EF08BC06FF0090E706F6C
:103B0800D8906F336E33702FFBD76E516A253B6E9A
:103B18006F516B213C6E000E6C213D6E000E6D21C5
:103B28003E6EA5EC52F000018C6F8C5101E004D27E
:103B38006A69010E6B6F8AC06CF08BC06DF06A51B8
:103B48006C176B516D1760C06EF061C06FF06C51EF
:103B58006E276D516F232E0E6E258D6F000E6F210F
:103B68008E6F8A4B8B2B62B104D066C086F0876B50
:103B78001AD066516A6F6B6B6A3B6B3BF00E6B1722
:103B88006A510F0B6B13F00E6A178DC0D9FF8EC0E8
:103B9800DAFFDF500F0B6C6F6D6B6A516C11866F1B
:103BA8006B516D11876F8DC0D9FF8EC0DAFF86C04B
:103BB800DFFF20EE04F06051D9266151DA22010EB0
:103BC800DF6E60C039F061C03AF020EE1EF060513F
:103BD800D9266151DA22DECF6AF0DECF6BF0DECF74
:103BE8006CF0DECF6DF08AC06EF08BC06FF0090EFE
:103BF800706FD8906F336E33702FFBD76E516A2574
:103C08003B6E6F516B213C6E000E6C213D6E000EB9
:103C18006D213E6EA5EC52F000018C6F8C5101E0D5
:103C28008BD16A69010E6B6F8AC06CF08BC06DF026
:103C38006A516C176B516D1760C06EF061C06FF000
:103C48006C516E276D516F232E0E6E258D6F000EF1
:103C58006F218E6F62B10CD067C06AF00F0E6A17C1
:103C68008DC0D9FF8EC0DAFFDF50F00B6A1112D079
:103C780066C06AF067C06BF068C06CF069C06DF030
:103C8800050E05D0D8906D336C336B336A33E82E4C
:103C9800F9D76A51886F896B8DC0D9FF8EC0DAFF5A
:103CA80088C0DFFF2BD160C039F061C03AF020EE48
:103CB8001EF06051D9266151DA22DECF6AF0DECFDC
:103CC8006BF0DECF6CF0DECF6DF063516E6F645138
:103CD8006F6F6551706F716B6A516E253B6E6B51DA
:103CE8006F213C6E6C5170213D6E6D5171213E6E9D
:103CF800A5EC52F000018C6F8C5101E01DD16A696E
:103D0800010E6B6F62C06CF063C06DF0D8906C37B9
:103D18006D376A516C176B516D1760C06EF061C0DA
:103D28006FF06C516E276D516F232E0E6E258D6FBF
:103D3800000E6F218E6F8DC0D9FF8EC0DAFF66C06E
:103D4800DFFF20EE01F08D51D9268E51DA2267C0AF
:103D5800DFFFD4D060C039F061C03AF020EE1EF029
:103D68006051D9266151DA22DECF6AF0DECF6BF0DE
:103D7800DECF6CF0DECF6DF062C06EF063C06FF026
:103D880064C070F065C071F0080E05D0D89071332A
:103D980070336F336E33E82EF9D76A516E253B6E58
:103DA8006B516F213C6E6C5170213D6E6D517121CC
:103DB8003E6EA5EC52F000018C6F8C5101E0BCD036
:103DC8006A69010E6B6F62C06CF063C06DF0D890C9
:103DD8006C376D37D8906C376D376A516C176B51EB
:103DE8006D1760C06EF061C06FF06C516E276D5139
:103DF8006F232E0E6E258D6F000E6F218E6F20EEB5
:103E080001F08D51D9268E51DA22DF506B6F6A6B23
:103E180020EE02F08D51D9268E51DA22DF506C6FD8
:103E28006CC06DF06E6B6F6B706B6EC070F06DC0B8
:103E38006FF06E6B6D6B20EE03F08D51D9268E51AD
:103E4800DA22DF50716F71C072F0736B746B756B2F
:103E580072C075F0746B736B726B6D517211766F03
:103E68006E517311776F6F517411786F70517511AE
:103E7800796F6A5176117A6F6B5177117B6F000EEB
:103E880078117C6F000E79117D6F8DC0D9FF8EC0BF
:103E9800DAFFDF507A117E6F7B517F6F7C51806F24
:103EA8007D51816F826B836B846BF00E8115856FFA
:103EB80082516613835167138451681385516913BE
:103EC8008DC0D9FF8EC0DAFF66C0DFFF20EE01F09B
:103ED8008D51D9268E51DA2267C0DFFF20EE02F01D
:103EE8008D51D9268E51DA2268C0DFFF20EE03F00B
:103EF8008D51D9268E51DA2269C0DFFF20EE04F0F9
:103F08006051D9266151DA22010EDF6E15D060C0EA
:103F1800D9FF61C0DAFFDF506A6F6B6B6B5101E04C
:103F2800C7D56A51010A01E1C6D5030A01E1BBD62A
:103F3800010A01E10FD7BCD58C5112004950481035
:103F4800471003E1020E465C0FE320EE12F04450E6
:103F5800D9264550DA22DE50465CDE504758DE50FE
:103F68004858DE50495808E3010E00017C6F000EE6
:103F78007D6B7E6B7F6BEFD100017C697D697E690B
:103F88007F69D4D146C080F047C081F0D890813194
:103F9800616F8031606F605180276151812344C017
:103FA80039F045C03AF020EE1EF04450D92645506D
:103FB800DA22DECF60F0DECF61F0DECF62F0DECF56
:103FC80063F080C064F081C065F0090E666FD89018
:103FD80065336433662FFBD7645160253B6E6551AA
:103FE80061213C6E000E62213D6E000E63213E6E23
:103FF800A5EC52F0000901E0AED100016069010EA4
:10400800616F80C062F081C063F0605162176151D6
:10401800631744C064F045C065F06251642763517A
:1040280065232E0E6425D96E000E6521DA6EDF50E9
:104038007A6F7B6B804B812B44C039F045C03AF0D6
:1040480020EE1EF04450D9264550DA22DECF60F02B
:10405800DECF61F0DECF62F0DECF63F080C064F0C7
:1040680081C065F0090E666FD89065336433662F9A
:10407800FBD7645160253B6E655161213C6E000E93
:1040880062213D6E000E63213E6EA5EC52F00009E0
:1040980001E061D100016069010E616F80C062F0CA
:1040A80081C063F0605162176151631744C064F0C6
:1040B80045C065F062516427635165232E0E64255F
:1040C800D96E000E6521DA6EDF50676F666B665138
:1040D8007A1367517B1346B006D07A51786F0F0E6A
:1040E8007B15796F0FD07AC060F07BC061F0040E49
:1040F800626FD89061336033622FFBD760C078F06D
:1041080061C079F078C07CF079C07DF05BD044C0A4
:1041180039F045C03AF020EE1EF04450D9264550FB
:10412800DA22DECF60F0DECF61F0DECF62F0DECFE4
:1041380063F04750646F4850656F4950666F676B0E
:10414800605164253B6E615165213C6E6251662168
:104158003D6E635167213E6EA5EC52F0000901E007
:10416800FAD000016069010E616F46C062F047C075
:1041780063F0D890623763376051621761516317F3
:1041880044C064F045C065F06251642763516523FB
:104198002E0E6425826F000E6521836F20EE01F0DC
:1041A8008251D9268351DA22DF50616F606B82C059
:1041B800D9FF83C0DAFFDF506013000E60C07CF0C7
:1041C80061C07DF07E6B7F6BC6D044C039F045C0BE
:1041D8003AF020EE1EF04450D9264550DA22DECFC0
:1041E80060F0DECF61F0DECF62F0DECF63F046C074
:1041F80064F047C065F048C066F049C067F0080E33
:1042080005D0D8906733663365336433E82EF9D721
:10421800605164253B6E615165213C6E6251662197
:104228003D6E635167213E6EA5EC52F0000901E036
:1042380092D000016069010E616F46C062F047C00C
:1042480063F0D89062376337D8906237633760512C
:1042580062176151631744C064F045C065F062514C
:104268006427635165232E0E6425826F000E652135
:10427800836F20EE01F08251D9268351DA22DF5074
:10428800616F606B20EE02F08251D9268351DA22E9
:10429800DF50626F62C063F0646B656B666B64C00D
:1042A80066F063C065F0646B636B20EE03F08251C7
:1042B800D9268351DA22DF50676F67C068F0696BCF
:1042C8006A6B6B6B68C06BF06A6B696B686B635188
:1042D80068116C6F645169116D6F65516A116E6F69
:1042E80066516B116F6F60516C11706F61516D1178
:1042F800716F000E6E11726F000E6F11736F82C0B6
:10430800D9FF83C0DAFFDF507011746F7151756F78
:104318007251766F7351776F74517C6F75517D6FE1
:1043280076517E6F0F0E77157F6F15D044C0D9FF79
:1043380045C0DAFFDF50606F616B615101E014D650
:104348006051010A01E11ED6030A01E1E0D6010A23
:1043580001E13BD709D67CC044F07DC045F07EC062
:1043680046F07FC047F012002A6E1BC041F01CC007
:1043780042F02A5001E0040C010E3F6E54B0030CC9
:10438800E9D147EC5DF0000901E1FDD13F6AFBD1BD
:10439800146A156A166A176A090E4AEC5BF0000976
:1043A80001E0F1D12B0E0B6E0C6A0E6A100E0D6E29
:1043B800C1EC57F0000901E1E6D12B44E846030BB4
:1043C800E8064DE132C01DF03F0E1D161DC01EF05F
:1043D8001F6A206A216A1FC021F01EC020F01F6AD0
:1043E8001E6A3350236E226A3450246E256A225086
:1043F80024262350252224501E24266E25501F20B3
:10440800276E000E2020286E000E2120296E2628F7
:104418003B6E000E27203C6E000E28203D6E000EDD
:1044280029203E6E3BC01DF03CC01EF03DC01FF071
:104438003EC020F00A0ED8901D361E361F36203694
:10444800E82EF9D71BC0D9FF1CC0DAFF1DC0DEFF5C
:104458001EC0DEFF1FC0DEFF20C0DEFF97D71D6A2B
:1044680035AE01D01D2A010E1D1630C01EF00F0EEC
:104478001E163450030B020DF3501E241D24020F88
:10448800406E3150030B1D6E1E6A0A0ED8901D3601
:104498001E36E82EFBD732501F6E206AD8901F3682
:1044A8002036D8901F3620363344E846030B216E59
:1044B800226A1F502126205022221D5021261E50DC
:1044C8002222212A000E222221C03BF022C03CF0E9
:1044D8003D6A3E6A40C01DF0F70E1D263BC01EF027
:1044E8003CC01FF03DC020F03EC021F01D2A05D081
:1044F800D8901E361F36203621361D2EF9D734D0D7
:1045080050A43FD0146A156A166A176A8D0E4AECD1
:104518005BF0000901E037D1A6EC5DF02B0E0B6EC5
:104528000C6A0E6A100E0D6EC1EC57F0000901E11D
:104538002AD1300E406E03D0A6EC5DF04006405004
:10454800FBE135C01DF01D3A0F0E1D16100E1E6E34
:104558001F6A206A216A1D2A05D0D8901E361F3688
:10456800203621361D2EF9D71BC0D9FF1CC0DAFF13
:104578001EC0DEFF1FC0DEFF20C0DEFF21C0DEFF41
:1045880005D7146A156A166A176A090E4AEC5BF0B1
:10459800000901E0F8D02B0E0B6E0C6A0E6A100EA3
:1045A8000D6EC1EC57F0000901E1EDD050A232D0F8
:1045B80038C01DF0060E1E6ED8901D321E2EFCD778
:1045C800FF0E1D2635503F0B1F6E206AD8901F36F0
:1045D80020363644010B1F26000E20221F2A2022D7
:1045E8001D2A03D0D8901F3620361D2EFBD71F500A
:1045F800216E2050226E236A246A1BC0D9FF1CC07A
:10460800DAFF21C0DEFF22C0DEFF23C0DEFF24C0A8
:10461800DEFFBCD63650030B1D6E1E6AD8901D36C1
:104628001E36D8901D361E36D8901D361E363638A2
:10463800E842070B1D26000E1E221D2A1E223540A9
:10464800E8423F0B1F0B1F6E206A1F2A000E202214
:104658001D501F02F3CF21F0F4CF22F02002F350B7
:1046680022261E501F02F35022262150236E22506C
:10467800246E256A266A1BC0D9FF1CC0DAFF23C036
:10468800DEFF24C0DEFF25C0DEFF26C0DEFF7ED6AB
:1046980041C0D9FF42C0DAFF50C0DFFF77D6146AA5
:1046A800156A166A176A090E4AEC5BF000096BE195
:1046B80041C00BF042C00CF00E6A100E0D6EC1EC3A
:1046C80057F0000901E062D65ED0146A156A166ACE
:1046D800176A0A0E4AEC5BF0000955E141C00BF07D
:1046E80042C00CF00E6A100E0D6EC1EC57F0E9D7FF
:1046F800146A156A166A176A3A0E4AEC5BF00009E2
:1047080042E1040E406E0AD0A6EC5DF041C0D9FF2C
:1047180042C0DAFFDF6E414A422A4006405001E1BA
:1047280035D6F2D7146A156A166A176A8D0E4AECDE
:104738005BF0000928E1A6EC5DF041C00BF042C037
:104748000CF00E6A400E0D6EC1EC57F0BAD7040E8D
:104758003F6E19D01A501D6E1E6A1E50F8E11D508A
:1047680001E10FD6010A01E113D6020A01E1C8D618
:10477800090A8EE0010A93E0070AA7E0010AB8E0F7
:10478800030AD0E0E4D7B9EC5DF03F5012006AC0EC
:104798006DF06BC06EF001017E6B7F6BF8D169C064
:1047A80046F06D0E476E6CC048F04750D96EDA6A15
:1047B800DECFF6FFDDCFF7FFF86A000EF86E0800CF
:1047C800F550250AD8A4C5D14750D96EDA6ADE2A31
:1047D800000EDD220101806B816B846B856B826921
:1047E80083694750D96EDA6ADECFF6FFDDCFF7FF6F
:1047F800F86A000EF86E0800F550780AD8B40FD0A1
:104808004750D96EDA6ADECFF6FFDDCFF7FFF86AD8
:10481800000EF86E0800F550580AD8A470D1475019
:10482800D96EDA6ADECFF6FFDDCFF7FFF86A000E41
:10483800F86E0800F5CF68F04750D96EDA6ADE2ABC
:10484800000EDD224850D96EDA6ADF50DF2ADF2AEF
:10485800D96EDA6ADECF49F0DDCF4AF049C060F0A0
:104868004AC061F00001626B636B646B656B666BD9
:10487800676B46C024F060C025F061C026F062C0B6
:1048880027F063C028F064C029F065C02AF066C02C
:104898002BF067C02CF068C02DF0010183BF01D058
:1048A800849383BF05D0835107E18205D8B004D033
:1048B800376A010E366E04D082C136F083C137F0F4
:1048C80080C140F081C141F084A904D0FE0E402689
:1048D800FF0E412225C038F026C039F027C03AF033
:1048E80028C03BF029C03CF02AC03DF02BC03EF068
:1048F8002CC03FF0436A1F0E426E02019F6B6DD0C1
:104908004206D8A043060F0E3814446E456A45BEC9
:1049180008D0455004E10A0E445CD8A002D0570ED6
:1049280001D0300E4426000E4522BF0E2E6E2F6891
:104938002D50306E316A2E5030262F503122315092
:1049480005E11A0E305C02E2010E01D0000E326E53
:10495800336A32503310D8B425D09F0E2E6E2F688C
:10496800200E4410306E000E4510316E2E50302649
:104978002F503122315005E11A0E305C02E2010E4F
:1049880001D0000E346E356A34503510D8B40AD0D0
:1049980044C011F045C012F0D6EC59F011C044F0F3
:1049A80012C045F0800E4224D96E020E4320DA6E02
:1049B80044C0DFFF3606D8A037064006D8A0410617
:1049C800040E2E6ED8903F323E323D323C323B329E
:1049D8003A32393238322E2EF5D743BE21D04350E1
:1049E80004E1020E425CD8A01BD0385039103A10AE
:1049F8003B103C103D103E103F10D8A481D737BE65
:104A080005D0375002E13604D8B07AD741BE08D075
:104A1800415003E14004D8A003D0010184B370D70A
:104A2800010184A916D04206D8A04306800E42246C
:104A3800D96E020E4320DA6E2DC0DFFF4206D8A0E1
:104A48004306800E4224D96E020E4320DA6E300EE1
:104A5800DF6E24C01AF0800E42241B6E020E432023
:104A68001C6E40C01DF041C01EF084A108D01BC0C0
:104A780014F01CC015F01AC016F02EEC5CF01EBE27
:104A880005D01DC022F01EC023F002D0226A236A7E
:104A9800206A216A0AD0000E0D6E200E0C6E1AC014
:104AA8000EF05BEC54F0204A212A2250205C215061
:104AB800800A1F6E2350800A1F58D8A0ECD7010126
:104AC80084B108D01BC014F01CC015F01AC016F031
:104AD8002EEC5CF01BC00BF01CC00CF03AEC5AF04A
:104AE80022500B241A6E23500C201B6E1AC024F07F
:104AF8001BC025F024C046F025C047F043D04750DE
:104B0800D96EDA6ADECFF6FFDDCFF7FFF86A000E5E
:104B1800F86E0800F550250AD8A412D04750D96E6F
:104B2800DA6ADE2A000EDD22000E0D6E250E0C6EEE
:104B380046C00EF05BEC54F0476A010E466E22D078
:104B48004750D96EDA6ADE2A000EDD22466A476AC5
:104B580019D04750D96EDA6ADECFF6FFDDCFF7FFFE
:104B6800F86A000EF86E0800F5500C6E0D6A46C023
:104B78000EF05BEC54F04750D96EDA6ADE2A000E6C
:104B8800DD22DAD7465001017E2747507F236DC0CA
:104B9800F6FF6EC0F7FF0800F55001E000D67EC1B1
:104BA80069F07FC16AF0120020EE04F0A651D92600
:104BB800A751DA22DECFAAF0DDCFABF0AA29B36F76
:104BC800000EAB21B46FB311D8B4040C20EE0EF074
:104BD800A651D926A751DA22DE50DE10DE10DE10EB
:104BE80001E1040CB3C0AAF00F0EAA1701E094D19A
:104BF80020EE0EF0A651D926A751DA22DE2A000EA1
:104C0800DE22DE22DE2220EE0AF0A651D926A751A6
:104C1800DA22DE50DE10DE10DE1011E1A6C0D9FF68
:104C2800A7C0DAFF10EE08F0DE50E126DD50E222E0
:104C3800E650B35DE650B45901E26ED1040CB3C03E
:104C4800AAF0B4C0ABF0040EAC6FD890AB33AA3363
:104C5800AC2FFBD7AD69AE69A6C0D9FFA7C0DAFFF4
:104C680010EE02F0DE50E126DD50E222E750AF6F91
:104C7800B06BAD51AF27AE51B023AA51AF17AB51AE
:104C8800B017AF51B01101E047D1A6C0D9FFA7C0F6
:104C9800DAFFDECF44F0DDCF45F020EE0AF0A65172
:104CA800D926A751DA22DECF46F0DECF47F0DECF95
:104CB80048F0DECF49F0A2EC1FF044C0B5F045C083
:104CC800B6F046C0B7F047C0B8F00001B851B71108
:104CD800B61104E1020EB55D01E2020CB52907E147
:104CE800B62905E1B72903E1B82901E1010CA6C0FD
:104CF800D9FFA7C0DAFF10EE12F0DE50E126DD5032
:104D0800E222E650B55DE650B659E650B759E6508E
:104D1800B85901E2D2D0A851A91101E1040CA6C0EA
:104D2800D9FFA7C0DAFFDECF8FF0DDCF90F020EEFD
:104D38000AF0A651D926A751DA22DECF91F0DECFAC
:104D480092F0DECF93F0DECF94F0FBEC34F08FC01E
:104D5800B5F090C0B6F091C0B7F092C0B8F0B551B8
:104D6800B611B711B81101E1070CB505B611B711A5
:104D7800B81101E1020CB52907E1B62905E1B72907
:104D880003E1B82901E1010CA6C0D9FFA7C0DAFFE9
:104D9800DECF24F0DDCF25F003EC49F0000901E077
:104DA800010CA6C0D9FFA7C0DAFFDECFAAF0DDCF7D
:104DB800ABF02E0E0001AA250B6E000EAB210C6E77
:104DC8000E6A0D6A020E106E0F6A87EC5CF0A6C0C0
:104DD800D9FFA7C0DAFFDECF0BF0DDCF0CF0B5C0EE
:104DE8000DF0B6C00EF0B7C00FF0B8C010F085ECEB
:104DF8004CF0A6C0D9FFA7C0DAFF10EE2AF0DE50AB
:104E0800E126DD50E2220BC0E6FF0CC0E6FF0DC034
:104E1800E6FF0EC0E6FF0001B16BB26B2BD0A6C057
:104E2800D9FFA7C0DAFF10EE04F0DE50E126DD500E
:104E3800E222010EE76EA6C0D9FFA7C0DAFFDECFD7
:104E480024F0DDCF25F003EC49F0000901E0010C66
:104E5800A6C0D9FFA7C0DAFF10EE2AF0DE50E1267F
:104E6800DD50E222E62A000EE622E622E6220001D2
:104E7800B14BB22BA6C0D9FFA7C0DAFF10EE02F0E3
:104E8800DE50E126DD50E222E750AA6FAB6BAA5153
:104E9800B15DAB51B259C3E3A6C0D9FFA7C0DAFFD1
:104EA80010EE2AF0DE50E126DD50E222B151E65E36
:104EB800B251E65A000EE65AE65A20EE0AF0A6511A
:104EC800D926A751DA22B5C0DEFFB6C0DEFFB7C0CB
:104ED800DEFFB8C0DEFFA6C0D9FFA7C0DAFFDECF6D
:104EE8000BF0DDCF0CF0B5C00DF0B6C00EF0B7C0BA
:104EF8000FF0B8C010F085EC4CF0000120EE0EF079
:104F0800A651D926A751DA220BC0DEFF0CC0DEFF5E
:104F18000DC0DEFF0EC0DEFF20EE04F0A651D9263C
:104F2800A751DA22B3C0DEFFB4C0DDFF0F0EB31500
:104F3800AA6FAB6B050ED890AA37AB37E82EFBD714
:104F4800A6C0D9FFA7C0DAFFDECFACF0DDCFADF049
:104F5800AA51AC27AB51AD232E0EAC27000EAD23C2
:104F680020EE12F0A651D926A751DA22ACC0DEFFF6
:104F7800ADC0DDFF000C000E846F020E856F340E8D
:104F8800866F0A0E876F020E896F886BDD0E8A6F37
:104F98008B6BC9EC15F0FC6FC00E606FFD0E616F76
:104FA800DDC062F0DEC063F08AEC5DF00001DF6B0B
:104FB800E06BDB6BDC6BE16BE26BE151BD0FD96E33
:104FC800DA6ADF6AE151CC0FD96EDA6A000EDF6E59
:104FD800E14BE22BE2BFF1D7E25103E10F0EE15DB5
:104FE800ECE3E36BE46B30D1340EE325D96E0A0EA3
:104FF800E421DA6E0D0EDE1801E0EBD08B0E0B6E9D
:10500800FF0E0C6EBD0E0D6E3EEC53F00B500C10E7
:1050180007E1CC0E126E0CEC4DF012500101FD6F41
:10502800850E0B6EFF0E0C6EBD0E0D6E3EEC53F032
:105038000B500C1007E1CC0E126E0CEC4DF0125018
:105048000101A06F6A0E0B6EFF0E0C6EBD0E0D6E89
:105058003EEC53F00B500C1007E1CC0E126E0CEC2A
:105068004DF0125001019C6FD00E0B6EFF0E0C6EAE
:10507800BD0E0D6E3EEC53F00B500C1007E1CC0E3C
:10508800126E0CEC4DF0125001019A6FD40E0B6E9B
:10509800FF0E0C6EBD0E0D6E3EEC53F00B500C1057
:1050A80007E1CC0E126E0CEC4DF012500101F16FBD
:1050B8000001E56BE66BAE0E6F6F706B710E716F72
:1050C800FF0E726FE5C073F0E6C074F0F4EC5AF0AE
:1050D800AE0E0B6E0C6ABD0E0D6E3EEC53F00B500F
:1050E8000C1018E10F0E0001E503F3CFACF0F4CF7C
:1050F800ADF0E603F350AD27340EAC250B6E0C0E65
:10510800AD210C6ECC0E0D6E0E6A106A0F0E0F6E6E
:105118004BEC58F00001E54BE62BE6BFCCD7E65147
:1051280003E1100EE55DC7E3E66B010EE56FAE0E19
:105138006F6F706B780E716FFF0E726FE5C073F052
:10514800E6C074F0F4EC5AF0AE0E0B6E0C6ABD0EAD
:105158000D6E3EEC53F00B500C1018E10F0E0001D1
:10516800E503F3CFACF0F4CFADF0E603F350AD2791
:10517800240EAC250B6E0D0EAD210C6ECC0E0D6EF3
:105188000E6A106A0F0E0F6E4BEC58F00001E54BDB
:10519800E62BE6BFCCD7E65103E1040EE55DC7E395
:1051A800E16BE26BE151BD0FD96EDA6ADF6AE1515A
:1051B800CC0FD96EDA6A000EDF6EE14BE22BE2BF4C
:1051C800F1D7E25103E10F0EE15DECE3DB6BDC6B41
:1051D80015D0340EE325D96E0A0EE421DA6E0A0ED4
:1051E800DE1830E0340EE325D96E0A0EE421DA6EBB
:1051F800200EDE1806E1DC6B010EDB6FDF6BE06B67
:1052080021D0DB51DC1109E0340EE325D96E0A0EFA
:10521800E421DA6EDF51CC0F08D0340EE325D96EC5
:105228000A0EE421DA6EDF51BD0FE16EE26ADFCFCC
:10523800E7FFE0BF05D0E05105E10F0EDF5D02E2B8
:10524800DF4BE02BE34BE42BDD51E35DDE51E4590A
:1052580001E2CAD6B00E606FFD0E616F9CC162F0AC
:10526800636B8AEC5DF01B0E0001606FFE0E616FD0
:10527800FDC162F0636B8AEC5DF00C0E0001606F9B
:10528800FE0E616FA0C162F0636B8AEC5DF00001F5
:10529800E56BE66B4E0E606FFD0E616FE5C062F068
:1052A800E6C063F00F0EE503F3CFACF0F4CFADF03A
:1052B800E603F350AD27340EAC25646F0C0EAD2118
:1052C800656F8AEC5DF00001E54BE62BE6BFE2D79F
:1052D800E65103E1100EE55DDDE3E46B010EE36FDB
:1052E8005F0E606FFD0E616FE3C062F0E4C063F0B3
:1052F8000F0EE303F3CFACF0F4CFADF0E403F350BB
:10530800AD27240EAC25646F0D0EAD21656F8AECB8
:105318005DF00001E34BE42BE4BFE2D7E45103E185
:10532800040EE35DDDE35E0E606FFC0E616F8AEFD5
:105338005DF018C0F6FF19C0F7FF0800F5CF46F07A
:10534800184A192A465001E11200250E461804E0B1
:10535800465075EC5DF0EDD7416A426A18C0F6FF19
:1053680019C0F7FF0800F5CF46F0184A192A300E81
:1053780046180DE1426A010E416E18C0F6FF19C0C9
:10538800F7FF0800F5CF46F0184A192A06D02D0E67
:10539800461803E1426A020EEFD7396A3A6A1CD00E
:1053A8000A0E3902F3CF1BF0F4CF1CF03A02F35087
:1053B8001C2646501B26000E1C22D00E1B24396EBC
:1053C800FF0E1C203A6E18C0F6FF19C0F7FF080040
:1053D800F5CF46F0184A192A2F0E466403D0390E25
:1053E8004664DED76C0E461803E04C0E46180AE1F8
:1053F800418418C0F6FF19C0F7FF0800F5CF46F042
:10540800184A192A465001E1120046C045F0600EBC
:10541800456472D0200E455E6FD01A50D96EDA6A94
:10542800020EDF26DF5CD96EDA6ADECF35F0DECF1A
:1054380036F03B6A3C6A02D03B4A3C2A3B50352452
:105448001B6E3C5036201C6E1BC0F6FF1CC0F7FFBD
:10545800000EF86E0E0EF76403D00800F55005D064
:10546800F6CFE9FFF7CFEAFFEF50000904E0E4D7F1
:10547800200E75EC5DF041B20BD03B501B6E3C50DA
:105488001C6E3B4A3C2A39501B5C3A501C58F0E3CE
:1054980035C00CF036C00DF0A0EC58F003D0200E4B
:1054A80075EC5DF03B501B6E3C501C6E3B4A3C2A31
:1054B80039501B5C3A501C5801E33BD7F0D71A50BF
:1054C800D96EDA6ADF50DF2ADF2AD96EDA6ADF504E
:1054D80075EC5DF02ED7386A020E08D0386A080ECF
:1054E80005D0386A0A0E02D0386A100E376E19D005
:1054F800465075EC5DF01DD745501B6E1C6A1C505C
:10550800F7E11B50420AE7E0010AD9E0070AE9E09F
:105518000B0AE4E01C0A81E0060AE3E00D0AE4E075
:10552800E7D741B430D0440E451813E01A50D96E6D
:10553800DA6ADF50DF2ADF2AD96EDA6ADECF1BF09B
:10554800DDCF1CF01BC02DF01CC02EF02F6A306A76
:1055580011D01A50D96EDA6ADF50DF2ADF2AD96EE5
:10556800DA6ADECF2DF0DDCF2EF0000E2EBEFF0E54
:105578002F6E306E2DC03DF02EC03EF02FC03FF094
:1055880030C040F010D01A50D96EDA6A040EDF2607
:10559800DF5CD96EDA6ADECF3DF0DECF3EF0DECFDB
:1055A8003FF0DECF40F0440E45180CE140AE0AD083
:1055B8003D6C3E1ED8B03E2A3F1ED8B03F2A000E92
:1055C80040564186436A446A3DC00BF03EC00CF029
:1055D8003FC00DF040C00EF037C00FF038C010F0DB
:1055E800116A126A90EC57F00B50456E3DC00BF0F3
:1055F8003EC00CF03FC00DF040C00EF037C00FF0B9
:1056080038C010F0116A126A5BEC55F00BC03DF01F
:105618000CC03EF00DC03FF00EC040F0090E4564CE
:105628000BD0780E461803E0326A070E02D0326AB1
:10563800270E316E3150452643501D0FD96EDA6A58
:105648004550300FDF6E434A442A3D503E103F100C
:10565800401005E0445003E1100E435CB5E341A659
:1056680008D043501D0FD96EDA6A2D0EDF6E434AFB
:10567800442A43C03BF044C03CF041B003D0346AF4
:10568800200E02D0346A300E336E33C045F003D09A
:10569800455075EC5DF041B20BD03B501B6E3C5051
:1056A8001C6E3B4A3C2A39501B5C3A501C58F0E3AC
:1056B8004306D8A0440643501D0FD96EDA6ADF505E
:1056C80075EC5DF04350441004E0F2D7200E75EC01
:1056D8005DF03B501B6E3C501C6E3B4A3C2A3950D7
:1056E8001B5C3A501C5801E324D6F0D7106E0C50BE
:1056F80002E096EC55F00F6A0B5001E171D1109E53
:10570800040E101803E0140E101807E10101866B4F
:10571800876B0C6A070E0B6E070C3F0E101807E11B
:105728004B6A0101866B876B0B6A0C6A12005F0E6D
:10573800101807E14C6A0101866B876B0B6A0C6ACB
:1057480012003F0E106406D05F0E106003D0400EAA
:105758001018F0E1400E101809E1010E4C6E4B6A6A
:105768000101866B876B0B6A0C6A1200200E1018F9
:1057780001E036D1010E4B6EF3D7600E101809E127
:105788004C5007E001019551080ED8B4030E0F6E76
:1057980073D0600E101809E14B5007E001019551D4
:1057A80002E0090E14D0050E12D0680E101809E197
:1057B8004B5007E01A0E0101876F900E04D18380C9
:1057C80069D1680E101805E14C5003E0020E0F6E07
:1057D80053D06A0E101807E14B5005E01A0E01016C
:1057E800876FF40EF0D06C0E101807E14B5005E0EF
:1057F8001A0E0101876F2C0EE6D0700E101808E102
:105808004C5006E0040E0F6E0101866B876BD7D7EC
:10581800700E101801E03ED14B5001E13BD11B0E38
:105828000101876F620ECFD08380020E101805E148
:105838001A0E0101876F920E866F050E101805E18A
:105848001A0E0101876FAE0E866F070E101805E15C
:105858001A0E0101876FB80E866F080E101805E141
:105868001A0E0101876FCC0E866F030E101802E026
:10587800102806E10F6A83900101866B876B0AD1B5
:10588800160E101801E006D11A0E0101876FA40E3A
:105898008BD0050E101801E0FDD01A0E0101876F9C
:1058A800F50E82D010C04FF01A0E0101876F9B0EC3
:1058B8007BD01A0E0101876F9C0E76D04F50070DD2
:1058C800500EF324D96E010EF420DA6E10C0DFFFFB
:1058D8001A0E0101876F9D0E67D04F50070D510EAC
:1058E800F324D96E010EF420DA6E10C0DFFF1A0E11
:1058F8000101876F9E0E58D04F50070D520EF324AA
:10590800D96E010EF420DA6E10C0DFFF0101866B3C
:10591800876B010E17D01A0E0101876FB90E53D08D
:105928001A0E0101876FBA0E3FD01A0E0101876F58
:10593800BB0E3AD00101866B876B3DD00101866BA7
:10594800876B060E0F6EA6D010C04FF00101866B54
:10595800876B0F6A30D00101956B1A0E876FF70EAF
:10596800866F29D01A0E0101876FF70E1DD083901C
:10597800270E0101876F0F0E17D0180E101801E0BF
:1059880089D01A0E0101876F2D0E0ED01A0E010153
:10599800876F2E0E09D01A0E0101876F2F0E04D0C3
:1059A8001A0E0101876F300E866F74D00101866B65
:1059B800876B0A0E0F6E83906DD0040E0F6E270E44
:1059C8000101876F0F0E866FFAD68380010104D01C
:1059D8008390010E0101956F866B876B0F6A5AD011
:1059E80086C10DF087C10EF00E5007E01A0A09E0D3
:1059F800010A48E03C0A4CE04DD00D5001E1BDD60B
:105A080049D00D502C0AB9E0010AC0E0030AC3E0EE
:105A1800010AC6E01F0ACAE0A00A01E105D7020A86
:105A280001E140D7090A01E144D7070A01E146D755
:105A3800010A01E152D7030A01E15ED73A0A01E1FE
:105A48007DD70A0AC5E0160A01E165D7010A01E116
:105A580067D7030A01E169D7010A01E16BD7790A1F
:105A680001E1B4D60E0A01E16FD7380A01E111D776
:105A7800010A01E170D7030A01E174D7010A01E1C3
:105A880076D708D00D50580A98E03A0A9EE002D01E
:105A98000D500F0A0FC00BF00C6A1200000E000127
:105AA800F66F0A0EF56F000EF46F050EF36F8ED1C8
:105AB800F66B140EF56F82D1610E0C6EFC0E0D6E36
:105AC800A0EC58F08FB204D00001F66B1E0EF56FF3
:105AD800090E0001F26F1E0EF16FE40EE82EFED7DC
:105AE800F12FFCD7F22FFAD700F068D1DB0E0C6E3D
:105AF800FE0E0D6EA0EC58F0060E0001D26F080ED7
:105B0800D36F600ED46FFC0ED56FD66BF3EC52F0EA
:105B1800FC6FFC51F3EC58F00001FC51D9E1F66B35
:105B2800230ED5D72A0E0C6EFE0E0D6EA0EC58F083
:105B3800000E0001D26F020ED36F090ED46FFF0E54
:105B4800D56F010ED66FE2EC1AF00001FC6FFC5124
:105B5800F3EC58F00001FC510AE1BFEC27F0000E0D
:105B6800486E020E496E9CEC5BF00001FC6FFC5124
:105B7800F3EC58F0000E0001F66F250EF56F0101E9
:105B88009C510DE1FE6B340E00016F6F0C0E706FAF
:105B9800A80E716FFE0E726FF4EC5AF00DD0C50EA0
:105BA8000001606FF80E616F9CC162F0636BFEC10B
:105BB80064F0656B8AEC5DF0390E0001606FFE0ED3
:105BC800616F0101FE510F0D340EF3240001626F65
:105BD8000C0EF420636F8AEC5DF07AD73D0E0C6EE4
:105BE800FD0E0D6EA0EC58F0000E0001D26F020EF3
:105BF800D36F9B0ED46FFE0ED56F010ED66FE2ECFD
:105C08001AF00001FC6FFC51F3EC58F00001FC5154
:105C18000AE1A7EC3EF0000E486E020E496E9CECBD
:105C28005BF00001FC6FFC51F3EC58F0000E000132
:105C3800F66F280EF56F01019C510DE1FE6B340ED5
:105C480000016F6F0C0E706FA80E716FFE0E726FF1
:105C5800F4EC5AF00DD0C50E0001606FF80E616FBC
:105C68009CC162F0636BFEC164F0656B8AEC5DF009
:105C7800390E0001606FFE0E616F0101FE510F0DBC
:105C8800340EF3240001626F0C0EF420636F8AEC6B
:105C98005DF01ED7CB0E606FFB0E616F0101FE51E8
:105CA8000F0D340EF3240001626F0C0EF420636FA5
:105CB8008AEC5DF0000E0001D26F020ED36F010175
:105CC800FE510F0D340EF3240001D46F0C0EF42096
:105CD800D56F030ED66FE2EC1AF00001FC6FFC5191
:105CE800F3EC58F00001FC5103E1F66B3C0EF56F44
:105CF800040EFC1901E0ECD6F66B320EE8D6F80E6D
:105D0800606FFC0E616F0101FE510F0D340EF3241C
:105D18000001626F0C0EF420636F8AEC5DF0000ED8
:105D28000001D26F020ED36F0101FE510F0D340E28
:105D3800F3240001D46F0C0EF420D56F070ED66F34
:105D4800E2EC1AF00001FC6FFC5101E0C1D6F66BE1
:105D58003C0EBDD69C0E606FFC0E616F0101FE51BA
:105D68000F0D340EF3240001626F0C0EF420636FE4
:105D78008AEC5DF00001F06B010EEF6F010CF5C0CD
:105D8800F1F0F6C0F2F0F25119E1F1510A0A01E11D
:105D98008FD61E0A01E190D60A0A01E1A7D63D0A6C
:105DA80001E1C0D6060A01E119D70D0A01E172D74F
:105DB800050A04E01F0AA3E00E0ACCE0140E000155
:105DC800F519F61103E0F307D8A0F407F4BF04D0DF
:105DD800F451D5E1F305D3E2EF6BF06B120000014B
:105DE800C16B010EC06F1C0E606FF50E616FCECFD8
:105DF80062F0636BCDCF64F0656B4F50070D500EAA
:105E0800F324D96E010EF420DA6EDF50666F676BEB
:105E18004F50070D510EF324D96E010EF420DA6E9F
:105E2800DF50686F696B4F50070D520EF324D96E1F
:105E3800010EF420DA6EDF506A6F6B6B4F50070D5E
:105E4800510EF324D96E010EF420DA6EDF50AC6FD8
:105E5800ACC0ADF0AE6BAF6BB06B040ED890AD3785
:105E6800AE37AF37B037E82EF9D74F50070D500E81
:105E7800F324D96E010EF420DA6EDF50B16FB1C091
:105E8800B2F0B36BB46BB56B050ED890B237B337BD
:105E9800B437B537E82EF9D7AD51B225B66FAE5144
:105EA800B321B76FAF51B421B86FB051B521B96FF5
:105EB8004F50070D520EF324D96E010EF420DA6EFE
:105EC800DF50B6256C6F000EB7216D6F000EB8213C
:105ED8006E6F000EB9216F6F8AEC5DF0838E838040
:105EE8000001BA6BBB6BBC6BBD6BF8D04F50200D7B
:105EF800000EF324846F020EF420856F340E866F33
:105F08000A0E876F010E896F886BC80E8A6F8B6BBC
:105F1800C9EC15F0C00E606FF80E616FC8C062F072
:105F2800C9C063F08AEC5DF04F50070D530EF3249F
:105F3800D96E010EF420DA6E74C1B1F075C1B2F0F9
:105F480076C1B3F00001B06B000EB025B46F010E3E
:105F5800B121B56F000EB221B66F000EB321B76F35
:105F6800DE50B41947E1DE50B51944E1DE50B619E8
:105F780041E1DE50B7193EE15CEC57F00FC0C4F0C8
:105F880010C0C5F011C0C6F012C0C7F0000EE8CFAF
:105F980034FA2AEE35F0C7C0DFFFE8CF36FA2AEE2A
:105FA80037F0C6C0DFFFE8CF38FA2AEE39F0C5C0AF
:105FB800DFFFE8CF3AFA2AEE3BF0C4C0DFFF730EEA
:105FC8000001606FF60E616F2AEE35F0DF50626FE8
:105FD800636B2AEE37F0DF50646F656B2AEE39F099
:105FE800DF50666F676B2AEE3BF0DF50686F696BB6
:105FF8008AEC5DF00101FF93C8C048F0C9C049F0C0
:10600800A4EC37F048C0C2F049C0C3F00001C25147
:10601800BA27C351BB23000EBC23BD238EAC63D06B
:10602800C851C21903E1C951C3190FE0050E80EC2C
:106038005DF0810E0001606FFE0E616FC2C062F0FC
:10604800C3C063F08AEC5DF04ED02CEC5DF00DEC33
:106058005DF00B500C1011E0D00E0001606FFD0ECA
:10606800616F0DEC5DF00BC062F00CC063F08AEC60
:106078005DF0010E0101966F36D00001BF6B050E71
:10608800BE6F1CD0D00E0001AC6FC90EE82EFED733
:10609800AC2FFCD700D00DEC5DF00B500C100EE0CF
:1060A8000001C06BC16B700E606FFD0E616FBEC0EA
:1060B80062F0BFC063F08AEC5DF008D00001BE0753
:1060C800D8A0BF07BE29DEE1BF29DCE10DEC5DF0F9
:1060D8000B500C1003E00001C06BC16B0001C051F4
:1060E800C11101E003D7F80E0001606FF90E616F6E
:1060F800CECF62F0636BCDCF64F0656BBAC066F04B
:10610800BBC067F0BCC068F0BDC069F08AEC5DF048
:106118000101966B839E8390120043C024F044C013
:1061280025F003EC49F0456E455001E08FD143C09E
:10613800D9FF44C0DAFF030EDE1801E077D120EE64
:1061480005F04350D9264450DA22DE0401E06ED12E
:106158002E0E43240B6E000E44200C6E0E6A0D6A40
:10616800020E106E0F6A87EC5CF022EE2CF04350A2
:10617800D9264450DA22550EDF6E22EE2DF0435018
:10618800D9264450DA22AA0EDF6E20EE2EF04350B4
:10619800D9264450DA22520EDF6E20EE2FF04350FB
:1061A800D9264450DA22520EDF6E20EE30F04350EA
:1061B800D9264450DA22610EDF6E20EE31F04350CA
:1061C800D9264450DA22410EDF6E22EE12F04350F7
:1061D800D9264450DA22720EDF6E22EE13F04350B5
:1061E800D9264450DA22720EDF6E22EE14F04350A4
:1061F800D9264450DA22410EDF6E22EE15F04350C4
:10620800D9264450DA22610EDF6E20EE0EF043509C
:10621800D9264450DA2212EE16F04350E1264450B3
:10622800E222DFCFE7FF22EE17F04350D926445091
:10623800DA2210EE0EF04350E1264450E222E6CF77
:1062480060F0E5CF61F061C060F00001616B605102
:10625800DF6E22EE18F04350D9264450DA2210EEB1
:106268000EF04350E1264450E222E6CF60F0E6CF3C
:1062780061F0E6CF62F0E6CF63F0110E05D0D8905A
:106288006333623361336033E82EF9D76051DF6ED0
:1062980022EE19F04350D9264450DA2210EE0EF0BF
:1062A8004350E1264450E222E6CF60F0E6CF61F0A9
:1062B800E6CF62F0E6CF63F0190E05D0D8906333CD
:1062C800623361336033E82EF9D76051DF6E20EE18
:1062D8000AF04350D9264450DA2212EE1AF04350FD
:1062E800E1264450E222DFCFE7FF22EE1BF04350C5
:1062F800D9264450DA2210EE0AF04350E1264450E1
:10630800E222E6CF60F0E5CF61F061C060F0616B3A
:106318006051DF6E22EE1CF04350D9264450DA2239
:1063280010EE0AF04350E1264450E222E6CF60F036
:10633800E6CF61F0E6CF62F0E6CF63F0110E05D04C
:10634800D8906333623361336033E82EF9D76051F4
:10635800DF6E22EE1DF04350D9264450DA2210EEAB
:106368000AF04350E1264450E222E6CF60F0E6CF3F
:1063780061F0E6CF62F0E6CF63F0190E05D0D89051
:106388006333623361336033E82EF9D76051DF6ECF
:1063980020EE1AF04350D9264450DA22DECF60F0BE
:1063A800DECF61F0DECF62F0DECF63F06029646F8C
:1063B800000E6121656F000E6221666F000E632179
:1063C800676F20EE2AF04350D9264450DA2264C081
:1063D800DEFF65C0DEFF66C0DEFF67C0DEFF2E0E93
:1063E80043241A6E000E44201B6E20EE2AF0435000
:1063F800D9264450DA22DECF1CF0DECF1DF0DECFE6
:106408001EF0DECF1FF0216A010E206E20EE01F093
:106418004350D9264450DA22DF507BEC4EF020EE70
:1064280005F04350D9264450DA22DF6A1A6A1B6AFB
:106438001C6A20EE01F04350D9264450DA22DF507E
:10644800B8EC21F0000902E0010E456E455012003B
:10645800838E83804D6A040E0001606FF70E616FB2
:10646800CECF62F0636BCDCF64F0656B4F50140DE7
:10647800070EF324D96E010EF420DA6EDECF66F033
:10648800DECF67F0DECF68F0DECF69F04F50140D35
:10649800070EF324D96E010EF420DA6EDECF6AF00F
:1064A800DECF6BF0DECF6CF0DECF6DF08AEC5DF006
:1064B800E0EC43F0CDC0B3F1CEC0B4F10101B3516B
:1064C800B41105E0B3C1EDF0B4C1EEF01200AE6B4B
:1064D800AF6BB06BB16BAD6B010EAC6FB76B0BD123
:1064E800B56BB66B1CD00DEC5DF00B500C1013E0C7
:1064F800B70E0B6E010E0C6E17EC54F00101AB6F6A
:10650800000E5324D96EDA6A030EDA22ABC1DFFF1C
:10651800532AB54BB62B0101B7AB8EAC04D0B6BF2E
:10652800E2D7B605E0E3B5C1EFF0B6C1F0F0000E72
:106538000001F0BFFF0EF16FF26FEF510101AE27BE
:106548000001F0510101AF230001F1510101B02315
:106558000001F2510101B1234F50140D0F0EF32425
:10656800D96E010EF420DA6EDE50AE5DDE50AF5902
:10657800DE50B059DE50B15902E3AC6BAD6BB7AB2E
:1065880002D0AC6BAD6B8EBC02D0AC6BAD6B535014
:106598000EE0DF0E0001606FFA0E616FB3C162F0AA
:1065A800B4C163F053C064F0656B8AEC5DF001011F
:1065B800B6BF02D0B60519E2000E53240B6E0C6A62
:1065C800030E0C22FF0E5324D96EDA6A020EDA2269
:1065D800DF500D6E0E6A535000080F6E000ED8A0E3
:1065E800E82A0108106E3CEC4AF04F50140D070ED3
:1065F800F324D96E010EF420DA6E74C1F4F075C17B
:10660800F5F076C1F6F00001F36B000EF325F76F95
:10661800010EF421F86F000EF521F96F000EF62136
:10662800FA6FDE50F7193CE1DE50F81939E1DE5017
:10663800F91936E1DE50FA1933E101C3BBF103C39E
:10664800BAF105C3B9F107C3B8F1B8C10EF0B9C1C1
:106658000FF0BAC110F0BBC111F0CAEC58F04B0EE4
:106668000001606FF50E616FCECF62F0636BCDCF26
:1066780064F0656B2AEE34F0DF50666F676B2AEEC4
:1066880035F0DF50686F696B2AEE36F0DF506A6FBD
:106698006B6B2AEE37F0DF506C6F6D6B8AEC5DF038
:1066A8000AEC56F0E4510101B26FB25124E0270E12
:1066B8000001606FFB0E616FB2C162F0636B8AEC20
:1066C8005DF0010E4D6E4F50140D130EF324D96E6C
:1066D800010EF420DA6E4F50140D130EF324E16E00
:1066E800010EF420E26EE7500409DF6E4DC0EDF0B4
:1066F8000001EE6B1200AC51AD1101E0F1D64D0E68
:106708000001606FF60E616FCECF62F0636BCDCF84
:1067180064F0656BAEC166F0AFC167F0B0C168F0F8
:10672800B1C169F08AEC5DF08FA402D0010E4D6E04
:106738008390839E0001ED6BEE6B12001550D96EAD
:10674800DA6ADECF22F0DDCF23F002D0224A232AF4
:1067580022C0F6FF23C0F7FF000EF86E0E0EF76496
:1067680003D00800F55005D0F6CFE9FFF7CFEAFFD0
:10677800EF502F0AEBE022C0F6FF23C0F7FF000E10
:10678800F86E0E0EF76403D00800F55005D0F6CF6A
:10679800E9FFF7CFEAFFEF505C0AD8E020EE14F0EB
:1067A8001350D9261450DA22DECF24F0DDCF25F09D
:1067B80024C00BF025C00CF00E6A200E0D6E106A76
:1067C8000B0E0F6E87EC5CF01E6A1EC026F0276A5F
:1067D80026C01CF027C01DF0206A080E1F6E1C5032
:1067E8002224166E1D502320176E16C0F6FF17C000
:1067F800F7FF000EF86E0E0EF76403D00800F55090
:1068080005D0F6CFE9FFF7CFEAFFEF50286E1C4A14
:106818001D2A200E2864A7D02F0E281801E1A3D026
:106828005C0E281801E19FD02E0E281805E01F5095
:10683800265C2050275814E3080E1F182010D8A4EF
:10684800060C2E0E281801E0060C276A080E266E84
:10685800206A0B0E1F6ED8901E36D8901E36BFD7F2
:106868007F0E286402D0030E1E12800E286403D007
:106878009F0E286406D0DF0E28644CD0FD0E2860D9
:1068880049D01C502224166E1D502320176E16C0A6
:10689800F6FF17C0F7FF000EF86E0E0EF76403D070
:1068A8000800F55005D0F6CFE9FFF7CFEAFFEF5023
:1068B800216E1C4A1D2A3F0E216403D07E0E2164DE
:1068C80006D07F0E2164060CFD0E2160060C1668AA
:1068D80017681FC018F020C019F016501826175056
:1068E80019221850265C1950275801E3060C265027
:1068F8002424D96E27502520DA6E28C0DFFF264AC7
:10690800272A26502424D96E27502520DA6E21C044
:10691800DFFF26D0EE0E0B6EFD0E0C6E28C00DF0BC
:106928000E6A2EEC5BF00B500C1001E0060C400ECA
:10693800286405D05B0E286002D01E8209D0600E44
:10694800286406D07B0E286003D01E80200E285EA7
:1069580026502424D96E27502520DA6E28C0DFFF60
:10696800264A272A3CD71C502224166E1D50232065
:10697800176E1550D96EDA6A16C0DEFF17C0DDFF34
:10698800200E286403D01A6A1B6A03D01B6A040EFF
:106998001A6E1AC028F02650271001E1060C24C0F0
:1069A800D9FF25C0DAFFE50EDE1806E124C0D9FFBD
:1069B80025C0DAFF050EDF6E080E1F18201004E14F
:1069C800D8901E36D8901E361E50030BE80601E1FB
:1069D80028881E500C0B040A01E1288620EE0BF0D3
:1069E8002450D9262550DA2228C0DFFF000C915107
:1069F80092119311941128E120EE0AF08F51D926B3
:106A08009051DA22DECF9AF0DECF9BF0DECF9CF0F9
:106A1800DECF9DF09A519B119C119D110FE020EE45
:106A280012F08F51D9269051DA22DE509A5DDE504D
:106A38009B59DE509C59DE509D5952E3010E9A6FC6
:106A48009B6B9C6B9D6B4CD08FC044F090C045F005
:106A580091C046F092C047F093C048F094C049F006
:106A6800A2EC1FF044C0A2F045C0A3F046C0A4F0B9
:106A780047C0A5F00001A551A411A31109E1020E18
:106A8800A25D06E2010E8F6F906B916B926B000C0A
:106A9800A2290FE1A3290DE1A4290BE1A52909E108
:106AA800A2C08FF0A3C090F0A4C091F0A5C092F04E
:106AB800120020EE12F08F51D9269051DA22DE50C2
:106AC800A25DDE50A359DE50A459DE50A559E8E373
:106AD80091C09AF092C09BF093C09CF094C09DF036
:106AE8009AC09EF09BC09FF09CC0A0F09DC0A1F0F2
:106AF8009E2B000E9F23A023A12320EE12F08F517E
:106B0800D9269051DA22DE509E5DDE509F59DE5024
:106B1800A059DE50A15911E3020E9E6F9F6BA06B26
:106B2800A16B9D519C119B1108E1020E9A5D05E233
:106B38008F6B906B916B926B12008FC044F090C07A
:106B480045F09EC046F09FC047F0A0C048F0A1C0E5
:106B580049F0A2EC1FF044C0A2F045C0A3F046C023
:106B6800A4F047C0A5F00001A251A311A411A511DA
:106B78001AE0A22906E1A32904E1A42902E1A52932
:106B88008FE0A205A311A411A5118AE09A519E19BC
:106B9800AFE19B519F19ACE19C51A019A9E19D510E
:106BA800A119C6E0A5D78FC060F090C061F09EC063
:106BB80062F09FC063F0A0C064F0A1C065F0666990
:106BC800676968690F0E696F45EC1DF0996F9951F7
:106BD8001CE1915192119311941117E08FC060F04C
:106BE80090C061F091C062F092C063F093C064F00D
:106BF80094C065F09EC066F09FC067F0A0C068F0C2
:106C0800A1C069F045EC1DF0996F995130E120EE73
:106C18000AF08F51D9269051DA229EC0DEFF9FC01C
:106C2800DEFFA0C0DEFFA1C0DEFF20EE0EF08F5118
:106C3800D9269051DA22DE2806E1DE2804E1DE2892
:106C480002E1DE2821E020EE0EF08F51D926905186
:106C5800DA22DE06000EDE5ADE5ADE5A20EE05F093
:106C68008F51D9269051DA22000EDB800DD099057C
:106C780007E0010E9E6F000E9F6BA06BA16B04D006
:106C88009E699F69A069A1699EC08FF09FC090F01E
:106C9800A0C091F0A1C092F0120020EE04F084513F
:106CA800D9268551DA2286C0DEFF87C0DDFF20EEB7
:106CB80006F08451D9268551DA22DECF95F0DECF51
:106CC80096F0DECF97F0DECF98F0950596119711E4
:106CD8009811D8B4020C84C0D9FF85C0DAFF10EE31
:106CE80012F0DE50E126DD50E222E650955DE650D6
:106CF8009659E6509759E650985901E3020C955178
:106D080096119711981121E184C0D9FF85C0DAFF47
:106D1800DECF88F0DDCF89F088C0D9FF89C0DAFFDF
:106D2800030EDE1812E184C0D9FF85C0DAFF10EE29
:106D380022F0DE50E126DD50E222E6CF95F0E6CFE4
:106D480096F0E6CF97F0E6CF98F095519611971107
:106D5800981123E184C0D9FF85C0DAFF10EE08F04E
:106D6800DE50E126DD50E222E650865DE650875986
:106D780001E3020C84C0D9FF85C0DAFF10EE22F0CF
:106D8800DE50E126DD50E222E6CF91F0E6CF92F028
:106D9800E6CF93F0E6CF94F074D084C0D9FF85C0D5
:106DA800DAFF10EE02F0DE50E126DD50E222E75075
:106DB800100DF3CF8FF0F4CF90F044D084C0D9FFFA
:106DC80085C0DAFFDECF44F0DDCF45F095C046F050
:106DD80096C047F097C048F098C049F0A2EC1FF061
:106DE80044C095F045C096F046C097F047C098F06B
:106DF8000001952907E1962905E1972903E19829DA
:106E080001E1010C98519711961104E1020E955D6C
:106E1800D8A0020C84C0D9FF85C0DAFF10EE12F0AA
:106E2800DE50E126DD50E222E650955DE6509659A7
:106E3800E6509759E650985901E3020C8F51865F46
:106E48009051875B8F51865D90518759B7E284C016
:106E5800D9FF85C0DAFFDECF0BF0DDCF0CF095C08F
:106E68000DF096C00EF097C00FF098C010F085ECAA
:106E78004CF00BC091F00CC092F00DC093F00EC016
:106E880094F0000120EE0AF08451D9268551DA22C7
:106E980095C0DEFF96C0DEFF97C0DEFF98C0DEFF1C
:106EA800915192119311941101E1020C86C088F05E
:106EB80087C089F0040E8A6FD890893388338A2F67
:106EC800FBD7885191258B6F895192218C6F000EC9
:106ED80093218D6F000E94218E6F20EE0EF0845159
:106EE800D9268551DA228BC0DEFF8CC0DEFF8DC02B
:106EF800DEFF8EC0DEFF0F0E8615886F896B050ECC
:106F0800D89088378937E82EFBD784C0D9FF85C049
:106F1800DAFFDECF8AF0DDCF8BF088518A278951DE
:106F28008B232E0E8A27000E8B2320EE12F084511D
:106F3800D9268551DA228AC0DEFF8BC0DDFF000C1E
:106F4800526A0101906B916B898689808982898454
:106F580089888B68849084928494849883B40CD0B4
:106F6800F2A707D0980E0001606FF60E616F8AECE9
:106F78005DF0486A496A12000F011391350EE82E38
:106F8800FED700F015D18EA88EBA14D0C20E00011B
:106F9800606FFE0E616F010E8DA0000E626F636B55
:106FA800010E83A0000E646F656B52C066F0676BBC
:106FB8008AEC5DF08EB80AD0480E0001606FFE0EB4
:106FC800616F8AEC5DF0630E526EF7D0100E01010E
:106FD800786F270E796F7A6B7B6BD1D08EB28EA4C7
:106FE80011D001017807000E795B7A5B7B5B782909
:106FF80006E1792904E17A2902E17B29D8A4D8D0CD
:10700800620EA4D0010EA2D08EA8D2D0020E9ED0BD
:107018008669876948C088F049C089F08651882701
:1070280087518923010190510001881908E1010164
:1070380091510001891903E10101FFB3899A340EC6
:1070480001019025D96E0A0E9121DA6EDF1C866E39
:10705800904B912B8B6A030E526E100E786F270E91
:10706800796F7A6B7B6B06D08EA204D08990050E5F
:10707800526E0FD07807000E795B7A5B7B5B7829BC
:10708800F3E17929F1E17A29EFE17B2901E190D057
:10709800EBD7100E786F270E796F7A6B7B6B11D058
:1070A8008EA40FD0898A89808B684850905D915151
:1070B800800A0001866F4950800A8659A7E3630E4B
:1070C80045D07807000E795B7A5B7B5B7829E8E12D
:1070D8007929E6E17A29E4E17B296AE0E1D78EB2F1
:1070E8000ED001017807000E795B7A5B7B5B78290B
:1070F80008E1792906E17A2904E17B2902E1040EF5
:10710800526E8EA255D0040E21D08990050E526E73
:10711800100E0101786F270E796F7A6B7B6B48D060
:1071280089848EB40ED001017807000E795B7A5BF2
:107138007B5B782908E1792906E17A2904E17B2932
:1071480002E1060E526E8EA433D0060E526E30D077
:10715800898A89808B6848500101905D9151800A25
:107168000001866F4950800A865901E24BD7A7D79C
:107178009D0E606FFF0E616F8AEC5DF0A0D75250D4
:107188000001866F876B875113E1865101E126D78D
:10719800010A01E139D7030A01E13AD7010A9FE060
:1071A800070AB3E0010ABCE0030AD2E0640AE0E09F
:1071B800630E521802E08EBCE6D6898089828984E3
:1071C8008988898A8B680F01138190C148F091C121
:1071D80049F01200340E0101B76F0A0EB86FEDC006
:1071E8000BF0EEC00CF03AEC5AF00B500101AB6F0B
:1071F800CD0E0001A66FA76BA86BA96BAA6BAB6B32
:10720800DFEC12F00101B46FB4510DE0AD0E0001D6
:10721800606FFA0E616F8AEC5DF00001CD6BCE6B8A
:10722800CF6BD06B1200CD0E0001846F856BB7C198
:1072380086F0B8C187F0010E896F886BB20E8A6F2D
:10724800010E8B6FC9EC15F00101B46FB45108E061
:107258009D0E0001606FFB0E616F8AEC5DF0DDD75B
:10726800B7C1D9FFB8C1DAFF800EDE1808E02C0ECE
:107278000001606FFD0E616F8AEC5DF0CED720EEE5
:107288000AF0B751D926B851DA22DF500001F06F61
:10729800EF6B010120EE0BF0B751D926B851DA2275
:1072A800DF500001EF250101B06F000E0001F02151
:1072B8000101B16F860E0001606FFB0E616FB0C1F6
:1072C80062F0B1C163F08AEC5DF0CD0E0001A66FEB
:1072D800A76B0101B0510001F06FEF6BEFC0A8F090
:1072E800F0C0A9F0AA6BAB6BDFEC12F00101B46F30
:1072F800B45193E1CD0E0001846F856BB7C186F060
:10730800B8C187F0010E896F886BB20E8A6F010EC3
:107318008B6FC9EC15F00101B46FB45101E07DD752
:10732800B56BB66BEDC00BF0EEC00CF0B5C1EFF06D
:10733800B6C1F0F0050ED8900001EF37F037E82E0F
:10734800FAD7EF510101B7250D6E0001F051010187
:10735800B8210E6EABC10FF0106A89EC53F00B50D8
:107368000C105DE1B5C1EFF0B6C1F0F0050ED89094
:107378000001EF37F037E82EFAD7B7C1F1F0B8C1FE
:10738800F2F0EF51F127F051F2230E0EF125D96EEC
:10739800000EF221DA6EDF50F46FF36BB5C1F5F031
:1073A800B6C1F6F0050ED890F537F637E82EFBD7BC
:1073B800B7C1F7F0B8C1F8F0F551F727F651F8233F
:1073C8000F0EF725D96E000EF821DA6EDF50F96F2F
:1073D800FA6BF351F927F451FA23F9C0ACF1FAC06A
:1073E800ADF10101000EADBFFF0EAE6FAF6FDF0E46
:1073F8000001606FFD0E616FACC162F0ADC163F05A
:10740800AEC164F0AFC165F08AEC5DF0ACC1CDF0FF
:10741800ADC1CEF0AEC1CFF0AFC1D0F01200B54BC8
:10742800B62BB6BF7FD7B65105E10F0EB55D01E3A8
:10743800F4D678D7F2D6D50E0001606FF50E616FDD
:10744800CECF62F0636BCDCF64F0656B4F50070D04
:10745800500EF324D96E010EF420DA6EDF50666FF9
:10746800676B4F50070D510EF324D96E010EF420AF
:10747800DA6EDF50686F696B4F50070D520EF324B8
:10748800D96E010EF420DA6EDF506A6F6B6B4F50C5
:10749800070D510EF324D96E010EF420DA6EDF5079
:1074A800E46FE4C0E5F0E66BE76BE86B040ED89098
:1074B800E537E637E737E837E82EF9D74F50070DB5
:1074C800500EF324D96E010EF420DA6EDF50E96F06
:1074D800E9C0EAF0EB6BEC6BED6B050ED890EA3780
:1074E800EB37EC37ED37E82EF9D7E551EA25EE6FA3
:1074F800E651EB21EF6FE751EC21F06FE851ED21F8
:10750800F16F4F50070D520EF324D96E010EF4207F
:10751800DA6EDF50EE256C6F000EEF216D6F000EF6
:10752800F0216E6F000EF1216F6F8AEC5DF0838E93
:1075380083807DEC56F048C0F3F049C0F4F0F4BF06
:107548000AD0040EF45D07E3000EF325F56FFC0E78
:10755800F421F66F04D0F3C0F5F0F4C0F6F04F5004
:10756800070D530EF324D96E010EF420DA6E74C1A0
:10757800E9F075C1EAF076C1EBF0E86B000EE8259A
:10758800EC6F010EE921ED6F000EEA21EE6F000E9F
:10759800EB21EF6FDE50EC1936E1DE50ED1933E1E7
:1075A800DE50EE1930E1DE50EF192DE101C3FAF09B
:1075B80003C3F9F005C3F8F007C3F7F0F7C00EF0FE
:1075C800F8C00FF0F9C010F0FAC011F0CAEC58F08A
:1075D800010E0001606FF60E616F2AEE34F0DF5085
:1075E800626F636B2AEE35F0DF50646F656B2AEECD
:1075F80036F0DF50666F676B2AEE37F0DF50686F42
:10760800696B8AEC5DF08FB415D04F50200D000ED9
:10761800F3240001A66F020EF420A76F000EA86FD6
:10762800030EA96F010EAB6FAA6BF50EAC6F71EC70
:107638000FF0F26F0001F25109E0800E606FFD0E4D
:10764800616FF2C062F0636B8AEC5DF0940E00012A
:10765800606FFA0E616FF5C062F0F6C063F08AECF5
:107668005DF093EC3DF0966B8390839E0A0E0001CB
:10767800606FFD0E616FCECF62F0636BCDCF64F0AB
:10768800656B8AEF5DF04F50070D520EF324D96EEB
:10769800010EF420DA6EDF500001CD6FCDC0CEF0C0
:1076A800CF6BD06BD16BD0C0D1F0CFC0D0F0CEC0F3
:1076B800CFF0CE6B4F50070D510EF324D96E010E4B
:1076C800F420DA6EDF50D26FD2C0D3F0D46BD56B12
:1076D800D66B0C0ED890D337D437D537D637E82E9B
:1076E800F9D74F50070D500EF324D96E010EF42030
:1076F800DA6EDF50D76FD7C0D8F0D96BDA6BDB6B97
:107708000D0ED890D837D937DA37DB37E82EF9D7C6
:10771800D351D825DC6FD451D921DD6FD551DA2169
:10772800DE6FD651DB21DF6FCE51DC25E16FCF5103
:10773800DD21E26FD051DE21E36FD151DF21E46F0B
:10774800890E606FF80E616F4FC062F0636B4F5027
:10775800070D500EF324D96E010EF420DA6EDF50B7
:10776800646F656B4F50070D510EF324D96E010EEF
:10777800F420DA6EDF50666F676B4F50070D520EBC
:10778800F324D96E010EF420DA6EDF50686F696B4E
:107798004F50070D510EF324D96E010EF420DA6E06
:1077A800DF50CD6FCDC0CEF0CF6BD06BD16B040E58
:1077B800D890CE37CF37D037D137E82EF9D74F50BA
:1077C800070D500EF324D96E010EF420DA6EDF5047
:1077D800D26FD2C0D3F0D46BD56BD66B050ED890D0
:1077E800D337D437D537D637E82EF9D7CE51D32566
:1077F800D76FCF51D421D86FD051D521D96FD1515E
:10780800D621DA6F4F50070D520EF324D96E010EB0
:10781800F420DA6EDF50D7256A6F000ED8216B6F1F
:10782800000ED9216C6F000EDA216D6F8AEC5DF0C5
:107838006F0E0001606FFB0E616FE1C062F0E2C085
:1078480063F0E3C064F0E4C065F0E1C066F0E2C054
:1078580067F0E3C068F0E4C069F08AEC5DF04F506F
:10786800200D000EF3240001A66F020EF420A76F6E
:10787800E1C0A8F0E2C0A9F0E3C0AAF0E4C0ABF010
:10788800DFEC12F0E06FE05111E00F0E606FFB0EBD
:10789800616FE1C062F0E2C063F0E3C064F0E4C08D
:1078A80065F0E0C066F0676B8AEC5DF04F50070D3D
:1078B800530EF324D96E010EF420DA6EE1C0DEFF18
:1078C800E2C0DEFFE3C0DEFFE4C0DEFF0101966B2D
:1078D800839012000001AE6FAA5102E0DDEC44F083
:1078E8000001AD6BA95101E100D1040EAE1903E00E
:1078F800140EAE1909E10101976B886B896B0001C1
:10790800AA6B070EA96F070C3F0EAE1907E14E6A66
:107918000101976B0001A96BAA6B12005F0EAE19EB
:1079280007E10101986B976B0001A96BAA6B120024
:107938003F0EAE6506D05F0EAE6103D0400EAE19A5
:10794800F0E1400EAE1908E1010E0101986F976B46
:107958000001A96BAA6B1200200EAE190CE1010EF2
:107968004E6E0101976B7F0E0001606FFF0E616F15
:107978008AEC5DF0EDD7650EAE1907E14E5005E0D3
:107988000101886B896B010E2BD06E0EAE1903E1D5
:10799800020E0101976F700E0001AE1907E1010197
:1079A800985104E0886B896B030E976F700E000185
:1079B800AE1908E14E5006E083800101886B896B9F
:1079C800040E0ED0720EAE1901E08FD04E5001E1B8
:1079D8008CD083801C0E0101896F2A0E886F050EDA
:1079E800976FB6D7AE51DAEC0BF00001AD6F92D0BD
:1079F800390E606FFC0E616FAEC062F0636B8AEC8B
:107A08005DF083800001AE51B5EC56F00001AD6F1A
:107A18000101976B7FD08380A70E606FF80E616FAE
:107A2800CECF62F0636BCDCF64F0656B4DC066F06E
:107A3800676B8AEC5DF0340E0B6E0A0E0C6E0E6AE4
:107A48000D6A010E106E0F6A3CEC4AF00101FF83CB
:107A58002AEE34F04DC0DFFF496A010E486EA4ECEF
:107A680037F00101FF93080ED1D78390AD6B2B0E31
:107A7800606FF80E616FCECF62F0636BCDCF64F0AC
:107A8800656BAEC066F0676B8AEC5DF043D0080E9C
:107A9800AE1918E18A0E606FF70E616FCECF62F0F3
:107AA800636BCDCF64F0656BAEC066F0676B8AEC34
:107AB8005DF083900001AD6B4D6A0101976B886B97
:107AC800896B28D0090EAE1925E18D0E606FF90E6D
:107AD800616FCECF62F0636BCDCF64F0656BAEC0E3
:107AE80066F0676B8AEC5DF0E4D7010197510001FD
:107AF800AB6FAC6BAC510EE1AB510CE0010A01E18C
:107B080071D7030A01E174D7010A85E0070AADE0DD
:107B1800010ABDE0ADC0A9F00001AA6B12004F50E8
:107B2800070D520EF324D96E010EF420DA6EDF2A07
:107B38004F50070D520EF324D96E010EF420DA6E61
:107B48000F0EDF642FD04F50070D520EF324D96E5D
:107B5800010EF420DA6EDF6A4F50070D510EF32440
:107B6800D96E010EF420DA6EDF2A4F50070D510E40
:107B7800F324D96E010EF420DA6E010EDF6412D000
:107B88004F50070D510EF324D96E010EF420DA6E12
:107B9800DF6A4F50070D500EF324D96E010EF42002
:107BA800DA6EDF2A4F50070D520EF324D96E010EFC
:107BB800F420DA6EDF500001CD6FCDC0CEF0CF6B70
:107BC800D06BD16BD0C0D1F0CFC0D0F0CEC0CFF049
:107BD800CE6B4F50070D510EF324D96E010EF420D1
:107BE800DA6EDF50D26FD2C0D3F0D46BD56BD66BC0
:107BF8000C0ED890D337D437D537D637E82EF9D7E7
:107C08004F50070D500EF324D96E010EF420DA6E92
:107C1800DF50D76FD7C0D8F0D96BDA6BDB6B0D0E9E
:107C2800D890D837D937DA37DB37E82EF9D7D35198
:107C3800D825DC6FD451D921DD6FD551DA21DE6F1B
:107C4800D651DB21DF6FCE51DC25E06FCF51DD212E
:107C5800E16FD051DE21E26FD151DF21E36F4F5048
:107C6800070D530EF324D96E010EF420DA6EE0C02E
:107C7800DEFFE1C0DEFFE2C0DEFFE3C0DEFFDE0EB6
:107C8800606FF90E616F4FC062F0636B4F50070D64
:107C9800500EF324D96E010EF420DA6EDF50646FB3
:107CA800656B4F50070D510EF324D96E010EF42069
:107CB800DA6EDF50666F676B4F50070D520EF32474
:107CC800D96E010EF420DA6EDF50686F696B8AECAA
:107CD8005DF04F50200D000EF3240001A66F020E38
:107CE800F420A76F4F50070D530EF324D96E010EE1
:107CF800F420DA6EDECFA8F0DECFA9F0DECFAAF04E
:107D0800DECFABF0DFEC12F04A6E4A5019E00F0EEE
:107D1800606FFB0E616F4F50070D530EF324D96E41
:107D2800010EF420DA6EDECF62F0DECF63F0DECF34
:107D380064F0DECF65F04AC066F0676B8AEC5DF0F0
:107D48000101966B1200C76B0101A16B030EF16173
:107D580005D09650F119F00BF11905D0F1C193FF38
:107D68009650F00B0A09966ECD6ACE6ADFD0C86BC2
:107D7800340E156E0A0E166E320E176EF40E186E4D
:107D880009EC52F015C0C5F016C0C6F0C5C0D9FF41
:107D9800C6C0DAFF3B0EDE1801E0C3D0C7D0C85119
:107DA80009E1C5C00FF0C6C010F0EDEC56F00001B7
:107DB800C76FA9D0C80511E10101FE510001C7191B
:107DC80003E07F0EC71909E1C5C00FF0C6C010F067
:107DD800EDEC56F001019F6F96D0020EC81911E123
:107DE8000101FE510001C71903E07F0EC71909E11F
:107DF800C5C00FF0C6C010F0EDEC56F001019E6F43
:107E080082D0020EC8651FD0080EC8611CD00101BF
:107E1800FE510001C71903E07F0EC71914E1F30EE4
:107E2800C36F010EC46FC5C00FF0C6C010F0EDECF3
:107E380056F00001C06FC851C325C16F000EC421A0
:107E4800C26FFD0E40D0070EC8651FD01B0EC8615B
:107E58001CD00101FE510001C71903E07F0EC719AC
:107E680014E1A00EC36F020EC46FC5C00FF0C6C0E8
:107E780010F0EDEC56F00001C06FC851C325C16F7A
:107E8800000EC421C26FF80E1ED0280EC86123D080
:107E98000101FE510001C71903E07F0EC7191BE15C
:107EA800C60EC36F020EC46FC5C00FF0C6C010F077
:107EB800EDEC56F00001C06FC851C325C16F000E2C
:107EC800C421C26FE50EC125D96EFF0EC221DA6E3C
:107ED800C0C0DFFF18D0280EC81915E10101FE51F6
:107EE8000001C71903E07F0EC7190DE1A10E0B6E43
:107EF800010E0C6EC5C00DF0C6C00EF0106A080E5B
:107F08000F6E4BEC58F00001C82B156A166A320E3A
:107F1800176EF40E186E09EC52F015C0C5F016C0B5
:107F2800C6F00001C551C61101E039D7340E000171
:107F3800AC6F0A0EAD6FAF6B910EAE6F000EB06FE7
:107F4800020EB16F57EC52F0AC51AD1101E00FD7F2
:107F58007A0E606FFA0E616FA10E626F010E636F89
:107F68008AEF5DF00001F46B270E606FF60E616F0B
:107F78004F50070D500EF324D96E010EF420DA6E1F
:107F8800DF50626F636B4F50070D510EF324D96EAB
:107F9800010EF420DA6EDF50646F656B4F50070DE9
:107FA800520EF324D96E010EF420DA6EDF50666F9C
:107FB800676B4F50070D510EF324D96E010EF42054
:107FC800DA6EDF50E46FE4C0E5F0E66BE76BE86B70
:107FD800040ED890E537E637E737E837E82EF9D7C3
:107FE8004F50070D500EF324D96E010EF420DA6EAF
:107FF800DF50E96FE9C0EAF0EB6BEC6BED6B050E57
:10800800D890EA37EB37EC37ED37E82EF9D7E5515A
:10801800EA25EE6FE651EB21EF6FE751EC21F06FA7
:10802800E851ED21F16F4F50070D520EF324D96E30
:10803800010EF420DA6EDF50EE25686F000EEF2196
:10804800696F000EF0216A6F000EF1216B6F8AECE8
:108058005DF08380838E8DD07DEC56F048C0F2F0C1
:1080680049C0F3F0F3BF06D0040EF35D03E3010E3D
:10807800F46F03D0F7C0F5F0F66B8FB414D04F50FF
:10808800200D000EF324A66F020EF420A76F000E39
:10809800A86F030EA96F010EAB6FAA6BF50EAC6F3C
:1080A80071EC0FF0F76FF75109E0800E606FFD0E6D
:1080B800616FF7C062F0636B8AEC5DF04F50070D9B
:1080C800530EF324D96E010EF420DA6E74C1E9F070
:1080D80075C1EAF076C1EBF00001E86B000EE82507
:1080E800EC6F010EE921ED6F000EEA21EE6F000E34
:1080F800EB21EF6FDE50EC192EE1DE50ED192BE18C
:10810800DE50EE1928E1DE50EF1925E101C3FBF03E
:1081180003C3FAF005C3F9F007C3F8F0F8C00EF08E
:10812800F9C00FF0FAC010F0FBC011F0CAEC58F01B
:10813800010E0001606FF60E616F00C362F0636BA1
:1081480001C364F0656B02C366F0676B03C368F034
:10815800696B8AEC5DF0720E0001606FF90E616F59
:10816800F5C062F0F6C063F08AEC5DF093EC3DF088
:10817800966B0001F45101E16FD7839E8390120042
:1081880046C00CF047C00DF0D0EC53F000016C6F06
:108198006C5101E000D120EE04F04650D92647503A
:1081A800DA22DFAAF8D046C0D9FF47C0DAFFDECF0F
:1081B80039F0DDCF3AF020EE1AF04650D926475074
:1081C800DA22DECF3BF0DECF3CF0DECF3DF0DECF73
:1081D8003EF0A5EC52F000016C6F6C5101E0DBD071
:1081E80020EE1EF04650D9264750DA22DECF71F035
:1081F800DDCF72F020EE0BF07151D9267251DA22E0
:10820800000EDB8A20EE0AF04650D9264750DA22C3
:1082180010EE1CF07151E1267251E222DFCFE7FF28
:1082280020EE1DF07151D9267251DA2210EE0AF0B3
:108238004650E1264750E222E6CF68F0E5CF69F0E4
:1082480069C068F0696B6851DF6E20EE1EF07151ED
:10825800D9267251DA2210EE0AF04650E12647502C
:10826800E222E6CF68F0E6CF69F0E6CF6AF0E6CF23
:108278006BF0110E05D0D8906B336A3369336833CD
:10828800E82EF9D76851DF6E20EE1FF07151D9261C
:108298007251DA2210EE0AF04650E1264750E222E7
:1082A800E6CF68F0E6CF69F0E6CF6AF0E6CF6BF08C
:1082B800190E05D0D8906B336A3369336833E82ECA
:1082C800F9D76851DF6E71C00BF072C00CF020EE68
:1082D8000EF04650D9264750DA22DECF0DF0DECF19
:1082E8000EF0DECF0FF0DECF10F019EC5AF00001DF
:1082F8006D6B6E6B210E6F6F460E706F20EE16F071
:108308007151D9267251DA22DF6A20EE17F07151C5
:10831800D9267251DA226EC0DFFF20EE18F07151B3
:10832800D9267251DA226FC0DFFF20EE19F07151A1
:10833800D9267251DA2270C0DFFF20EE12F0715197
:10834800D9267251DA22DF6A20EE13F07151D9264C
:108358007251DA22DF6A20EE04F04650D9264750DF
:10836800DA22DF0EDF1646C0D9FF47C0DAFF10EE6B
:1083780004F0DE50E126DD50E222010EE76E46C031
:10838800D9FF47C0DAFFDECF43F0DDCF44F091ECF0
:1083980030F000016C6F6C51120020EE04F0445074
:1083A800D9264550DA22DF6A20EE2AF04450D92631
:1083B8004550DA22DE68DE68DE68DD6844C039F0E0
:1083C80045C03AF046C03BF047C03CF048C03DF0DD
:1083D80049C03EF0A5EC52F0000901E0030C22EE82
:1083E8002DF04450D9264550DA22DF500001616F44
:1083F800606B22EE2CF04450D9264550DA22DF502B
:108408006013550E601903E1AA0E611901E0020C10
:1084180020EE65F04450D9264550DA22DF50616FCE
:10842800606B20EE66F04450D9264550DA22DF50C2
:10843800626F62C063F0646B656B666B64C066F004
:1084480063C065F0646B636B20EE67F04450D92617
:108458004550DA22DF50676F67C068F0696B6A6B56
:108468006B6B68C06BF06A6B696B686B6351681102
:108478006C6F645169116D6F65516A116E6F665149
:108488006B116F6F60516C11706F61516D11716F6D
:10849800000E6E11726F000E6F11736F20EE64F094
:1084A8004450D9264550DA22DF507011746F71514B
:1084B800756F7251766F7351776F7451786F75510C
:1084C800796F76517A6F7B6B460E781908E1410E09
:1084D800791905E1540E7A197B1101E1000C20EE9F
:1084E80081F04450D9264550DA22DF50616F606B25
:1084F80020EE82F04450D9264550DA22DF50626FD0
:1085080062C063F0646B656B666B64C066F063C0E1
:1085180065F0646B636B20EE83F04450D9264550B8
:10852800DA22DF50676F67C068F0696B6A6B6B6B44
:1085380068C06BF06A6B696B686B635168116C6F2C
:10854800645169116D6F65516A116E6F66516B11D7
:108558006F6F60516C11706F61516D11716F000E0A
:108568006E11726F000E6F11736F20EE80F0445021
:10857800D9264550DA22DF507011746F7151756F2A
:108588007251766F7351776F7451786F7551796F37
:1085980076517A6F7B6B460E781908E1410E79198E
:1085A80005E1540E7A197B1101E1000C010C260E2D
:1085B8000001606FF70E616FCECF62F0636BCDCFB5
:1085C80064F0656B4FC066F0676B8AEC5DF0010183
:1085D800FF83340E0B6E0A0E0C6E0E6A0D6A010EC6
:1085E800106E0F6A3CEC4AF02AEE34F04FC0DFFF01
:1085F800FF0EE8CF35FA4F50140D130EF324D96E41
:10860800010EF420DA6EDFA403D0010EE8CF38FAA9
:108618004F50140D130EF324D96E010EF420DA6EA8
:10862800DFA003D0020EE8CF3AFA4F50140D130E14
:10863800F324D96E010EF420DA6EDFA203D0020E05
:10864800E8CF3AFA4F50140D130EF324D96E010EE9
:10865800F420DA6EDFA603D0800EE8CF39FA8FA4B3
:1086680003D0080EE8CF3AFA00018B6B8C6BCB0E67
:10867800606FF70E616FCECF62F0636BCDCF64F0A1
:10868800656B8BC066F08CC067F0360E8B25D96E93
:108698000A0E8C21DA6EDF50686F696B8AEC5DF028
:1086A8006C0E00018B25D96E010E8C21DA6EDF1C51
:1086B8008A6F360E8B25D96E0A0E8C21DA6E360E2D
:1086C8008B25E16E0A0E8C21E26EE7508A15DF6E6B
:1086D800630E606FFF0E616F360E8B25D96E0A0E22
:1086E8008C21DA6EDF50626F636B8AEC5DF00001FB
:1086F8008B4B8C2B8CBFBBD78C5103E1070E8B5D4A
:10870800B6E34F50140D130EF324D96E010EF42066
:10871800DA6EDF504D6E4F50140D010EF324D96EF2
:10872800010EF420DA6EDF504A6E4AC03FFA4F500D
:10873800140D020EF324D96E010EF420DA6EDF5008
:108748004A6E4AC040FA4F50140D030EF324D96EF6
:10875800010EF420DA6EDF504A6E4AC041FA4F50DB
:10876800140D040EF324D96E010EF420DA6EDF50D6
:108778004A6E4AC042FA4F50140D050EF324D96EC2
:10878800010EF420DA6EDF504A6E4AC043FA4F50A9
:10879800140D060EF324D96E010EF420DA6EDF50A4
:1087A8004A6E4AC044FA496A140E486EA4EC37F07F
:1087B8000101FF93839012004F50140D070EF3240C
:1087C800D96E010EF420DA6EDECFE0F0DECFE1F0F4
:1087D800DECFE2F0DECFE3F0A80E0001606FF50E09
:1087E800616FCECF62F0636BCDCF64F0656BE0C094
:1087F80066F0E1C067F0E2C068F0E3C069F0E0C08D
:108808006AF0E1C06BF0E2C06CF0E3C06DF08AEC96
:108818005DF04F50140D070EF324D96E010EF420AD
:10882800DA6E4F50140D0B0EF324E16E010EF42096
:10883800E26EDE50E65CDE50E658DE50E658DE506A
:10884800E6581CE2E60E0001606FFC0E616F8AECD0
:108858005DF0010E4D6E4F50140D130EF324D96EBA
:10886800010EF420DA6E4F50140D130EF324E16E4E
:10887800010EF420E26EE7500409DF6E4F50140D2C
:108888000F0EF324D96E010EF420DA6EDECFCFF08E
:10889800DECFD0F0DECFD1F0DECFD2F04F50140DC6
:1088A800070EF324D96E010EF420DA6EDECFD3F072
:1088B800DECFD4F0DECFD5F0DECFD6F00001CF5139
:1088C800D325D76FD051D421D86FD151D521D96FA5
:1088D800D251D621DA6F4F50140D0B0EF324D96EF6
:1088E800010EF420DA6ED751DE5CD851DE58D9512A
:1088F800DE58DA51DE581BE2D40E606FFC0E616F51
:108908008AEC5DF0010E4D6E4F50140D130EF324DA
:10891800D96E010EF420DA6E4F50140D130EF324A5
:10892800E16E010EF420E26EE7500409DF6E4D6A35
:108938004F50200D000EF3240001A66F020EF42004
:10894800A76FE0C0A8F0E1C0A9F0E2C0AAF0E3C0B8
:10895800ABF0DFEC12F0DF6FDF5126E00F0E606F37
:10896800FB0E616FE0C062F0E1C063F0E2C064F04A
:10897800E3C065F0DFC066F0676B8AEC5DF0010E5E
:108988004D6E4F50140D130EF324D96E010EF420C2
:10899800DA6E4F50140D130EF324E16E010EF4201D
:1089A800E26EE7500409DF6E4DC0CDF00001CE6BDA
:1089B80012004F6A4F6A030E4F6401D0E9D04F503E
:1089C80003E1486A496A03D0496A010E486E4F506C
:1089D800140D130EF324D96E010EF420DA6EDF6A3B
:1089E8004F50140D000EF324D96E010EF420DA6EE8
:1089F800DF6A4F50140D070EF324D96E010EF420D0
:108A0800DA6EDE6ADE6ADE6ADD6A0D0E4802F3CFD0
:108A180086F0F4CF87F04902F35000018727D10E82
:108A28008625D96E020E8721DA6EDF50886F88C0DE
:108A380089F08A6B8B6B8C6B8BC08CF08AC08BF047
:108A480089C08AF0896B0D0E4802F3CF8DF0F4CF00
:108A58008EF04902F3508E27D00E8D25D96E020E66
:108A68008E21DA6EDF508F6F8FC090F0916B926B12
:108A7800936B91C093F090C092F0916B906B0D0E38
:108A88004802F3CF94F0F4CF95F04902F3509527BC
:108A9800CF0E9425D96E020E9521DA6EDF50966FAF
:108AA80096C097F0986B996B9A6B97C09AF0996BF0
:108AB800986B976B0D0E4802F3CF9BF0F4CF9CF0A8
:108AC8004902F3509C27CE0E9B25D96E020E9C219D
:108AD800DA6EDF5097259D6F000E98219E6F000E6D
:108AE80099219F6F000E9A21A06F90519D25A16F2B
:108AF80091519E21A26F92519F21A36F9351A02162
:108B0800A46F8951A125A56F8A51A221A66F8B5107
:108B1800A321A76F8C51A421A86F4F50140D0B0EE1
:108B2800F324D96E010EF420DA6EA5C0DEFFA6C0CC
:108B3800DEFFA7C0DEFFA8C0DEFFAB0E606FF70E3A
:108B4800616F4FC062F0636B4F50140D0B0EF3242E
:108B5800D96E010EF420DA6EDECF64F0DECF65F058
:108B6800DECF66F0DECF67F04F50140D0B0EF32406
:108B7800D96E010EF420DA6EDECF68F0DECF69F030
:108B8800DECF6AF0DECF6BF08AEC5DF04F2A13D7A8
:108B98000101986B4E6A976B886B896B020E4D6E5C
:108BA8008390020C8EA605D04A0E0001866FFC0E3B
:108BB80004D0B20E0001866FFF0E876F8EAA04D014
:108BC8004A0E886FFC0E03D0AD0E886FFF0E896FBA
:108BD8008EA804D04A0E8A6FFC0E03D0B70E8A6F97
:108BE800FF0E8B6F8EAE04D04A0E8C6FFC0E03D036
:108BF800BC0E8C6FFF0E8D6F8EAC04D04A0E8E6F3C
:108C0800FC0E03D0A80E8E6FFF0E8F6F8EA404D0BB
:108C18004A0E906FFC0E03D0C60E906FFF0E916F38
:108C28008EA204D04A0E926FFC0E03D0CB0E926F28
:108C3800FF0E936F8EA004D04A0E946FFC0E03D0E3
:108C4800C10E946FFF0E956F90AE04D04A0E966FCA
:108C5800FC0E03D0F90E966FFF0E976F90AC04D000
:108C68004A0E986FFC0E03D0F60E986FFF0E996FA0
:108C780090AA04D04A0E9A6FFC0E03D0F30E9A6F96
:108C8800FF0E9B6F90A804D04A0E9C6FFC0E03D079
:108C9800F00E9C6FFF0E9D6F90A604D04A0E9E6F3B
:108CA800FC0E03D0ED0E9E6FFF0E9F6F90A404D0B4
:108CB8004A0EA06FFC0E03D0EA0EA06FFF0EA16F44
:108CC80090A204D04A0EA26FFC0E03D0E70EA26F4A
:108CD800FF0EA36F90A004D04A0EA46FFC0E03D021
:108CE800E40EA46FFF0EA56F340E606FF40E616F73
:108CF800901C626F636B8ECF64F0656BA4C066F0E6
:108D0800A5C067F0A2C068F0A3C069F0A0C06AF06F
:108D1800A1C06BF09EC06CF09FC06DF09CC06EF05F
:108D28009DC06FF09AC070F09BC071F098C072F04F
:108D380099C073F096C074F097C075F094C076F03F
:108D480095C077F092C078F093C079F090C07AF02F
:108D580091C07BF08EC07CF08FC07DF08CC07EF01F
:108D68008DC07FF08AC080F08BC081F088C082F00F
:108D780089C083F086C084F087C085F08AEF5DF0F3
:108D8800BD0E0001606FF60E616F4F50070D500E5B
:108D9800F324D96E010EF420DA6EDF50626F636B34
:108DA8004F50070D510EF324D96E010EF420DA6EE0
:108DB800DF50646F656B4F50070D520EF324D96E68
:108DC800010EF420DA6EDF50666F676B4F50070DA7
:108DD800510EF324D96E010EF420DA6EDF50AC6F19
:108DE800ACC0ADF0AE6BAF6BB06B040ED890AD37C6
:108DF800AE37AF37B037E82EF9D74F50070D500EC2
:108E0800F324D96E010EF420DA6EDF50B16FB1C0D1
:108E1800B2F0B36BB46BB56B050ED890B237B337FD
:108E2800B437B537E82EF9D7AD51B225B66FAE5184
:108E3800B321B76FAF51B421B86FB051B521B96F35
:108E48004F50070D520EF324D96E010EF420DA6E3E
:108E5800DF50B625686F000EB721696F000EB82184
:108E68006A6F000EB9216B6F8AEC5DF0838E838088
:108E78000001BC6BBD6BBE6BBF6B4F50200D000E6D
:108E8800F324846F020EF420856F340E866F0A0E69
:108E9800876F010E896F886BC10E8A6F8B6BC9EC67
:108EA80015F0C06FE30E606FF80E616FC0C062F01E
:108EB800636BC1C064F0C2C065F08AEC5DF001016B
:108EC800FF93C1C048F0C2C049F0A4EC37F048C0D5
:108ED800BAF049C0BBF00001BA51BC27BB51BD2351
:108EE800000EBE23BF23C20E606FFC0E616FBCC0B4
:108EF80062F0BDC063F0BEC064F0BFC065F08AEC2C
:108F08005DF00101966B839E839012001B6E1B50CF
:108F180001E0010C54A202D054501200000EB1EC32
:108F28005CF00A0E266E03D0A6EC5DF026062650ED
:108F3800FBE1236A000E146A156A166A176A4AEC7E
:108F48005BF0E80601E097D0AA0E146E010E156ECC
:108F5800166A176A080E4AEC5BF0E80651E1266AC1
:108F680026501C0FD96EDA6AA6EC5DF0DF6E262A51
:108F7800030E2664F5D71E047EE1AA0E1F187BE1B6
:108F8800030E256EE80E246E15D0146A156A166A4B
:108F9800400E176EA90E4AEC5BF000090EE0150EA4
:108FA8001A6EC60EE82EFED71A2EFCD700D024065D
:108FB800D8A0250624502510E8E1245025105BE0B0
:108FC800146A156A166A176A3A0E4AEC5BF00009C9
:108FD80052E1266A26501C0FD96EDA6AA6EC5DF0BB
:108FE800DF6E262A030E2664F5D71CBC03D0216A3F
:108FF800040E02D0216A0C0E206E20C023F03BD054
:10900800146A156A166A176AA90E4AEC5BF01A6E9A
:10901800020E1A6003D0236EA90E02D0010E236E31
:10902800226E030E256EE80E246E14D0146A156A9B
:10903800166A176A22504AEC5BF000090EE0150E1A
:109048001A6EC60EE82EFED71A2EFCD700D02406BC
:10905800D8A0250624502510E9E1245025100AE05F
:10906800146A020E156E166A176A100E4AEC5BF047
:10907800000901E0236A23C050F0B9EC5DF02350E9
:1090880001E14AD7549048D7C1C0F6FFC2C0F7FFE4
:10909800000EF86E0E0EF76403D00800F55005D0E8
:1090A800F6CFE9FFF7CFEAFFEF502F0A13E0C1C070
:1090B800F6FFC2C0F7FF000EF86E0E0EF76403D07D
:1090C8000800F55005D0F6CFE9FFF7CFEAFFEF50DB
:1090D8005C0A03E10001C14BC22B000120EE06F03F
:1090E800BF51D926C051DA22DE6ADE6ADE6ADD6A3D
:1090F800C1C0F6FFC2C0F7FF000EF86E0E0EF7648F
:1091080003D00800F55005D0F6CFE9FFF7CFEAFF06
:10911800EF504A6E200E4A6013D0BFC084F0C0C022
:1091280085F00001876B866B51EC36F0C66F20EE38
:1091380012F0BF51D926C051DA22DE6ADD6A5DD04D
:10914800BFC013F0C0C014F0C10E156EA2EC33F00E
:109158000001C66FC65151E1BFC0B9F0C0C0BAF036
:109168002FEC50F0C66F20EE14F0BF51D926C05135
:10917800DA2210EE0BF0DE50E126DD50E222E75055
:10918800C56FC65108E0040EC61937E1C5B535D01C
:10919800050EC66F32D0C5B530D020EE12F0BF51E3
:1091A800D926C051DA22DECFC3F0DDCFC4F020EEDD
:1091B8000BF0C351D926C451DA22DFA8E9D7BFC0C2
:1091C800D9FFC0C0DAFFDECF0BF0DDCF0CF0C3C093
:1091D8000DF0C4C00EF062EC51F0000120EE06F074
:1091E800BF51D926C051DA220BC0DEFF0CC0DEFF0A
:1091F8000DC0DEFF0EC0DEFFA3D7C6511200326AD3
:1092080020EE04F02450D9262550DA22DF5001E15F
:1092180097D020EE2AF02450D9262550DA22DECF26
:1092280035F0DECF36F0DECF37F0DECF38F02E0E59
:1092380024241A6E000E25201B6E35C01CF036C083
:109248001DF037C01EF038C01FF0216A010E206ED5
:1092580020EE01F02450D9262550DA22DF507BEC8D
:109268004EF0000903E0010E326E6AD020EE04F0E1
:109278002450D9262550DA22DF6A20EE16F0245031
:10928800D9262550DA2210EE1EF02450E12625506A
:10929800E222E6CF2AF0E6CF2BF0E6CF2CF0E6CF9D
:1092A8002DF02A50355C2E6E2B5036582F6E2C50D0
:1092B8003758306E2D503858316EDE502E5CDE50E7
:1092C8002F58DE503058DE5031583AE220EE03F085
:1092D8002450D9262550DA22DF50336E346A3450B0
:1092E80003E1020E335C2CE320EE16F02450D9265D
:1092F8002550DA22DE503526DE503622DE5037225F
:10930800DD5038222E0E24241A6E000E25201B6EE6
:1093180035C01CF036C01DF037C01EF038C01FF035
:10932800216A010E206E20EE01F02450D926255026
:10933800DA22DF507BEC4EF03306D8A03406CFD7C4
:10934800325012002F6C696664617461302E626954
:109358006E20002F6C696664617461312E62696EDB
:1093680020002F6C696664617461322E62696E2018
:10937800002F6C696664617461332E62696E200027
:109388002F6C696664617461342E62696E20002FE7
:109398006C696664617461352E62696E20002F6C99
:1093A800696664617461362E62696E20002F6C698B
:1093B8006664617461372E62696E20002F6C69667D
:1093C80064617461382E62696E20002F6C6966646E
:1093D800617461392E62696E20002F6C6966646160
:1093E8007461612E62696E20002F6C696664617415
:1093F80061622E62696E20002F6C69666461746117
:10940800632E62696E20002F6C6966646174616402
:109418002E62696E20002F6C696664617461652E26
:1094280062696E20002F6C696664617461662E62E1
:10943800696E20000000000000000000000000002D
:109448000000000000000000000000000000000014
:109458000000000000000000000000000000000004
:1094680000000000000000000000000000000000F4
:109478000BC015F00CC016F00F50101001E11200CF
:1094880015C0D9FF16C0DAFF0DC0DFFF0F50152435
:10949800116E10501620126EFF0E1124D96EFF0E99
:1094A8001220DA6E0DC0DFFF105004E1030E0F5CCE
:1094B80001E2120020EE01F01550D9261650DA22EA
:1094C8000DC0DFFF20EE02F01550D9261650DA2223
:1094D8000DC0DFFF0F501524116E10501620126EAC
:1094E800FE0E1124D96EFF0E1220DA6E0DC0DFFFBA
:1094F8000F501524116E10501620126EFD0E1124F7
:10950800D96EFF0E1220DA6E0DC0DFFF105004E195
:10951800070E0F5C01E2120020EE03F01550D92669
:109528001650DA220DC0DFFF0F501524116E1050AF
:109538001620126EFC0E1124D96EFF0E1220DA6E60
:109548000DC0DFFF105004E1090E0F5C01E21200AC
:1095580015C011F016C012F0111E121E114A122A5F
:10956800030E1114136E146A135015261450162284
:1095780013500F5E1450105AFC0E0F160BD015C066
:10958800D9FF16C0DAFF0DC0DFFF0F06D8A01006FE
:10959800154A162A0F501010F2E1120000019451DA
:1095A8009311921103E1020E915D0FE320EE12F088
:1095B8008F51D9269051DA22DE50915DDE509259B2
:1095C800DE509359DE50945902E3020E2CD0996B69
:1095D8006AD08FC044F090C045F091C046F092C068
:1095E80047F093C048F094C049F0A2EC1FF044C083
:1095F8009AF045C09BF046C09CF047C09DF0000122
:109608009A519B119C119D115DE09A059B119C112B
:109618009D11DBE09A2909E19B2907E19C2905E1D5
:109628009D2903E1010E996F4DD08FC060F090C065
:1096380061F091C062F092C063F093C064F094C08E
:1096480065F0666B676B686B696B45EC1DF0996F2D
:10965800995138E120EE0EF08F51D9269051DA2237
:10966800DE2806E1DE2804E1DE2802E1DE2813E038
:1096780020EE0EF08F51D9269051DA22DE2A000E04
:10968800DE22DE22DE2220EE05F08F51D92690510F
:10969800DA22000EDB809AC091F09BC092F09CC049
:1096A80093F09DC094F020EE12F08F51D92690517E
:1096B800DA22DE50915DDE509259DE509359DE5029
:1096C800945987E399511200136814680B50D96EA6
:1096D800DA6ADE50DE1001E181D00B50D96EDA6A09
:1096E800DECF17F0DDCF18F002D0174A182A17C0BE
:1096F800F6FF18C0F7FF000EF86E0E0EF76403D0E1
:109708000800F55005D0F6CFE9FFF7CFEAFFEF5094
:109718000D6E200E0D6413D017C0F6FF18C0F7FFAA
:10972800000EF86E0E0EF76403D00800F55005D051
:10973800F6CFE9FFF7CFEAFFEF503A0AD6E117C0B4
:10974800F6FF18C0F7FF000EF86E0E0EF76403D090
:109758000800F55005D0F6CFE9FFF7CFEAFFEF5044
:109768003A0A41E10B50D96EDA6ADECF11F0DDCF4B
:1097780012F011C0F6FF12C0F7FF000EF86E0E0EC1
:10978800F76403D00800F55005D0F6CFE9FFF7CF0E
:10979800EAFFEF500D6ED00E0D24156E166AFF0EFF
:1097A8001622114A122A165019E10A0E155C16E201
:1097B8001750111813E11850121810E1155016100F
:1097C8000DE115C013F016C014F0174A182A0B50F3
:1097D800D96EDA6A17C0DEFF18C0DDFF13C00BF0C0
:1097E80014C00CF01200136A146AF8D7FEC186F090
:1097F80077D0FCEC5CF00001866F0101FE5100019E
:1098080086197CE0290E496E960E486E7F0EE82E6A
:10981800FED7482EFCD7492EFAD700F06FD06DEC52
:1098280059F00001876F875169E087B1512A87B3E2
:1098380051060F0E5116000E0B6EC00E45EC59F076
:109848009CEC5CF0000E0B6EC00E45EC59F05150CC
:109858000F0D340EF3240F6E0C0EF420106EE2EC94
:1098680054F0110E496E3C0E486ECB0EE82EFED712
:10987800482EFCD7492EFAD700F0000187A53ED024
:109888000C6A0B6A51C00DF011EC5BF0AF0E0001D1
:10989800606FFC0E616F51C062F0636B8AEC5DF023
:1098A80051C086F0000E0B6E800E45EC59F09CEC12
:1098B8005CF0000E0B6E800E45EC59F051500F0D08
:1098C800340EF3240F6E0C0EF420106EE2EC54F0FC
:1098D800000E0B6EC00E45EC59F09CEC5CF00ED0FF
:1098E80001019C51486E496A495008E14850010AF3
:1098F80080E0030A01E17DD7010A91E00001865169
:109908001200020E0D5E000E0E5A0F5A105A20EE6B
:1099180012F00B50D9260C50DA22FE0EDE24116EFE
:10992800FF0EDE20126EFF0EDE20136EFF0EDE200D
:10993800146E11500D5C12500E5813500F581450DD
:10994800105805E30B6A0C6A0D6A0E6A120020EEC5
:1099580026F00B50D9260C50DA22DECF11F0DECFDC
:1099680012F0DECF13F0DECF14F020EE02F00B5031
:10997800D9260C50DA22DF50156E15C016F0176A7A
:10998800186A196A16500D02F3CF1AF0F4CF1BF0BB
:109998001C6A1D6A0E02F3501B26F4501C22000E8E
:1099A8001D2217500D02F3501B26F4501C22000EE6
:1099B8001D2216500F02F3501C26F4501D2217507A
:1099C8000E02F3501C26F4501D2218500D02F350BD
:1099D8001C26F4501D2210501602F3501D26175055
:1099E8000F02F3501D2618500E02F3501D26195071
:1099F8000D02F3501D2611501A240B6E12501B2015
:109A08000C6E13501C200D6E14501D200E6E12008B
:109A18001F6A206A186A196A01D0122A010E1E6E7E
:109A28001250D96EDA6A200EDE1813E0F70E146EA3
:109A380015681250D96EDA6ADF50166E176A14501C
:109A4800162615501722175003E1050E165C01E380
:109A58001E6A1EC01AF01B6A1A501B1006E0DDD7DA
:109A6800196A010E186E122A25D01250D96EDA6AB8
:109A7800DF50146E156A15501DE114502B0AF3E0DF
:109A8800060AEEE017D00A0E1F02F3CF14F0F4CF47
:109A980015F02002F35015261250D96EDA6ADF50FD
:109AA800145E000E155A300E14241F6E000E152079
:109AB800206ED9D7D00E146E15681250D96EDA6A96
:109AC800DF50166E176A14501626155017221750B5
:109AD80005E10A0E165C02E2010E01D0000E1C6EB2
:109AE8001D6A1C501D10CFE1185019100DE11FC040
:109AF80014F020C015F0141E151E144A152A14C09F
:109B080012F015C013F012001FC012F020C013F09D
:109B180012008380838E000E0B6E030E0C6E0E6A8D
:109B2800F60E0D6E010E106E0F6A3CEC4AF0650ED3
:109B38000001606FFE0E616F8AEC5DF00001E96B59
:109B4800EA6B2E0E75EC5DF08FB415D04F50200DDA
:109B5800000EF3240001A66F020EF420A76F000E7A
:109B6800A86F030EA96F010EAB6FAA6BE60EAC6F60
:109B780071EC0FF0E86F0001E85109E05C0E606FCE
:109B8800FF0E616FE8C062F0636B8AEF5DF00DEC69
:109B98005DF00B500C1027E0EB0E0B6E0C6A17EC07
:109BA80054F00001E56FEB51100B0B6E000E0C6EBC
:109BB800E5517AEC2BF00BC0ECF00CC0EDF0040E84
:109BC8000001EC19ED1102E19AEC5AF0020E0001C5
:109BD800EC19ED1102E1F0EC57F00001EC05ED1184
:109BE80002E147EC3BF00001E94BEA2BEA5103E1C3
:109BF800C80EE95DA6E3140E606FFF0E616F8AEC74
:109C08005DF0839E839012000F015969116B196BE7
:109C1800216B8C948C928C90889A110E106E3C0E4D
:109C28000F6ECB0EE82EFED70F2EFCD7102EFAD7CC
:109C380000F0110E106E3C0E0F6ECB0EE82EFED704
:109C48000F2EFCD7102EFAD700F0020E106EA00EC1
:109C58000F6E920EE82EFED70F2EFCD7102EFAD7D5
:109C680000D0000E0B6E300E45EC59F02A0E0F6E28
:109C78008E0EE82EFED70F2EFCD7000E0B6E300E80
:109C880045EC59F0000E0B6E300E45EC59F0000E05
:109C98000B6E390E45EC59F0000E0B6E140E45ECA8
:109CA80059F0000E0B6E560E45EC59F0000E0B6E77
:109CB8006D0E45EC59F0000E0B6E700E45EC59F028
:109CC800000E0B6E0C0E45EC59F0000E0B6E060ED6
:109CD80045EC59F0000E0B6E010E45EC59F0D00E14
:109CE8000F6ECA0EE82EFED70F2EFCD71200236E79
:109CF8002350D8A4040C2050211001E1040C54B0C6
:109D0800030C54B4020C50B608D0090ED8901C3677
:109D18001D361E361F36E82EF9D7200421101AE109
:109D28001CC014F01DC015F01EC016F01FC017F09F
:109D3800180E4AEC5BF0000945E11AC00DF01BC093
:109D48000EF0FE0E0F6E76EC58F000093BE0206A2C
:109D5800216A38D050C022F0060E221609E020C031
:109D680014F021C015F0166A176A970E4AEC5BF0DA
:109D78001CC014F01DC015F01EC016F01FC017F04F
:109D8800190E4AEC5BF000091DE11AC00DF01BC06A
:109D98000EF0FC0E0F6E76EC58F0000908E0020E8B
:109DA8001B262006D8A0210620502110EEE10D6ABE
:109DB8000E6AFD0E0F6E76EC58F0000903E1216A79
:109DC800010E206EB9EC5DF020502110D8A4010CD2
:109DD800000C818E819C4C0EF66E930EF76E000E71
:109DE800F86E0CEE34F011EE2CF00900F5CFEEFF12
:109DF800E550E150FAE1E250F8E1B60EF66EB40E25
:109E0800F76E000EF86E02EEA0F010EE40F00900BA
:109E1800F5CFEEFFE550E150FAE15A0EF66EBB0EB3
:109E2800F76E000EF86E01EEF1F010EE0CF009007E
:109E3800F5CFEEFFE550E150FAE1900EF66EBB0E5D
:109E4800F76E000EF86E0900F5CF54F004EE00F03E
:109E580018EE34F0EE6AE550E150FCE1E250FAE128
:109E680003EE00F011EE00F0EE6AE550E150FCE17F
:109E7800E250FAE102EE00F0A00EEE6AE806FDE11B
:109E880001EE00F0AB0EEE6AE806FDE10001FC6BA6
:109E980000EE4BF0090EEE6AE806FDE1559055928A
:109EA800000EF86E0001F2EF07F01D0E0001606F62
:109EB800F90E616FCECF62F0636BCDCF64F0656B46
:109EC8004FC066F0676B8AEC5DF00101FF834F506D
:109ED80028E1340E0B6E0A0E0C6EF30E0D6E010E99
:109EE8000E6E106A050E0F6EF8EC59F0390E0B6EF7
:109EF8000A0E0C6EA00E0D6E020E0E6E106A130E78
:109F08000F6EF8EC59F04C0E0B6E0A0E0C6EC60E66
:109F18000D6E020E0E6E106A0D0E0F6EF8EC59F0F3
:109F280027D0340E0B6E0A0E0C6EF80E0D6E010E55
:109F38000E6E106A050E0F6EF8EC59F0390E0B6EA6
:109F48000A0E0C6EB30E0D6E020E0E6E106A130E14
:109F58000F6EF8EC59F04C0E0B6E0A0E0C6ED30E09
:109F68000D6E020E0E6E106A0D0E0F6EF8EC59F0A3
:109F7800496A250E486EA4EC37F00101FF938390DF
:109F880012004F50140D070EF324D96E010EF42061
:109F9800DA6E000EDE24CD6F010EDE20CE6F000ECD
:109FA800DE20CF6F000EDE20D06F4F50140D070E4D
:109FB800F324D96E010EF420DA6ECDC0DEFFCEC0D8
:109FC800DEFFCFC0DEFFD0C0DEFF4F50140D070EFE
:109FD800F324D96E010EF420DA6EDECFD2F0DDCF95
:109FE800D3F0B90E606FF40E616FCECF62F0636B81
:109FF800CDCF64F0656BD2C066F0D3C067F0D2C035
:10A0080068F0D3C069F08AEC5DF04F50200D000E67
:10A01800F3240001A66F020EF420A76FD2C0A8F0A7
:10A02800D3C0A9F0AA6BAB6BDFEC12F0D16FD151A2
:10A0380010E00F0E606FFB0E616FD2C062F0D3C0EC
:10A0480063F0D1C064F0656B8AEC5DF0010E4D6E73
:10A05800010C4D6A1200B9C084F0BAC085F0876B54
:10A06800866B51EC36F0BE6FBE5102E0BE51120055
:10A07800B9C0D9FFBAC0DAFFDECF39F0DDCF3AF088
:10A0880020EE0EF0B951D926BA51DA22DECF3BF0D4
:10A09800DECF3CF0DECF3DF0DECF3EF0A5EC52F057
:10A0A8000001BE6FBE51E2E120EE12F0B951D9268F
:10A0B800BA51DA22DECFBCF0DDCFBDF0BCC0D9FF8B
:10A0C800BDC0DAFFDF50BB6FBB5103E1040EBE6FAA
:10A0D800CDD720EE0BF0BC51D926BD51DA22DFB620
:10A0E80016D0BCC00BF0BDC00CF020EE14F0B95176
:10A0F800D926BA51DA22DECF0DF0DDCF0EF0106A84
:10A108000B0E0F6E1EEC58F00B500C10AFE0B9C0E0
:10A11800A6F0BAC0A7F0A96BA86BD8EC25F000018F
:10A12800BE6FBE51A3E1A4D7B9C084F0BAC085F010
:10A13800876B866B51EC36F0C26FC25157E1C06B2A
:10A14800C16BB9C0D9FFBAC0DAFFDECF39F0DDCFB5
:10A158003AF020EE0EF0B951D926BA51DA22DECF04
:10A168003BF0DECF3CF0DECF3DF0DECF3EF0A5EC9D
:10A1780052F00001C26FC25139E120EE12F0B9511C
:10A18800D926BA51DA22DECFBDF0DDCFBEF0BDC090
:10A19800D9FFBEC0DAFFE50EDE1810E020EE12F09F
:10A1A800B951D926BA51DA22DECFBDF0DDCFBEF0E3
:10A1B800BDC0D9FFBEC0DAFFDF5009E1C04BC12BDB
:10A1C800BB51C01906E1BC51C11910E002D0C06BE7
:10A1D800C16BB9C0A6F0BAC0A7F0A96B010EA86FF1
:10A1E800D8EC25F00001C26FC251ABE0040EC219D1
:10A1F80002E1070EC26FC2511200C3C0B9F0C4C059
:10A20800BAF0BC6B010EBB6F98EC50F04A6E4A5026
:10A2180053E1C3C0D9FFC4C0DAFFDECF39F0DDCFC8
:10A228003AF020EE0EF0C351D926C451DA22DECF1F
:10A238003BF0DECF3CF0DECF3DF0DECF3EF0A5ECCC
:10A2480052F04A6E4A5038E1000120EE12F0C35134
:10A25800D926C451DA22DECF0BF0DDCF0CF00E6A1E
:10A268000D6A106A200E0F6E87EC5CF0000120EE7C
:10A2780012F0C351D926C451DA22DECF0BF0DDCF5C
:10A288000CF020EE14F0C351D926C451DA22DECFE7
:10A298000DF0DDCF0EF0106A0B0E0F6E7BEC5AF04E
:10A2A800C3C0D9FFC4C0DAFF10EE04F0DE50E126C7
:10A2B800DD50E222010EE76E4A5012001A0E0D24FC
:10A2C8000F6E000E0E20106E0F28D96E000E102093
:10A2D800DA6EDF50126E116A1A0E0D24D96E000E56
:10A2E8000E20DA6EDF50111211C017F012C018F0EC
:10A2F800196A1A6A0BC0D9FF0CC0DAFF030EDE1800
:10A3080029E1140E0D240F6E000E0E20106E0F287A
:10A31800D96E000E1020DA6EDF50126E116A140E1C
:10A328000D24D96E000E0E20DA6EDF501110136E58
:10A338001250146E156A166A14C016F013C015F080
:10A34800146A136A13501712145018121550191260
:10A3580016501A1217C00BF018C00CF019C00DF0E7
:10A368001AC00EF01200226E2250D8A4040C2050FD
:10A37800211001E1040C54B0030C50B608D0090EAA
:10A38800D8901C361D361E361F36E82EF9D72150B8
:10A3980006E1020E205C03E2246A110E02D0246A50
:10A3A800120E236E23C025F01CC014F01DC015F03A
:10A3B8001EC016F01FC017F025504AEC5BF00009CC
:10A3C8001DE11AC00BF01BC00CF0020E0E6E0D6AD8
:10A3D800C1EC57F0000908E0020E1B262006D8A0A1
:10A3E800210620502110EDE1120E251807E1146A0C
:10A3F800156A166A176A0C0E4AEC5BF0B9EC5DF048
:10A4080020502110D8A4010C000C155016100AE198
:10A418007CC115F07DC116F01550161003E1156AC0
:10A42800166A120015C00FF016C010F017C011F010
:10A4380018C012F092EC59F00F5015261050162241
:10A4480015C0D9FF16C0DAFFDF5006E101017C6BA9
:10A458007D6B156A166A120015C00FF016C010F051
:10A4680017C011F018C012F0B4EC59F00F501524B1
:10A4780001017C6F105016207D6F7CC1D9FF7DC112
:10A48800DAFFDF5009E07CC1D9FF7DC1DAFF000E99
:10A49800DF6A7C4B7D2B02D07C6B7D6B15C015F081
:10A4A80016C016F01200B96BBA6BACC0BBF0ADC0E9
:10A4B800BCF024D0B0C084F0B1C085F0B70E866F70
:10A4C800876B896B010E886FBD0E8A6F8B6BC9EC29
:10A4D80015F0BD05BE1125E1B7C0BFF00D0EBF19BF
:10A4E8000DE0BBC0D9FFBCC0DAFFBFC0DFFFBB4B6C
:10A4F800BC2BB94BBA2B0A0EBF1913E0B269B3696A
:10A50800AEC0B4F0AFC0B5F0B251B427B351B52363
:10A51800B451B95DBA51800AB66FB551800AB659BF
:10A52800C9E3BBC0D9FFBCC0DAFFDF6AB951BA11B1
:10A5380003E1AC6BAD6B1200ACC0ACF0ADC0ADF0DC
:10A548001200436A20EE2AF03950D9263A50DA220E
:10A558003B50DE1809E13C50DE1806E13D50DE189C
:10A5680003E13E50DE1839E039C024F03AC025F046
:10A5780003EC49F0436E435030E12E0E39241A6E35
:10A58800000E3A201B6E3BC01CF03CC01DF03DC0C5
:10A598001EF03EC01FF0216A010E206E20EE01F071
:10A5A8003950D9263A50DA22DF50B7EC51F0000979
:10A5B80006E03B683C683D683E68010E436E20EE4D
:10A5C8002AF03950D9263A50DA223BC0DEFF3CC087
:10A5D800DEFF3DC0DEFF3EC0DEFF43501200D4C0A8
:10A5E800DAF0D5C0DBF0DA0E0B6E68EC4BF00BC07E
:10A5F800DCF00CC0DDF00001DDBF0B0CD890DC35C1
:10A60800D96EDD35DA6E8C0ED926010EDA22DECF50
:10A61800D8F0DDCFD9F0D851D91105E0D8C0D9FF8D
:10A62800D9C0DAFFDF6AD251D31105E0D2C0D9FF11
:10A63800D3C0DAFFDF6AD890DC35D96EDD35DA6E43
:10A648008C0ED926010EDA22D2C0DEFFD3C0DDFF80
:10A65800D251D311D8B4000CD60501E0000CD20EAB
:10A668007C6F7D6BD40E7E6F7F6BAEEC00F0D76F86
:10A67800D751120003D00B4A0C2A0D2A0D50D96E5F
:10A68800DA6ADF500E6E0BC0F6FF0CC0F7FF000E43
:10A69800F86E0E0EF76403D00800F55005D0F6CF1B
:10A6A800E9FFF7CFEAFFEF500E1813E10BC0F6FFF2
:10A6B8000CC0F7FF000EF86E0E0EF76403D008000A
:10A6C800F55005D0F6CFE9FFF7CFEAFFEF500009C4
:10A6D800D2E10BC0F6FF0CC0F7FF000EF86E0E0EAD
:10A6E800F76403D00800F55005D0F6CFE9FFF7CF9F
:10A6F800EAFFEF500E6E0D50D96EDA6ADF500E5C2D
:10A708000B6E0C6AD8A00C0612000BC012F00CC01D
:10A7180013F00DC014F00EC015F00F06D8A01006E7
:10A728000F280CE110280AE10B6A0C6A1200124A81
:10A73800132A144A152A0F06D8A0100612C0F6FFCD
:10A7480013C0F7FF0800F55015E014C0D9FF15C075
:10A75800DAFFDF500FE00F5010100CE014C0D9FFE3
:10A7680015C0DAFF12C0F6FF13C0F7FFDE5009006C
:10A77800F518DDE012C0F6FF13C0F7FF0800F5CFAB
:10A7880011F014C0D9FF15C0DAFFDF50115C0B6E51
:10A798000C6AD8A00C0612000CC012F00DC013F001
:10A7A80012501310D8B4090C12C0D9FF13C0DAFF25
:10A7B800DE50DE10D8B4090C12C0D9FF13C0DAFF7E
:10A7C800DECF0EF0DDCF0FF00EC0D9FF0FC0DAFFDD
:10A7D800DF50D8B4090C20EE02F01250D9261350DD
:10A7E800DA2212C0E1FF13C0E2FF00EE06F0E650E5
:10A7F800E926E550EA22DE50EE1813E1DE50EE18A5
:10A80800D8A4090C12C0D9FF13C0DAFF10EE01F06A
:10A81800DE50E126DD50E222E750B3EC5DF00E6E2B
:10A828000EB0090C000C24EE04F0DE50DE10FBE044
:10A8380000C413F001C414F0060E1324D96E040EDC
:10A848001420DA6EDF50116E060E1324D96E060E30
:10A858001420DA6EDF50126E134A142A0D68010EA6
:10A868000E6E13C00FF014C010F00D500F160E50DE
:10A8780010160FC000F410C001F4F29E24EE04F08C
:10A88800DE06000EDD5AF28E0BC0D9FF0CC0DAFFCF
:10A8980012C0DFFF24EE04F0010EDBBE05D0000E6F
:10A8A800DE5C020EDE5801E28982115012000E5061
:10A8B80002E00E5003E10C506AEF5DF00E50D96EC5
:10A8C800DA6A040ED926DE50DE1014E00E50D96E76
:10A8D800DA6A040ED9260E50E16EE26A020EE1260B
:10A8E800DE50E65CE650800A136EDE50800A13588C
:10A8F800D8B012000E50D96EDA6A020ED926DECF11
:10A908000FF0DDCF10F00E50D96EDA6ADECF11F0FD
:10A91800DDCF12F00F501124D96E10501220DA6ECC
:10A928000CC0DFFF0E50D96EDA6A020ED926DE2A75
:10A93800000EDD22000C0B500F02F3CF13F0F4CF02
:10A9480014F0156A166A0B501002F3501426F450CE
:10A958001522000E16220C500F02F3501426F45044
:10A968001522000E16220B501102F3501526F45032
:10A9780016220C501002F3501526F45016220D50D2
:10A988000F02F3501526F450162212500B02F35002
:10A9980016260C501102F35016260D501002F350D3
:10A9A80016260E500F02F350162613C00BF014C0D3
:10A9B8000CF015C00DF016C00EF01200150E116E39
:10A9C800C60EE82EFED7112EFCD700D020D0150ECB
:10A9D800116EC60EE82EFED7112EFCD700D0010E40
:10A9E8000B6E0FC0F6FF10C0F7FF000EF86E0E0ECC
:10A9F800F76403D00800F55005D0F6CFE9FFF7CF8C
:10AA0800EAFFEF5045EC59F00F4A102AD7D70FC08C
:10AA1800F6FF10C0F7FF000EF86E0E0EF76403D0B5
:10AA28000800F55005D0F6CFE9FFF7CFEAFFEF5061
:10AA38000009CDE11200F70E0001606FFA0E616F98
:10AA4800CECF62F0636BCDCF64F0656B8AEC5DF0BE
:10AA5800486A496A4F50140D070EF324D96E010E47
:10AA6800F420DA6EDE6ADE6ADE6ADD6A4F50140DA3
:10AA7800130EF324D96E010EF420DA6EDF6A4F50FC
:10AA8800140D0F0EF324D96E010EF420DA6EDE6A6F
:10AA9800DE6ADE6ADD6A484A492A49BEDBD7495080
:10AAA80003E1040E485CD6E383904D6A1200136AF2
:10AAB800146A156A166A0F5010101110121029E046
:10AAC800010E176E06D0D8900F3610361136123692
:10AAD800172A12AEF8D7D89013361436153616360C
:10AAE8000F500B5C10500C5811500D5812500E5846
:10AAF80009E30F500B5E10500C5A11500D5A1250AA
:10AB08000E5A1380D8901232113210320F32172E8B
:10AB1800E2D713C00BF014C00CF015C00DF016C02E
:10AB28000EF012004C6A4B6A0101866B876B020EAD
:10AB3800966F8390956B946B4F6A030E4F6401D0A8
:10AB480029D04F50070D520EF324D96E010EF42070
:10AB5800DA6EDF6A4F50070D510EF324D96E010EDD
:10AB6800F420DA6EDF6A4F50070D500EF324D96EC9
:10AB7800010EF420DA6EDF6A4F50070D530EF324EE
:10AB8800D96E010EF420DA6EDE6ADE6ADE6ADD6AEC
:10AB98004F2AD3D74F6A1200F30E0001606FFE0EE2
:10ABA800616F8AEC5DF04F6A030E4F6401D029D0C3
:10ABB8004F50070D520EF324D96E010EF420DA6EB1
:10ABC800DF6A4F50070D510EF324D96E010EF420A1
:10ABD800DA6EDF6A4F50070D500EF324D96E010E5E
:10ABE800F420DA6EDF6A4F50070D530EF324D96E46
:10ABF800010EF420DA6EDE6ADE6ADE6ADD6A4F2A4A
:10AC0800D3D74F6A83900101966B1200E0EC43F0B2
:10AC1800CDC0E8F0CEC0E9F0E851E91105E0E8C0A0
:10AC2800E4F0E9C0E5F012008FB414D04F50200DC5
:10AC3800000EF324A66F020EF420A76F000EA86F73
:10AC4800030EA96F010EAB6FAA6BE60EAC6F71EC29
:10AC58000FF0EC6FEC510EE0800E606FFD0E616F2F
:10AC6800ECC062F0636B8AEC5DF0ECC0E4F00001CC
:10AC7800E56B1200C5EC4FF00001E46BE56B1200C8
:10AC8800136E0C0E131807E0B9EC5DF047EC5DF09D
:10AC9800000901E1FF0C135040099DEC5DF01050D4
:10ACA8009DEC5DF00F509DEC5DF00E509DEC5DF05D
:10ACB8000D509DEC5DF0010E126E135002E1950EE1
:10ACC800126E080E131802E1870E126E12509DECD8
:10ACD8005DF00C0E131802E1A6EC5DF00A0E126E80
:10ACE800A6EC5DF0116E11AE02D0122EF9D71150FC
:10ACF8001200570E0001606FFE0E616F8AEC5DF066
:10AD08000001886B896B876B23D00DEC5DF00B50CD
:10AD18000C1012E0870E0B6E0C6A17EC54F0000151
:10AD2800866F000E5324D96EDA6A030EDA2286C0C3
:10AD3800DFFF532A884B892B000187AB07D0000E11
:10AD48008825486E040E8921496E12008EAC04D005
:10AD580089BFDBD78905D9E388C048F089C049F0A5
:10AD6800120011D0030E0BD0050E0D6E0101886B79
:10AD7800896B2DD00A0E03D0010E01D0020E0D6E84
:10AD880026D00D6A24D088C10BF089C10CF00C5074
:10AD980009E0020A0DE00E0A0FE0010A11E02A0A92
:10ADA80013E0EFD70B500A0ADDE01E0ADDE0E9D711
:10ADB8000B50BC0AE3E0E5D70B501C0ADBE0E1D7F7
:10ADC8000B50AC0AD9E0DDD70B500F0ADAE10D5071
:10ADD80012000F501010D8B4000C0FC0D9FF10C0CB
:10ADE800DAFFDF5001E1000C0FC00BF010C00CF0CF
:10ADF8003AEC5AF00BC011F00CC012F0020E111808
:10AE0800121001E0000C130E0B6E0FC0D9FF10C01A
:10AE1800DAFFDF501CEC59F00009D8B4000C140E0E
:10AE28000B6E20EE01F00F50D9261050DA22DF50B9
:10AE38001CEC59F0000901E1000C1338F00B141058
:10AE48001200866A846A8B688968536A839283943D
:10AE58000101926B936B09D0000E9225D96E030EF7
:10AE68009321DA6EDF6A924B932B93BFF5D7930544
:10AE7800F3E3926B936B09D0340E9225D96E0A0EC8
:10AE88009321DA6EDF6A924B932B93BFF5D7930524
:10AE9800F3E30F011769D6501F0B4009D66ED698F9
:10AEA8000F0ED612D588D5120E01C29BD58E0F0C67
:10AEB800D6EC5AF0CC0E3AEC5DF0660E3AEC5DF04A
:10AEC8001DEC5DF0156E155005E10F6A106A116AE8
:10AED800126A1200136A146A1350150FD96EDA6ACF
:10AEE8001DEC5DF0DF6E134A142A14BEF5D714501A
:10AEF80003E1040E135CF0E318501710161003E179
:10AF0800060E155CE2E315C00FF016C010F017C06E
:10AF180011F018C012F012000F501010111012107A
:10AF280023E0010E136E06D0D8900F361036113676
:10AF38001236132A12AEF8D70F500B5C10500C586B
:10AF480011500D5812500E5808E30F500B5E105058
:10AF58000C5A11500D5A12500E5AD8901232113202
:10AF680010320F32132EE8D70BC00BF00CC00CF0C8
:10AF78000DC00DF00EC00EF01200070E106ED00EB0
:10AF88000F6E0FD0A6EC5DF0116E11280DE1E40EE6
:10AF980000D000D0E82EFCD700D000D00F06D8A0F3
:10AFA80010060F501010EEE1FE0E111801E0000C13
:10AFB800A6EC5DF00BC0D9FF0CC0DAFFDF6E0B4AC0
:10AFC8000C2A0D06D8A00E060D500E10F1E1A6ECC5
:10AFD8005DF0A6EC5DF0010C1B0E0001606FFD0E2C
:10AFE800616F8AEC5DF083800101FF832AEE34F003
:10AFF80094C1DFFF000EE8CF35FA0D0EE8CF36FA20
:10B00800000EE8CF37FA8FA403D0600EE8CF37FAE6
:10B018008FA406D036CA4AF0200E4A124AC036FA21
:10B02800496A040E486EA4EC37F00101FF93946B53
:10B03800839012000BC012F00CC013F00DC014F076
:10B048000EC015F0166A176A0F06D8A010060F284A
:10B0580002E1102817E012C0D9FF13C0DAFF124A24
:10B06800132ADF50116E14C0D9FF15C0DAFF144A35
:10B07800152ADF50115C166E176AD8A017061650ED
:10B088001710E2E016C00BF017C00CF012000BC04E
:10B0980011F00CC012F013D00F06D8A010060DC086
:10B0A800D9FF0EC0DAFF0D4A0E2A11C0E1FF12C007
:10B0B800E2FF114A122ADFCFE7FFE7500BE00F50FB
:10B0C800101008E0E9D711C0D9FF12C0DAFFDF6A13
:10B0D800114A122A0F06D8A010060F28F4E11028EA
:10B0E800F2E1120081EC5BF0000901E1000C0F5065
:10B0F8009DEC5DF0FD0E0F181EE0020E116E106A39
:10B108000DC0D9FF0EC0DAFFDF509DEC5DF00D4A8F
:10B118000E2A1006D8A0110610501110F1E1A6EC65
:10B128005DF0A6EC5DF0A6EC5DF0126E12501F0B00
:10B13800050A01E0000C010C15D00CC0F6FF0DC08B
:10B14800F7FF000EF86E0E0EF76403D00800F550F6
:10B1580005D0F6CFE9FFF7CFEAFFEF5075EC5DF0C9
:10B168000C4A0D2A0CC0F6FF0DC0F7FF000EF86E52
:10B178000E0EF76403D00800F55005D0F6CFE9FFAE
:10B18800F7CFEAFFEF500009D8E112000EC012F025
:10B198000FC013F010C014F011C015F0D6EC5AF01F
:10B1A800CC0E3AEC5DF0990E3AEC5DF00C0E3AECF0
:10B1B8005DF0166A176A1650120FD96EDA6ADF50F8
:10B1C8003AEC5DF0164A172A17BEF5D7175002E079
:10B1D800D6EF5AF0040E165CEEE3D6EF5AF00001F3
:10B1E800876FED0E886FF30E896F866B0AD088C063
:10B1F800F6FF89C0F7FF884B892B0800F550F7E167
:10B20800862B8751861907E088C0F6FF89C0F7FFAB
:10B218000800F550ECE1730E606FFE0E616F87C099
:10B2280062F0636B88C064F089C065F08AEF5DF0F6
:10B238000C6E0B5001E1000C2F0E0C6409D03A0E75
:10B248000C6006D00B50D96EDA6A0C50D00F17D0AC
:10B25800400E0C6409D0470E0C6006D00B50D96E16
:10B26800DA6A0C50C90F0BD0600E0C64000C670E24
:10B278000C60000C0B50D96EDA6A0C50A90FDF6E07
:10B28800010C0C6E87920A0EE82EFED700D00BB088
:10B2980002D0879401D08784000E0E6E010E0D6EC9
:10B2A8000CAE02D0838A01D0839AD8900C3687904E
:10B2B80000F000F0878000F000F087900D4A0E2A19
:10B2C8000EBEEED70E5003E1090E0D5CE9E387824E
:10B2D8001200010E0B6E0C6A88868782878400F044
:10B2E80000F0879400F000F00D6A0E6A8DA602D077
:10B2F8000B500C12D8900B36879000F000F0878026
:10B3080000F000F087900D4A0E2A0EBEEFD70E50BF
:10B3180003E1030E0D5CEAE30C501200136A146A91
:10B3280004D00F4A102A134A142A0FC0D9FF10C09C
:10B33800DAFFDF5010E011C00BF012C00CF00FC0A4
:10B34800D9FF10C0DAFFDF500D6E0E6AB6EC5BF065
:10B358000B500C10E6E113C00FF014C010F01200EF
:10B36800136A146A04D00F4A102A134A142A0FC009
:10B37800D9FF10C0DAFFDF5010E011C00BF012C087
:10B388000CF00FC0D9FF10C0DAFFDF500D6E0E6A47
:10B39800B6EC5BF00B500C10E6E013C00FF014C0D5
:10B3A80010F012009F0E136E146811C015F012C031
:10B3B80016F01350152614501622165005E11A0ED1
:10B3C800155C02E2010E01D0000E176E186A1750C4
:10B3D800181005E05F0E1114116E126A120011C0E8
:10B3E80011F012C012F012000DC013F00EC014F0CC
:10B3F8000BC011F00CC012F010D013C0D9FF14C04C
:10B40800DAFFDF50156E134A142A11C0D9FF12C093
:10B41800DAFF15C0DFFF114A122A0F06D8A010065E
:10B428000F28EBE11028E9E1120020EE1AF00B508A
:10B43800D9260C50DA220DC0DFFF20EE1BF00B508E
:10B44800D9260C50DA220EC0DFFF20EE14F00B5084
:10B45800D9260C50DA220FC0DFFF20EE15F00B5072
:10B46800D9260C50DA221050DF6E12000BC00DF0F6
:10B478000CC00EF002D00B4A0C2A0BC0F6FF0CC011
:10B48800F7FF000EF86E0E0EF76403D00800F550B3
:10B4980005D0F6CFE9FFF7CFEAFFEF500009EBE15F
:10B4A8000D500B5C0B6E0E500C580C6E1200000702
:10B4B80095810100400001000300005001F40101E2
:10B4C80000000795810100400001000300005001C1
:10B4D800F401010000062305003E000000091127C1
:10B4E8000000062305003E000000091127000BC0DC
:10B4F80011F00CC012F00DC013F00EC014F00ED0F5
:10B5080013C0D9FF14C0DAFF11C0E1FF12C0E2FF77
:10B51800DFCFE7FF134A142A114A122A0F06D8A0D0
:10B5280010060F28EDE11028EBE11200280E0001AB
:10B53800606FFF0E616F8AEC5DF0340E0B6E0A0EC1
:10B548000C6E0E6A0D6A010E106E0F6A3CEC4AF022
:10B558002AEE34F096C1DFFF496A010E486EA4EC6A
:10B5680037F00101966B12000B6E0B500EE0BDEC2C
:10B578005DF0200EE82EFED7C0EC5DF0CC0E00D0BA
:10B58800E82EFDD700D000D01200BDEC5DF0C00E53
:10B5980000D0E82EFDD7C0EC5DF0350EE82EFED7C2
:10B5A80000F01200BDEC5DF00A0E0C6EF80EE82EED
:10B5B800FED70C2EFCD700D0C0EC5DF0E00E00D01A
:10B5C800E82EFDD794EC5DF00D6E090E0C6E840E1E
:10B5D800E82EFED70C2EFCD7C0EC5DF00D50120003
:10B5E800730E776F6FC078F070C079F07A6B7B6BF1
:10B5F8007C6B7D6B780E696F71C06AF072C06BF0FE
:10B60800770E6C6FCBEC23F000017A516F25D96E61
:10B618007B517021DA6EDF6A000C000EF2BE010E5B
:10B628000E6E0C50030B7F6E0BC07EFF0DC080FFAB
:10B638003F0E81168184F29E550E826EAA0E826E8E
:10B64800818281B2FED781940EB002D0F29E01D0E1
:10B65800F28E120002D00B4A0C2A0BC0F6FF0CC067
:10B66800F7FF0800F55009E00BC0F6FF0CC0F7FF24
:10B678000800F5500D180E10EEE10BC0F6FF0CC0D7
:10B68800F7FF0800F5500B6E0C6A1200186E18AE22
:10B698000ED0189E0D6A0E6A0F6A106A370E44ECB7
:10B6A80056F0196E010E196402D01950120014C018
:10B6B8000DF015C00EF016C00FF017C010F018509E
:10B6C80044EF56F0010E116E200E0B180C1011E00D
:10B6D800F70E0D6E0E680BC00FF00CC010F00D5079
:10B6E8000F260E501022105003E1050E0F5C01E3E7
:10B6F800116A11C00BF00C6A1200130E0C6E880E42
:10B708000B6E0ED0A6EC5DF0FF0A0DE0E40E00D043
:10B7180000D0E82EFCD700D000D00B06D8A00C062D
:10B728000B500C10EFE10B500C10D8A4010C000CBE
:10B7380048C046F049C047F0C4EC40F04A6E4A5051
:10B748000FE148C00CF049C00DF0D0EC53F04A6E40
:10B758004A5006E148C0D9FF49C0DAFFDE6ADD6A0F
:10B768004A5012000BC0F6FF0CC0F7FF0800F55056
:10B778000D1805E10BC00BF00CC00CF012000BC04B
:10B78800F6FF0CC0F7FF0B4A0C2A0800F550EAE157
:10B798000B6A0C6A120060900F0E0F01596F070EAA
:10B7A800396F356F4F0E936E8A6A8A888A828A82C9
:10B7B800010E8F6E130E0E01B76F0F0EFA6F100E7B
:10B7C800FC6F140EB86F140C9F0E0D6E0E68200ED1
:10B7D8000B100F6E000E0C10106E0D500F260E5031
:10B7E8001022105005E11A0E0F5C02E2010E01D082
:10B7F800000E0B6E0C6A12009F869E84090E0E01C5
:10B80800FD6F9F98890E9B6E9C6A9E989D8E9D8861
:10B818009D9AC599F28AF28E9E909D9C9E9A9E8AC8
:10B82800010199911200340E0B6E0A0E0C6E0E6A0D
:10B838000D6A010E106E0F6A3CEC4AF0010EE8CF5B
:10B8480034FA0101FF83496A486EA4EC37F001011C
:10B85800FF931200186A196A09D017C00CF00D6A14
:10B8680016C00EF05BEC54F0184A192A185014242C
:10B87800D96E19501520DA6EDF50176E1750EDE1AA
:10B8880012009F0E0D6E0E680BC00FF00CC010F06A
:10B898000D500F260E501022105005E11A0E0F5CA5
:10B8A80002E2010E01D0000E0B6E0C6A1200BF0EF0
:10B8B8000D6E0E680BC00FF00CC010F00D500F2667
:10B8C8000E501022105005E11A0E0F5C02E2010E14
:10B8D80001D0000E0B6E0C6A1200D00E0D6E0E68B1
:10B8E8000BC00FF00CC010F00D500F260E50102298
:10B8F800105005E10A0E0F5C02E2010E01D0000EA5
:10B908000B6E0C6A12000BC011F00CC012F008D0BC
:10B9180011C0D9FF12C0DAFF0DC0DFFF114A122A89
:10B928000F06D8A010060F28F3E11028F1E1120045
:10B93800106A110E0F6E09D00A0EE82EFED700D03D
:10B94800010E0B6E200E45EC59F00F06D8A010061C
:10B958000F28F2E11028F0E112000B6E0B5009E0FD
:10B96800966A4F0E936E220E966E400E956E968ACC
:10B97800400C966A100E966E2A0E966E900E936E76
:10B98800F4D78380010E4D6E3F0E0001606FFB0EF1
:10B99800616FCECF62F0636BCDCF64F0656B8AECDC
:10B9A8005DF083904D6A1200BDEC5DF0200EE82E2C
:10B9B800FED7C0EC5DF0300EE82EFED794EC5DF0BB
:10B9C8000C6EB00E00D0E82EFDD70C50120083800C
:10B9D8002C0E0001606FFA0E616FCECF62F0636BC0
:10B9E800CDCF64F0656B8AEC5DF04D6A83901200F0
:10B9F8009150070B0B6E888A8DAA02D0080E0B2671
:10BA0800020E01019C1903E10B1C0F0B0B6E0B506E
:10BA1800120024EE04F0010EDBBE05D0000EDE5C41
:10BA2800020EDE5801E2898204C40BF005C40CF052
:10BA380012000D6A0E6AD8900D32D8EC5CF000093D
:10BA480001E00D8E0E2A070E0E64F5D70D50120078
:10BA5800000EE8CF00F4E8CF01F4E8CF02F4E8CF15
:10BA680003F4E8CF04F4E8CF05F4000C0C6E0D6A7B
:10BA78000C50010BB8EC5AF0D8900C320D2A070E76
:10BA88000D64F6D7070CC5EC5DF0A6EC5DF081EC13
:10BA98005BF0000901E0010CB9EC5DF0000C0C5002
:10BAA800030B7F6E0BC07EFF3F0E8116818000F076
:10BAB80000F080501200CF0E0001606FFE0E616F23
:10BAC8008AEC5DF083900101966B12000B6E03D037
:10BAD800C7EC5DF004000E01CDA9FAD70BC09AFFA0
:10BAE80012000B6E03D0C7EC5DF004000E01CDA967
:10BAF800FAD70BC09AFF12000B6E02D0838C839C7E
:10BB08000B060B28FBE100F000F01200620E476EF6
:10BB180060C018F061C019F0470E1A6E9DEF29F049
:10BB280088888DA803D0010E0B6E01D00B6A0B50CC
:10BB380012000B6E0BC092FF95B0FED795A0FED7F2
:10BB480092501200926895B0FED795A0FED79250F9
:10BB580012001FE7800103E800800103E8000B6E74
:10BB68000B5001E0010C54501200C3EC5DF0A6EF3D
:10BB78005DF08398889812008398888812008580E1
:09BB880012008590120012000168
:10F3EC00004F4B004449534B5F455252004E4F5413
:10F3FC005F5245414459004E4F5F46494C45004EC3
:10F40C004F545F4F50454E4544004E4F545F454E50
:10F41C0041424C4544004E4F5F46494C455F535961
:10F42C005354454D000020000D0A2025325820254C
:10F43C003258202532732025327320253273202533
:10F44C003273202532732025327320253273202508
:10F45C0032732025347320253473202534732025F2
:10F46C0034732025347320253473202534732025E0
:10F47C00347320000D0A2530325825303258205371
:10F48C005338303A53657420537461747573206D1E
:10F49C0061736B202558202558202558202558208D
:10F4AC00255820255820255820255820000D0A25A0
:10F4BC003032582530325820535338303A20496E68
:10F4CC006372656D656E743A205365656B696E6722
:10F4DC0020746F20256C752028256C582920000D70
:10F4EC000A48504469736B204D6B204949202831E0
:10F4FC00384634364B34302920257320257320258B
:10F50C0073205374617274696E672E2E2E0D0A006F
:10F51C000D0A253032582530325820414D3A556E5F
:10F52C006275666620726420632F682F733A2025FB
:10F53C00642F25642F256420733A256C6420000DFC
:10F54C000A25303258253032582052656365697669
:10F55C0065642052544320627974657320253258B7
:10F56C0020253258202532582025325820000D0AEB
:10F57C0025303258253032582053656E64696E67D9
:10F58C00205254432062797465732025325820250B
:10F59C003258202532582025325820000D0A2530AB
:10F5AC003258253032582053533830783A536565E9
:10F5BC006B3A205365656B696E6720746F20256C00
:10F5CC00752028256C582920000D0A253032582525
:10F5DC0030325820414D3A4275666620777220636E
:10F5EC002F682F733A2025642F25642F25642073F0
:10F5FC003A256C64000D0A52656365697665642072
:10F60C005254432062797465732025325820253278
:10F61C0058202532582025325820000D0A414D3AE9
:10F62C00556E6275666620777220632F682F733A69
:10F63C002025642F25642F256420733A256C6420C3
:10F64C00000D0A25303258253032582053533830AB
:10F65C003A4275666620777220256C642062797454
:10F66C00657320727820000D0A53656E64696E67AD
:10F67C00205254432062797465732025325820251A
:10F68C003258202532582025325820000D0A547249
:10F69C0069656420746F2074616C6B207768696C89
:10F6AC007374206E6F742061646472657373656427
:10F6BC00000D0A414D3A4275666620726420632F34
:10F6CC00682F733A2025642F25642F256420733A04
:10F6DC00256C6420000D0A25303258253032582014
:10F6EC00313A526561642072746E2025582C2025A5
:10F6FC0064207265616420000D0A25303258253073
:10F70C0032582053533830783A5772697465202533
:10F71C006C642028256C582920000D0A253032589D
:10F72C00253032582053533830783A5374617475FD
:10F73C00732C20756E697420256420000D0A253009
:10F74C003258253032582053533830783A5265614C
:10F75C006420256C752028256C582920000D0A255D
:10F76C003032582530325820535338303A53657460
:10F77C00206164647265737320256C5820000D0A37
:10F78C00253032582530325820535338303A43689C
:10F79C0020696E6420436C65617220256420000D25
:10F7AC000A4D617820566563746F72206469736BBF
:10F7BC0020256420256C642028256C582920000DF8
:10F7CC000A25303258253032582053533830783A85
:10F7DC005374617475735B25645D20255820000D8E
:10F7EC000A253032582530325820535338303A538A
:10F7FC0065742072656C6561736520255820000D59
:10F80C000A253032582530325820535338303A5369
:10F81C006574206C656E67746820256C5820000D2B
:10F82C000A253032582530325820535338303A415B
:10F83C006D69676F20436C65617220256420000D33
:10F84C000A253032582530325820535338303A5329
:10F85C00657420766F6C756D6520256420000D0A2B
:10F86C00253032582530325820535338303A466FB1
:10F87C00726D617420706172616D7320000D0A41AC
:10F88C004D3A5365656B3A20256420256420256428
:10F89C002025642C20733A256C64000D0A25303227
:10F8AC00582530325820535338303A527074205106
:10F8BC005354415420256420000D0A44736B736526
:10F8CC006C2069732025642C206E756D6265722026
:10F8DC00697320256420000D0A52656164207274DE
:10F8EC006E2025582C202564206279746573207253
:10F8FC00656164000D0A253032582530325820538A
:10F90C005338303A53657420756E69742025642021
:10F91C00000D0A25303258253032582053533830D8
:10F92C00783A4465736372207520256420000D2598
:10F93C003032582530325820566563746F7220254A
:10F94C006C642028256C582920000D0A253032586B
:10F95C002530325820535338303A556E6B6E6F77D2
:10F96C006E20255820000D0A414D3A556E62756681
:10F97C006620777220256420627974657320727812
:10F98C00000D0A2530325825303258205353383068
:10F99C003A43616E63656C20256420000D0A2530A6
:10F9AC0032582530325820535338303A496E6974E6
:10F9BC00206469736B20000D0A25303258253032D3
:10F9CC005820535338303A527120737461747573E4
:10F9DC0020000D0A414D3A20496E63723A2025648D
:10F9EC002025642025642025642C20000D0A253058
:10F9FC0032582530325820256C6420627974657336
:10FA0C002073656E74000D0A25303258253032583B
:10FA1C0020535338303A4465736372696265200031
:10FA2C000D0A25303258253032582053533830784F
:10FA3C003A466D74206F70747300466F756E642057
:10FA4C00616E205254432066696C652061742025D8
:10FA5C00580D0A004C6F6F6B696E6720666F7220D1
:10FA6C00616E205254432066696C650D0A000D0AC4
:10FA7C005573696E67206469736B2067656F6D657C
:10FA8C0074727920257320000D0A414D3A42756637
:10FA9C0066207772202564206279746573207278F1
:10FAAC000046696E6446696C65206661696C6564C4
:10FABC00207365617263680D0A0025303258253059
:10FACC00325820256C642062797465732073656EDE
:10FADC007420000D0A475049422072633A25642075
:10FAEC0025642062797465730D0A000D0A25303285
:10FAFC0058253032582053533830783A436C65616E
:10FB0C007220000D0A5365656B20746F20256C64A0
:10FB1C00206661696C6564202564000D0A57726962
:10FB2C0074655F736563746F7273206661696C20B2
:10FB3C002564000D0A253032582530325820535395
:10FB4C003830783A466F726D6174000D0A446973EF
:10FB5C006B2073656C656374206E756D62657220C5
:10FB6C002564000D0A5365656B696E6720746F2000
:10FB7C00256C642028256C5829005365656B696ECB
:10FB8C006720746F20736563746F722025580D0A9B
:10FB9C000046696E6446696C65206661696C6564D3
:10FBAC0020726561640D0A000D0A2530325825302B
:10FBBC00325820535338303A577269746520000D0F
:10FBCC000A4F70656E696E67206578697374696E2B
:10FBDC006720257320000D0A476F7420256C752053
:10FBEC00202D20726573657474696E67000D0A258B
:10FBFC003032582530325820535338303A526561E0
:10FC0C006420000D0A2530325825303258205353C9
:10FC1C0038303A44534A20000D0A253032582530EA
:10FC2C00325820535338303A4E4F5020000D0A545E
:10FC3C0052616E20457865632025582020202020B5
:10FC4C00004469736B206368616E67653A202564B4
:10FC5C0020200D0A000D0A57616974696E672066D1
:10FC6C006F72206361726420003C6964656E743E3F
:10FC7C00202558202558202564202564000D566524
:10FC8C0063746F7220256C642028256C5829200021
:10FC9C000D0A46696C65202573206973206F7065A9
:10FCAC006E20000D0A57726F7465206469736B6E59
:10FCBC006F3A202564000D0A20256C64206279744B
:10FCCC0065732073656E74000D0A52656164206261
:10FCDC0065796F6E6420656E64000D0A5365656B03
:10FCEC00206265796F6E6420656E64000D0A4F703A
:10FCFC00656E696E67206E657720257320000D0A8E
:10FD0C002530325825303258204578697420000D42
:10FD1C000A414D3A53656E642073746174757300B7
:10FD2C004E6F742061204C4946206469736B0D0A38
:10FD3C00000D0A52656164206465736372696265C3
:10FD4C0020000D0A46696C65202558206973202512
:10FD5C007320000D0A4469736B20255820697320A9
:10FD6C00257320000D0A4873742062797465733210
:10FD7C00202564000D0A5772697465206661696CF0
:10FD8C00202564000D0A52656164696E6720525427
:10FD9C00430D0A000D0A416D69676F20393132310C
:10FDAC00440D0A000D0A44736B73656C2069732053
:10FDBC00256420000D0A5265616420256420627957
:10FDCC00746573000D0A487374206279746573202E
:10FDDC00256400566563746F722069732025580D75
:10FDEC000A00222A2B2C3A3B3C3D3E3F5B5D7C7F3C
:10FDFC00000D0A4F70656E696E6720257320200018
:10FE0C000D0A446562756720697320256420000D16
:10FE1C000A50726F746F20697320256420000D0ADC
:10FE2C005265616420636F6E66696720000D0A4637
:10FE3C00696C656E616D6520257320002041544E00
:10FE4C0020617373657274656420000D0A526563DA
:10FE5C006569766532353620000D0A466F726D6124
:10FE6C007474696E67200072633D25752046525F7D
:10FE7C0025730D0A000D0A736279746573312025A0
:10FE8C0064000D0A4E6F2063617264202564006467
:10FE9C00657363726962652E636667002F6C6966B1
:10FEAC00646174612E62696E000D0A2573202558F9
:10FEBC002025580D0A007B505025642025642025F0
:10FECC00647D000D0A414D3A57616B657570000DEC
:10FEDC000A4D6F756E74696E672000536570203122
:10FEEC00332032303230000D0A414D3A436C65619B
:10FEFC0072004C6F6164696E672E2E2E0068706400
:10FF0C0069736B2E63666700466D7420657869743F
:10FF1C0020005B535251206F66665D000D0A414D07
:10FF2C003A44534A0031383A30373A3536005B257B
:10FF3C0032582025645D005B535251206F6E5D007A
:10FF4C0048504469736B20004E6F206361726400EB
:10FF5C0072633D256420002D3E202558200044531B
:10FF6C004B53454C004E414D452558004449534B8D
:10FF7C002558005B4D4C415D0044454255470050AF
:10FF8C00524F544F0052656164790020253032582D
:10FF9C00007B4552527D00302E31330049464320C0
:10FFAC0000454F49200052454E200041544E200040
:10FFBC00535251200044415620004E444143004EC0
:10FFCC005246440052544300434C4B0020255800E9
:10FFDC0025325800207C200044300044310044324B
:10FFEC0000443300443400443500443600443700A8
:04FFFC002563000079
:020000040020DA
:10000000FF0FFF0FFF0FFF0FFF0FFF0FFF0FFF0F80
:020000040030CA
:0C0000008CFFFFFF8EFFFFFFFFFFFFFFE4
:00000001FF
